:020000040801F1
:1000000098B7002039010108094101080B41010896
:100010003141010835410108394101080000000063
:10002000000000000000000000000000F5FB0108D7
:100030003D4101080000000061FC010871FC01085D
:10004000530101085301010853010108DD6C010847
:10005000530101085301010853010108530101082C
:10006000530101085301010853010108530101081C
:10007000530101085301010853010108530101080C
:1000800053010108530101085301010853010108FC
:1000900053010108530101085301010853010108EC
:1000A00053010108530101085301010853010108DC
:1000B000B358010853010108530101085301010815
:1000C00053010108530101085301010853010108BC
:1000D0005301010893430108D1580108C54F010895
:1000E000EB6D01086D6C0108530101085301010813
:1000F000530101085301010853010108530101088C
:10010000F97001086D7D01085301010853010108D0
:10011000530101085301010853010108530101086B
:1001200053010108DFF80CD010F0B8FA004800477E
:10013000793D010898B700200648804706480047E7
:10014000FEE7FEE7FEE7FEE7FEE7FEE7FEE7FEE787
:10015000FEE7FEE7B73F01082501010832490143E8
:10016000324A1160704770B5002100230F22C47815
:100170001CB32E4C246804F4E064C4F5E064C4F3BA
:100180000721C1F10404E3B20A4144789C40E1B282
:100190008478144021430C07210E254C05786155C5
:1001A000047804F01F050124AC4005786D11AD0002
:1001B00005F1E025C5F8004109E0047804F01F05C9
:1001C0000124AC401B4D0678761145F8264070BDE1
:1001D000194A0A400243154B1B1F1A60704739B178
:1001E000124A121D12680243104B1B1D1A6006E0D2
:1001F0000E4A121D126882430C4B1B1D1A60704779
:10020000042808D14FF0E021096941F004014FF0C2
:10021000E022116107E04FF0E021096921F00401BB
:100220004FF0E022116170470000FA050CED00E08C
:1002300000E400E080E100E080FFFF1F10B504460D
:10024000FE48844207D10121401500F09FFE0021A5
:10025000601500F09BFE10BD30B502460020002363
:100260005068F74C20400D790C6844EA052420437F
:1002700050609068F34C2040D1E903542C438D68C2
:100280002C434D7944EA450420439060106B20F0E4
:10029000F8700C7D641EE4B2234340EA03501063FF
:1002A00030BD002101600171417181604FF04071EA
:1002B000C1600021016101210175704701460020E4
:1002C000E14A106820F440300A681043DE4A1060AA
:1002D000704700210160704721B1826842F001023D
:1002E000826003E0826822F001028260704721B1DF
:1002F000826842F00402826003E0826822F0040215
:10030000826070471AB143680B43436002E0436860
:100310008B43436070470A460021816821F0F00159
:100320001143816070470A4600214168C74B19405C
:100330001143416070478162C26270470A460021E2
:10034000416821F01F0111434160704730B1BE493F
:10035000096841F40001BC4A116005E0BA49096826
:1003600021F40001B84A11607047F0B504460D460B
:10037000002000211D2D11DDE06DA5F11E0606EB0C
:100380004607072606FA07F18843A5F11E0606EB85
:10039000460603FA06F10843E06534E0132D11DD4B
:1003A000E068A5F1140606EB4607072606FA07F1F2
:1003B0008843A5F1140606EB460603FA06F1084346
:1003C000E06020E0092D11DD2069A5F10A0606EBA9
:1003D0004607072606FA07F18843A5F10A0606EB49
:1003E000460603FA06F1084320610CE0606905EB5C
:1003F0004507072606FA07F1884305EB450603FA89
:1004000006F108436061072A0FDA206C561E06EBDE
:1004100086071F2606FA07F18843561E06EB860656
:1004200005FA06F1084320644AE00D2A0FDAE06B72
:10043000D61F06EB86071F2606FA07F18843D61F4C
:1004400006EB860605FA06F10843E06338E0132A56
:1004500011DAA06BA2F10D0606EB86071F2606FA3D
:1004600007F18843A2F10D0606EB860605FA06F1B0
:100470000843A06324E0192A11DA606BA2F1130685
:1004800006EB86071F2606FA07F18843A2F113063A
:1004900006EB860605FA06F10843606310E0206B60
:1004A000A2F1190606EB86071F2606FA07F1884314
:1004B000A2F1190606EB860605FA06F10843206349
:1004C000F0BD816841F080418160704701460020A5
:1004D0008A6802F080420AB1012000E000207047E3
:1004E00021B1826842F48062826003E0826822F473
:1004F00080628260704721B1826842F002028260AD
:1005000003E0826822F002028260704710B50A465A
:1005100000210023416821F46041531E41EA433128
:10052000416010BD21B1426842F40062426003E0C4
:10053000426822F40062426070470146886D80B2D2
:10054000704721B1826842F48072826003E0826861
:1005500022F480728260704721B1826842F4007296
:10056000826003E0826822F4007282607047F0B516
:10057000044615460020002200261D2911DDE06DED
:10058000A1F11E0707EB470C072707FA0CF290436F
:10059000A1F11E0707EB470703FA07F21043E065D6
:1005A00034E0132911DDE068A1F1140707EB470CD3
:1005B000072707FA0CF29043A1F1140707EB47074E
:1005C00003FA07F21043E06020E0092911DD2069F9
:1005D000A1F10A0707EB470C072707FA0CF2904333
:1005E000A1F10A0707EB470703FA07F2104320615E
:1005F0000CE0606901EB410C072707FA0CF290430D
:1006000001EB410703FA07F210436061606CC0F32D
:100610000156EF1C06F1010CA7EB0C0707EB870C4A
:100620001F2707FA0CF29043EF1C06F1010CA7EB11
:100630000C0707EB870701FA07F209E000240140E5
:10064000FFFEFFFCFDF7FFC004270140FFFD3FFF59
:1006500010436064F0BD10B50A4600210023416CD0
:1006600021F44011531E41EA0351416410BD08B505
:10067000002300930090009B0B440093009B1A60A2
:1006800008BD0A460021816821F470211143816070
:1006900070470A460021816821F4401111438160AE
:1006A0007047816841F480018160704701460020F5
:1006B0008A6802F480020AB1012000E0002070473D
:1006C00021B1426842F48062426003E0426822F451
:1006D00080624260704721B1426842F480524260B9
:1006E00003E0426822F480524260704708B5024637
:1006F00000200090009201F13000009B184400900F
:100700000098006880B208BD10B50B460021D9B230
:10071000012404FA01F11AB144680C43446002E078
:1007200044688C43446010BD0246002013680B40AF
:100730000BB1012000E000207047CA4302607047FF
:1007400070B502460020002300240B0A55680126DC
:100750008E4005EA060415681D4015B10CB1012054
:1007600000E0002070BD00220A12D34303607047EE
:10077000002044490860091D0860091D0860091D22
:1007800008606FF07F403F491431086070470021D6
:100790003C498279002A3AD00A46126803689A4393
:1007A0000B461A600A1D126803689A430B1D1A60F3
:1007B000027911440A6803681A430A60314A083210
:1007C000126803689A432F4B08331A601A1D126887
:1007D00003689A432B4B0C331A604279102A0ED1CE
:1007E0001A1F126803681A43264B08331A601A1D31
:1007F000126803681A43234B0C331A600DE0214939
:10080000427911440A6803681A430A6005E00279D4
:1008100011440A6803689A430A6070470021016026
:1008200001710C214171002181717047154910310E
:1008300009680143134A10321160704701460020D5
:10084000104A143212680A400AB1012000E0002068
:1008500070470C491431086070470146002000229F
:10086000084B1B6803EA0102064B14331B680B405C
:1008700013B10AB1012000E0002070470149143192
:10088000086070470004014010B504468548844262
:1008900008D10121084600F068FB0021012000F08A
:1008A00064FB52E08048844208D10121022000F01C
:1008B0005CFB0021022000F058FB46E07B488442AC
:1008C00008D10121042000F050FB0021042000F099
:1008D0004CFB3AE07648844208D10121082000F020
:1008E00044FB0021082000F040FB2EE071488442C8
:1008F00008D10121102000F038FB0021102000F069
:1009000034FB22E06C48844208D10121402000F0F1
:100910002CFB0021402000F028FB16E067488442B1
:1009200008D10121802000F020FB0021802000F070
:100930001CFB0AE06248844207D10121202000F01C
:1009400014FB0021202000F010FB10BDF0B50A467A
:1009500000210023002400BF3DE0012505FA01F33A
:10096000156805EA03049C4234D105684F0003264C
:10097000BE40B543056015794E00B5400668354365
:1009800005601579012D02D01579022D16D18568E3
:100990004F000326BE40B543856055794E00B540F3
:1009A000866835438560858801268E40B5438580FD
:1009B000858896798E40B6B235438580C5684F00EC
:1009C0000326BE40B543C560D5794E00B540C66824
:1009D0003543C560491C1029BFD3F0BD4FF6FF71E8
:1009E00001600021017141718171C171704708B5C9
:1009F0004FF480320092009A0A430092009AC2613A
:100A0000C161009AC261C2690092C269009208BDC8
:100A100002460020138A0B400BB1012000E00020A9
:100A200070470146088A704702460020938A0B40AF
:100A30000BB1012000E0002070470146888A704712
:100A400001837047418370470AB1018300E041830D
:100A5000704781827047828A4A4082827047F0B52F
:100A6000002300244D07ED0E02FA05F3CE1000F12D
:100A7000200555F826504E07F70E0F26BE40B54309
:100A8000CF1000F1200646F82750CE1000F12005C7
:100A900055F8265045EA0304CE1000F1200545F82C
:100AA0002640F0BD00000240000402400008024061
:100AB000000C02400010024000180240001C0240DE
:100AC0000014024010B50121080700F070FA00215F
:100AD0004FF0805000F06BFA10BD4D49086270472E
:100AE000014600204B4A106820F0E00008431060E7
:100AF000704747490861704708B500220092444A90
:100B0000A03202440092009A116008BD40498862F8
:100B100070473F4948627047014600203D4A1068CF
:100B200020F4C050084320F00C023A4B1A60704782
:100B300058B13849096841F00101364A116011463F
:100B4000096841F4804111600AE03249096821F4E2
:100B50008041304A11601146096821F0010111609D
:100B6000704710B5024600202A4B186820F0030099
:100B700010431860284B1B6823F00403264C2360A5
:100B8000012901D130BF00E020BF10BD10B50246E1
:100B90000020204B186820F00300104318601E4B03
:100BA0001B6843F004031C4C2360012901D130BFB2
:100BB00000E020BF184B1B6823F00403164C236091
:100BC00010BD1448006840F004001249086008464F
:100BD000006840F0020008600F48006840F0040020
:100BE0000D49086000BF00BF30BF704701460020BC
:100BF000084A52680A400AB1012000E0002070470C
:100C00000449096841EA8001024A11607047000006
:100C100000000E420070004010ED00E0F94800684E
:100C200040F48070F7490860F64808300068F649DB
:100C30000840F44908310860F2480068F349084068
:100C4000F04908600846006820F480200860ED48FC
:100C50000830006820F47D00EA490831086000206F
:100C6000091D086070470021E64A921C1170114668
:100C70000870704710B501460022002300204A1179
:100C8000012A02D1DF4C236802E0DE4C34342368B1
:100C900001F01F02012494401C400CB1012000E02F
:100CA000002010BD38B5002000900024002500BFB2
:100CB0003120FFF7DFFF05460098401C00900098A8
:100CC000B0F5A06F01D0002DF2D03120FFF7D2FF98
:100CD00008B1012400E00024204638BDC949C91DDF
:100CE0000870704701460020C64A121D106820F4A3
:100CF0006040084310607047C5490862704701466C
:100D00000020C04A121D106820F4F85040EA01206B
:100D100010607047BE49086070470021B94A3532FB
:100D20001170114608707047BA490860704710B5D5
:100D300041EA02030343B34C0A34237010BDB449A3
:100D400008667047B24908677047B2492C3108609D
:100D5000704740EA0102AB4B0B331A7070470146F3
:100D60000020A84A0832106820F0030008431060F1
:100D70007047A4480830006800F00C007047014636
:100D80000020A04A0832106820F0F00008431060EC
:100D90007047014600209B4A0832106820F4E0604A
:100DA00008431060704701460020964A08321068D8
:100DB00020F4605040EAC10010607047F0B5002197
:100DC000002200230026002400258E4F08373F68AC
:100DD00007F00C0131B1042912D0082913D00C29D5
:100DE00037D113E0874F3F1D3F68C7F342356F1C73
:100DF0004FF0010C0CFA07FC4FEACC37076036E0E5
:100E0000854F076033E0854F076030E07D4F08373E
:100E10003F6807F470127B4F08373F6807F44003C0
:100E20007F4F07EB92473A78012707EB9353754FB3
:100E300008373F6807F480362EB9774F5743B7FB22
:100E4000F3F7076004E0754F5743B7FBF3F707600C
:100E50000DE06C4F3F1D3F68C7F342356F1C4FF0EC
:100E6000010C0CFA07FC4FEACC37076000BF00BF4B
:100E7000644F08373F6807F0F0010909694F7C5C4F
:100E80000768E74047605F4F08373F6807F4E06155
:100E9000090A644F7C5C4768E7408760594F083710
:100EA0003F6807F46051C90A5E4F7C5C4768E740C1
:100EB000C760F0BD002100F44032B2F5403F08D1D8
:100EC000504A116821F0C04100F0C04211434D4A20
:100ED00011604C4A3432126822F44032494B3433A8
:100EE0001A601A46126800F440331A43454B3433F3
:100EF0001A607047474958310860704745495C316E
:100F00000860704739B13F4A1C32126802433D4BBA
:100F10001C331A6006E03B4A1C3212688243394B8C
:100F20001C331A60704739B1364A203212680243C6
:100F3000344B20331A6006E0324A20321268824372
:100F4000304B20331A60704739B12E4A2432126870
:100F500002432C4B24331A6006E02A4A24321268DA
:100F60008243284B24331A60704739B1254A103226
:100F700012680243234B10331A6006E0214A1032F4
:100F8000126882431F4B10331A60704739B11D4AF3
:100F90001432126802431B4B14331A6006E0194ADC
:100FA000143212688243174B14331A60704739B1F8
:100FB000144A183212680243124B18331A6006E0C2
:100FC000104A1832126882430E4B18331A60704769
:100FD00039B10C4A2832126802430A4B28331A608E
:100FE00006E0084A283212688243064B28331A600A
:100FF0007047C9B1034A2C3212680243014B2C33AB
:101000001A6016E0003802400CC0FF88FEFFFEEEBA
:1010100000004742800647420024F40000127A0094
:1010200050620020596200201F4A126882431E4B02
:101030001A60704739B11C4A121D126802431A4BDC
:101040001B1D1A6006E0184A121D12688243164BD7
:101050001B1D1A60704739B1134A1F3A12780243B8
:10106000114B1F3B1A7006E00F4A1F3A1278824359
:101070000D4B1F3B1A7070470B480830006840F05A
:101080008070094908310860704701460020064A0F
:10109000203A12680A400AB1012000E0002070479F
:1010A00001491E39087070472C38024008B50022EB
:1010B000009200200021CA22F94B1A6053221A60C4
:1010C000F74A183A126822F0A002F54B183B1A6052
:1010D00000BFF34A183A126802F02001009A521C2D
:1010E0000092009AB2F5004F01D00029F1D0EC4AED
:1010F000183A126802F020020AB1012000E0002034
:10110000FF22E74B1A6008BD08B5002200920020BC
:101110000021E34A183A126802F04002E2B9421E86
:10112000DF4B183B1A6000BFDD4A183A126802F024
:101130004001009A521C0092009AB2F5005F01D063
:101140000029F1D0D64A183A126802F040020AB1DA
:10115000012002E0002000E0012008BD38B5002099
:10116000009000240025CA20CD4908605320086063
:10117000FFF7CAFF00B952E00020C94924390860CE
:1011800042F20110091D0860081D006800F0070008
:10119000091D086000BFC2481838006800F0040448
:1011A0000098401C00900098B0F5005F01D0002C22
:1011B000F1D0BB481838006800F0040008B90025D9
:1011C0002DE0B7481C3800680020B5491C3908607C
:1011D0004FF6FF70B24910390860B248091F086025
:1011E0000020AF490C390860091D0860091D08601E
:1011F000AB4908310860AA4918310860A849203174
:101200000860091D0860A64918390860A4491C3106
:101210000860FFF74BFF08B9002500E00125FF201B
:101220009F490860284638BD9D481838006820F05E
:1012300080009B4918390860704730B50446002586
:10124000CA209749086053200860FFF75DFF00B986
:101250001DE093481C38006820F0400090491C397C
:10126000086008460068216808438D491C390860F9
:101270008B491439A068086008460068A18840EAD4
:101280000140874914390860FFF7CEFF0125FF2090
:1012900083490860284630BD002101607F214160FC
:1012A000FF218160704718B1FF217D4A116004E081
:1012B000CA217B4A116053211160704730B5044642
:1012C0000025CA207649086053200860FFF71CFFFC
:1012D00000B914E044B172481C38006840F01000B6
:1012E0006F491C39086007E06D481C38006820F021
:1012F00010006B491C390860FFF796FF0125FF209D
:1013000067490860284630BDCA21654A11605321EB
:10131000116040B162491C39096841F02001604AFE
:101320001C3A116007E05E491C39096801F0DF01D1
:101330005B4A1C3A1160FF21594A1160704701460F
:10134000002204E0501CC2B2A1F10A00C1B20A2975
:10135000F8DA100741EA10607047014600BF08093B
:1013600000EB8000420001F00F001044C0B2704753
:101370002DE9F04105460C460026002755B948489E
:101380001C38006800F0400000B102E00020E0706E
:1013900000BF0EE042481C38006800F0400020B159
:1013A0002078FFF7DAFF064602E00020E07000BF79
:1013B00000BF55B120780004617840EA0120A1788F
:1013C0000843E17840EA014611E02078FFF7B7FFD3
:1013D0004FEA00486078FFF7B2FF48EA0028A0789B
:1013E000FFF7ADFF48EA0008E07848EA0046CA2067
:1013F0002B49086053200860FFF786FE08B90027D4
:1014000014E029483040264924390860FFF70CFFD2
:1014100023481C38006800F0200030B9FFF746FE72
:1014200008B9002702E0012700E00127FF201C493E
:1014300008603846BDE8F0810021C170017041703C
:101440008170704770B506460C4600251448243854
:101450000068154900EA0105C5F305402070C5F391
:101460000620607005F07F00A07005F48000000C7D
:10147000E0705EB92078FFF770FF20706078FFF7AA
:101480006CFF6070A078FFF768FFA07070BD00204F
:101490000349091D0868024920390968704700009E
:1014A00024280040FF007F007F7F7F002DE9F0416E
:1014B00005460C46002600274DB9607800F0100064
:1014C000102804D1607820F010000A30607005B94F
:1014D00008E06078FFF741FF0646A078FFF73DFF80
:1014E000064600BF55B1E0780004617840EA01206B
:1014F000A1780843217840EA413611E0E078FFF70F
:101500001EFF4FEA00486078FFF719FF48EA0028FD
:10151000A078FFF714FF48EA0008207848EA403630
:10152000CA20FE49086053200860FFF7EDFD08B9A6
:10153000002714E0FA483040F84920390860FFF7E6
:1015400073FEF6481C38006800F0200030B9FFF741
:10155000ADFD08B9002702E0012700E00127FF20C8
:10156000EE4908603846BDE8F081012101708170C4
:1015700041700021C170704770B506460C460025C9
:10158000E64820380068E64900EA0105280CE070CA
:10159000C5F30420607005F03F00A070C5F3423031
:1015A00020705EB9E078FFF7D8FEE0706078FFF752
:1015B000D4FE6070A078FFF7D0FEA07070BD2DE95A
:1015C000F04105460E46144600276DB9D3481C3835
:1015D000006800F0400000B102E00020E07000BFB1
:1015E000A06800B91AE019E0CC481C38006800F087
:1015F000400020B12078FFF7B0FE074602E000204F
:10160000E07000BFA06820B9207BFFF7A6FE074668
:1016100004E0207BFFF7A1FE074600BF95B12078CC
:101620000004617840EA0120A1780843E17840EAAB
:101630000140217B40EA0160A1680843616840EAFB
:1016400001071BE02078FFF77AFE4FEA0048607838
:10165000FFF775FE48EA0028A078FFF770FE48EA19
:101660000008E07848EA0048207BFFF768FE48EA77
:101670000060A1680843616840EA0107CA20A749E1
:10168000086053200860B6F5807F03D1A34808386E
:10169000076002E0A148001F0760FF209F49086023
:1016A000BDE8F0810021C1700170417081708160DE
:1016B000012101730021416070472DE9F041064688
:1016C0000F4614460025B7F5807F03D193480838AC
:1016D000056802E09148001F0568C5F305402070C9
:1016E000C5F30620607005F07F00A07005F480004F
:1016F000000CE070C5F30560207305F08040A06029
:1017000005F0803060607EB92078FFF726FE2070FB
:101710006078FFF722FE6070A078FFF71EFEA070D1
:10172000207BFFF71AFE2073BDE8F08138B5024632
:101730000024009400230020CA24784D2C605324F8
:101740002C6041B1754C1C3C24681443734D1C3D06
:101750002C6001201EE0714C1C3C246894436F4DAA
:101760001C3D2C6000BF6D4C183C246804EA122319
:10177000009C641C0094009CB4F5005F01D0002B19
:10178000F1D0664C183C246804EA12240CB90020FD
:1017900000E00120FF24614D2C6038BD30B50023EE
:1017A000CA245E4D2C6053242C6041EA0203B0F53C
:1017B000807F03D1594C2034236002E0574C2434FD
:1017C0002360FF24554D2C6030BD01460020B1F54B
:1017D000807F05D1514A20321268C2F30E0004E026
:1017E0004E4A24321268C2F30E007047CA214B4A97
:1017F00011605321116049491C39096821F0070122
:10180000464A1C3A11601146096801431160FF21E4
:10181000424A11607047CA21404A11605321116049
:101820003E4910390860FF21116070473B4810386D
:10183000006880B2704718B501460023009300226B
:101840000020CA23354C23605323236049B1334B16
:101850001C3B1B6843F48063304C1C3C236001201C
:101860001FE02E4B1C3B1B6823F480632B4C1C3C5D
:10187000236000BF294B183B1B6803F00402009B48
:101880005B1C0093009BB3F5005F01D0002AF1D0F0
:10189000224B183B1B6803F004030BB9002000E047
:1018A0000120FF231D4C236018BDCA221B4B1A6068
:1018B00053221A60194A1C3A126822F48022174BEC
:1018C0001C3B1A601A46126840EA01031A43134B84
:1018D0001C3B1A60FF22114B1A6070470F481C38DE
:1018E000006800F480207047CA220C4B1A60532213
:1018F0001A600A4A1C3A126822F4E002074B1C3BA9
:101900001A601A46126840EA01031A43034B1C3B53
:101910001A60FF22014B1A60704700002428004023
:101920003FFFFF0070B504460D460026CA20FE4961
:10193000086053200860FFF7E7FB00B907E044EABE
:101940000500F9490C390860FFF76EFC0126FF20FD
:10195000F5490860304670BD30B504460025CA2000
:10196000F149086053200860FFF7CEFB00B914E08E
:1019700044B1ED481C38006840F08000EA491C3949
:10198000086007E0E8481C38006820F08000E6495D
:101990001C390860FFF748FC0125FF20E249086078
:1019A000284630BDCA21E04A11605321116040B180
:1019B000DD491C39096841F40001DB4A1C3A116019
:1019C00007E0D9491C39096821F40001D64A1C3ABC
:1019D0001160FF21D44A11607047CA21D24A1160B8
:1019E00053211160D0491C39096821F40021CE4AE5
:1019F0001C3A11601146096801431160FF21CA4A6F
:101A00001160704770B5034600200024CA25C64EF9
:101A1000356053253560C44D183D2D6805F480357B
:101A200055B100E0641CC04D183D2D6805F48035AB
:101A300015B1B4F5805FF5D1BB4D183D2D6805F4A7
:101A400080353DB943EA01051543B74E1836356078
:101A5000012000E00020FF25B34E356070BD10B5B9
:101A60000A460021B04B1C3B1B6840F6080423EAE1
:101A700004011AB140F40063194300E00143CA2392
:101A8000A94C236053232360A74B1C3B1960FF2301
:101A9000236010BD2DE9F04180460C461546002616
:101AA0000027A1480C300068A04900EA01069E48C2
:101AB000103000689E4900EA0107C6F30540207017
:101AC000C6F30620607006F07F00A07006F4800068
:101AD000000CE0700020E870C7F30420687007F085
:101AE0003F00A870C7F342302870B8F1000F17D13B
:101AF0002078FFF732FC20706078FFF72EFC6070D2
:101B0000A078FFF72AFCA0706878FFF726FC6870C1
:101B1000A878FFF722FCA8702878FFF71EFC287031
:101B2000BDE8F081804814300068704741B97E4AB2
:101B30001C32126822EA40027B4B1C331A6007E019
:101B4000794A1C32126842EA4002774B1C331A6011
:101B5000704739B1744A1C3212680243724B1C330D
:101B60001A6006E0704A1C32126882436E4B1C33C6
:101B70001A6070476C491C31096821F4C0516A4AE7
:101B80001C321160114609680143116070476649B3
:101B90001C31096821F4E061634A1C32116011466E
:101BA00009680143116070475F491C31096821F4DD
:101BB000C0415D4A1C321160114609680143116041
:101BC000704740B158491C31096841F08001564ABC
:101BD0001C32116007E054491C31096821F0800172
:101BE000514A1C321160704740B14F491C3109689D
:101BF00021F400414C4A1C32116007E04A491C3173
:101C0000096841F40041484A1C321160704708B528
:101C100000220092444A2C320092009A02EB800289
:101C20000092009A116008BD08B50146002000909E
:101C30003D482C300090009800EB81000090009807
:101C4000006808BD38491C31096821F48021364AF2
:101C50001C32116011460968014311607047F0B5EC
:101C600004460D4600270026CA202F49086053204D
:101C700008602D481838006800F0080050B100E0F6
:101C8000761C29481838006800F0080010B1B6F535
:101C9000005FF5D124481838006800F0080098B9B2
:101CA00021481C38006800F0100058B945EA0400CB
:101CB0001D4908310860FFF7F9F908B9002704E069
:101CC000012702E0002700E00027FF2016490860F6
:101CD0003846F0BDCA22144B1A6053221A6091B1E3
:101CE000114A1C3A126820F004031A430E4B1C3BA5
:101CF0001A600D4A1C32126800F004031A430A4BA2
:101D00001C331A6018E0084A1C3A126820F00403D9
:101D10009A43054B1C3B1A60034A1C32126800F0C0
:101D200004039A43004B05E0242800407F7F7F0096
:101D30003FFFFF001C331A60FF222A4B1A607047D6
:101D400010B5014600200022264B183B1B68264C8C
:101D500003EA040202EA01030BB1012000E00020C3
:101D600010BDC0F3100141F080011E4A183A1268FC
:101D700002F0800262EA01011A4A183A11607047C3
:101D800030B50146002000220023164C1C34246884
:101D900004F00402134C1C3C24680C408D0C21FA06
:101DA00005F502EAD53544EA05030E4C183C2468D3
:101DB00004EA11121BB194B20CB1012000E0002022
:101DC00030BD002101098AB242F08002054B183B68
:101DD0001B6803F0800363EA0202024B183B1A609F
:101DE00070470000242800407FFF010010B5044622
:101DF000BA48844208D101218014FFF7C7F80021B6
:101E0000A014FFF7C3F816E0B548844208D10121B9
:101E10000014FFF7CCF800212014FFF7C8F80AE0FF
:101E2000B048844207D10121C013FFF7C0F8002158
:101E3000E013FFF7BCF810BD10B50022028802F4D1
:101E400041520B884C8823438C882343CC882343FE
:101E50000C8923434C8923438C892343CC89234316
:101E60001A430280838B4FF2FF74234083830B8AD3
:101E7000038210BD2DE9FF5F05460C464FF00009B7
:101E800002274FF000084FF0010B0026B246A88B46
:101E90004FF240010840A88302202884B5F81C9026
:101EA000A068022801D100BF33E0A08810B94FF02C
:101EB000010B01E04FF0020B6846FEF77FFFDDF8F3
:101EC00000A0E088B0F5007F0AD14FEA1A2000EBAD
:101ED00080004000A168B0FBF1F0401D86B20BE02D
:101EE0004FEA4B10BAFBF0F000EB80004000A16815
:101EF000B0FBF1F0401D86B20A20B6FBF0F606F00A
:101F00000108A6EB0800C0F34F074FF6FF7000EA88
:101F10000828022F01DBFF2F02DD02274FF0000807
:101F2000E08840EA080038432884A088A189084353
:101F3000618808432188084340F4006040EA0909A9
:101F4000A5F81C90BDE8FF9F0021018041808180A1
:101F5000C180018141818181C18107210182704756
:101F60000021018041808180C180022181600021A7
:101F70008181704721B1028842F04002028004E072
:101F800002884FF6BF731A400280704721B1828BDE
:101F900042F48062828304E0828B4FF6FF331A4062
:101FA0008283704702884FF2FF731A4002800288D2
:101FB0000A4302807047B1F5804F04D1028842F491
:101FC0008042028004E002884BF6FF731A400280D0
:101FD00070474FF6FF62914204D0028842F480724B
:101FE000028004E002884FF6FF631A4002807047C7
:101FF00021B1828842F00402828004E082884FF698
:10200000FB731A408280704701468889704781813E
:10201000704721B1028842F40052028004E0028835
:102020004DF6FF731A4002807047018841F48051D9
:102030000180704702460020012901D0108B00E08A
:10204000908A70470146088A70471AB183880B430B
:10205000838002E083888B438380704730B50024FF
:1020600000230C110125A540ABB21AB185881D4390
:10207000858002E085889D43858030BD0246002032
:1020800013890B400BB1012000E000207047CA43C8
:1020900002817047F0B5024600200024002300258D
:1020A00001F00F070126BE40B4B20B1101269E407D
:1020B000B3B2968806EA03051689264016B10DB11B
:1020C000012000E00020F0BD10B5002201F00F0457
:1020D0000123A3409AB2D343038110BD00300140D5
:1020E00000380040003C004010B501210846FEF7D2
:1020F0004DFF00210120FEF749FF10BD0020B2492D
:102100000860091D0860091D0860091D0860091D97
:102110000860091D0860091D08607047AB49086028
:102120007047AA48006800F44070704730B1A74972
:10213000496841F00101A54A516005E0A349496899
:1021400021F00101A14A5160704730B500228B0790
:102150001C0F0F2303FA04F29C4B08338C1053F826
:1021600024309343994C08348D1044F8253023468D
:102170008C1053F824308C07240F00FA04F4234306
:10218000924C08348D1044F8253030BD01460020B3
:102190008D4A106820F440300843106070470246B2
:1021A0000020894B1868104302F48023B3F5802F78
:1021B00002D120F00F00084302F40023B3F5002FF2
:1021C00003D120F0F00040EA011002F48013B3F5CF
:1021D000801F03D120F4706040EA012002F4001354
:1021E000B3F5001F03D120F4704040EA0130764B74
:1021F0001860704739B1744A121F12680243724B5B
:102200001B1F1A6006E0704A121F126882436E4B51
:102210001B1F1A60704739B16B4A121F1268824344
:10222000694B1B1F1A6006E0674A121F12680243BF
:10223000654B1B1F1A60704710B50022C20F20F0BB
:10224000004081B13AB1604B1B1D1B6803435E4CDB
:10225000241D236017E05C4B08331B6803435A4C72
:10226000083423600FE03AB1574B1B1D1B688343B2
:10227000554C241D236006E0534B08331B688343F1
:10228000514C0834236010BD40B14F49091D096805
:1022900041F000414C4A121D116007E04A49091DF6
:1022A000096821F00041484A121D1160704710B5BD
:1022B000012810D13AB1444B0C331B688B43424C7C
:1022C0000C3423607FE0404B0C331B680B433E4CC7
:1022D0000C34236077E0022813D14AB13A4B0C3317
:1022E0001B68CC4303EA0443374C0C3423606AE098
:1022F000354B0C331B6843EA0143334C0C342360E9
:1023000061E0032810D13AB12F4B10331B688B4387
:102310002D4C1034236056E02B4B10331B680B43BD
:10232000294C103423604EE0042813D14AB1264BC7
:1023300010331B68CC4303EA0443234C103423605E
:1023400041E0214B10331B6843EA01431E4C10341B
:10235000236038E0052810D13AB11B4B14331B68B9
:102360008B43194C143423602DE0174B14331B6836
:102370000B43154C1434236025E0062813D14AB1D1
:10238000114B14331B68CC4303EA04430E4C143442
:10239000236018E00C4B14331B6843EA01430A4CDA
:1023A000143423600FE03AB1074B18331B688B439A
:1023B000054C1834236006E0034B18331B680B43AD
:1023C000014C1834236010BD047C00400000014023
:1023D00010B50446B4F1804F08D101210846FEF73C
:1023E000E6FD00210120FEF7E2FD5EE0FB488442AD
:1023F00008D101210220FEF7DAFD00210220FEF7BC
:10240000D6FD52E0F648844208D101210420FEF7AF
:10241000CEFD00210420FEF7CAFD46E0F1488442CB
:1024200008D101210820FEF7C2FD00210820FEF797
:10243000BEFD3AE0EC48844208D101211020FEF7AD
:10244000B6FD00211020FEF7B2FD2EE0E7488442E1
:1024500008D101212020FEF7AAFD00212020FEF74F
:10246000A6FD22E0E248844208D101210420FEF7C3
:102470008DFD00210420FEF789FD16E0DD48844231
:1024800008D101210820FEF781FD00210820FEF778
:102490007DFD0AE0D848844207D101211020FEF7D3
:1024A00075FD00211020FEF771FD10BD002202888D
:1024B000B0F1804F08D0C94B984205D0C84B984224
:1024C00002D0C84B984204D14FF68F731A404B8804
:1024D0001A43C54B984207D0C44B984204D04FF6DC
:1024E000FF431A400B891A4302804B68C3620B8872
:1024F00003850123838270474FF0FF314160002143
:1025000001800181418070470185828270470A46BF
:10251000002101884FF68F731940114301807047E5
:1025200041627047C16270470146486A7047014680
:10253000088D704721B1028842F00202028004E057
:1025400002884FF6FD731A400280704721B102885D
:1025500042F00402028004E002884FF6FB731A4046
:102560000280704721B1028842F08002028004E0BC
:1025700002884FF67F731A400280704702884FF638
:10258000F7731A40028002880A430280704702886B
:102590004FF6FF431A40028002880A4302807047C8
:1025A00021B1028842F00102028004E002884FF665
:1025B000FE731A400280704730B500230022048C5D
:1025C0004FF6FE752C400484028C038B4FF68F74FB
:1025D0002340AC1E23400C8823436C1E22400C89F0
:1025E00022434C8822434C6844630383028430BDF9
:1025F00030B500230022048C4FF6EF752C40048484
:10260000028C038B48F6FF7423400C884FF6FF754D
:1026100005EA042423434FF6DF7422400C8905EABF
:10262000041422434C8805EA041422434C68846352
:102630000383028430BD30B500230022048C4FF6A2
:10264000FF652C400484028C838B4FF68F742340EB
:102650000C8823434FF6FF5422400C894FF6FF7538
:1026600005EA042422434C8805EA042422434C68EA
:10267000C4638383028430BD30B500230022048C00
:102680004EF6FF752C400484028C838B48F6FF7451
:1026900023400C884FF6FF7505EA042423434DF6CA
:1026A000FF7422400C8905EA043422434C8805EA71
:1026B000043422434C6804648383028430BD0021C7
:1026C0000180418041600181704770B50346002060
:1026D00000241846183001258D40ACB21D8CA5434E
:1026E0001D8409B1082909D100EB6100056825F0B6
:1026F000700505600568154305600EE00D1FC5F304
:102700004E052844056825F4E045056005684FF648
:10271000FF7606EA02263543056070BD41637047C7
:1027200081637047C1637047016470470A460021A6
:10273000018B4FF68F7319401143018370470A468E
:102740000021018B48F6FF7319404FF6FF7303EA2F
:1027500002231943018370470A460021818B4FF6FB
:102760008F7319401143818370470A460021818B82
:1027700048F6FF7319404FF6FF7303EA022319432B
:10278000818370470A460021018B4FF6F773194089
:102790001143018370470A460021018B4FF2FF73FA
:1027A00019404FF6FF7303EA022319430183704770
:1027B0000A460021818B4FF6F7731940114381833C
:1027C00070470A460021818B4FF2FF7319404FF684
:1027D000FF7303EA0223194381837047000400401A
:1027E00000080040000C00400010004000140040B1
:1027F00000080140000C0140001001400A46002181
:10280000018B4FF6FB7319401143018370470A4651
:102810000021018B4FF6FF3319404FF6FF7303EA97
:1028200002231943018370470A460021818B4FF62A
:10283000FB7319401143818370470A460021818B45
:102840004FF6FF3319404FF6FF7303EA0223194393
:10285000818370470A460021018B4FF67F73194030
:102860001143018370470A460021018BC1F30E0119
:102870004FF6FF7303EA02231943018370470A46A8
:102880000021818B4FF67F7319401143818370477C
:102890000A460021818BC1F30E014FF6FF7303EA54
:1028A00002231943818370470A460021018C4FF6A9
:1028B000FD7319401143018470470A460021018CC1
:1028C0004FF6DF7319404FF6FF7303EA0213194303
:1028D000018470470A460021018C4FF6FF531940CE
:1028E0004FF6FF7303EA02231943018470470A4637
:1028F0000021018C4DF6FF7319404FF6FF7303EA78
:10290000023319430184704702894FF6F7731A4066
:10291000028102890A430281704730B500230124F5
:102920008C40A3B2048C9C430484048C02FA01F50D
:10293000ADB22C43048430BD828B4FF2FF331A407A
:102940008283828B4FF6FF7303EA01231A4382834B
:102950007047F0B50C461546002100220026078C72
:102960004EF6FF7C07EA0C070784818B028C4FF63A
:10297000FF7707EA043640F6FF4739404FF6FF7706
:1029800007EA052739434FF6FF7707EA033739434C
:1029900045F6FF773A4046F480573A4381830284F4
:1029A000F0BD828B4FF6F3731A408283828B0A4309
:1029B00082837047F0B50C461546002100220026A0
:1029C000078C4FF6FF6C07EA0C070784818B028C9B
:1029D0004FF6FF7707EA04264FF60C7739404FF69B
:1029E000FF7707EA03172F4339434FF2FF573A4067
:1029F00046F480773A4381830284F0BD028B4FF224
:102A0000FF331A400283028B4FF6FF7303EA012360
:102A10001A4302837047F0B50C4615460021002288
:102A20000026078C4FF6EF7C07EA0C070784018B22
:102A3000028C4FF6FF7707EA041640F6FF4739404D
:102A40004FF6FF7707EA033739434FF6FF7707EA78
:102A5000052739434FF65F773A4046F010073A436F
:102A600001830284F0BD028B4FF6F3731A40028398
:102A7000028B0A4302837047F0B50C4615460021CD
:102A80000022068C4FF6FE773E400684018B028CB6
:102A90004FF60C7631407E1C06EA03162E43314376
:102AA0004FF6F576324044F001063243018302844A
:102AB000F0BD70B505460C46208850B92389A28820
:102AC00061882846FFF7D8FFE1882846FFF7CBFF4B
:102AD00025E0208804280AD12389A2886188284615
:102AE000FFF799FFE1882846FFF788FF17E0208865
:102AF00008280AD12389A28861882846FFF75AFF4F
:102B0000E1882846FFF74DFF09E02389A288618804
:102B10002846FFF71EFFE1882846FFF70DFF70BD2E
:102B2000002101804180012181800021C18001813B
:102B300070472DE9F04105460C46002601276088C4
:102B400008B9022600E00026A088012801D102274A
:102B500000E001272088A0B92389A288618828463F
:102B6000FFF78AFFE1882846FFF77DFF23893A4671
:102B700031462846FFF74FFFE1882846FFF73EFF22
:102B800013E02389A28861882846FFF744FFE18883
:102B90002846FFF733FF23893A4631462846FFF798
:102BA0006BFFE1882846FFF75EFFBDE8F081014634
:102BB000486B70470146886B70470146C86B704789
:102BC0000146086C70471AB183890B43838102E088
:102BD00083898B438381704781827047024600203E
:102BE000138A0B400BB1012000E000207047CA435C
:102BF0000282704730B50246002000230024158A67
:102C000005EA0103958905EA010413B10CB101201D
:102C100000E0002030BDCA430282704741EA02034F
:102C2000A0F8483070471AB183890B43838102E0D2
:102C300083898B438381704721B1828842F00802E7
:102C4000828004E082884FF6F7731A4082807047D2
:102C500001894FF6F8721140018170470A46002140
:102C600001894FF68F73194011430181704730B5C8
:102C700004460D4629462046FFF7F0FF208940F024
:102C80000700208130BD2DE9F04104460D4616466F
:102C90001F46602D06D13B46012231462046FFF7F4
:102CA000BAFE05E03B46012231462046FFF7E4FE2E
:102CB00029462046FFF7D2FF208940F007002081F7
:102CC000BDE8F08130B50C4600210189C9B24FF64C
:102CD000FF7505EA0325154325432943018130BDCE
:102CE0002DE9F04105460E46174698460024434616
:102CF0003A4631462846FFF7E5FF2C894FF6F87033
:102D0000044044F007044FF68F70044044F0700410
:102D10002C81BDE8F081F0B504460D4616461F46ED
:102D20003B46324629462046FFF7CCFF208940F437
:102D300080402081F0BD82884FF68F731A408280D8
:102D400082880A438280704702894FF6F8731A40DE
:102D5000028102890A430281704702894FF67F731C
:102D60001A40028102890A4302817047F0B50C467D
:102D700015461E460021002200230189028B038C88
:102D80004FF6F877394021434FF6FC473A4040F27E
:102D900001173A434FF6DD773B404FF6FF7707EADE
:102DA00006172F433B43018102830384F0BD21B109
:102DB000828842F08002828004E082884FF67F732E
:102DC0001A408280704730F8502F02EA1142028088
:102DD00002888BB21A4320F85029704710B5044678
:102DE000F748844209D101218803FEF7CFF800217A
:102DF0004FF48040FEF7CAF832E0F248844209D12D
:102E000001214804FEF7D3F800214FF40030FEF70B
:102E1000CEF825E0EC48844209D101218804FEF770
:102E2000C6F800214FF48020FEF7C1F818E0E7480B
:102E3000844209D10121C804FEF7B9F800214FF4FA
:102E40000020FEF7B4F80BE0E148844208D10121EC
:102E50000805FEF7ACF800214FF48010FEF7A7F844
:102E600010BD2DE9FF4705460E460024A14600BFD0
:102E7000A046B08900B100BF2C8A24F44054F088E9
:102E800004432C82AC8941F20C608443B0883189C0
:102E90000843718908430443AC81AC8A24F440742C
:102EA000B0890443AC826846FDF788FFC448854278
:102EB00002D1DDF80C9001E0DDF80890A88900F45B
:102EC000004040B109EBC90000EB0910316849002E
:102ED000B0FBF1F707E009EBC90000EB091031681E
:102EE0008900B0FBF1F76420B7FBF0F00401200982
:102EF000642101FB1078A88900F4004040B1322021
:102F000000EBC800B0FBF1F000F00700044308E05C
:102F1000322000EB08106421B0FBF1F000F00F004C
:102F200004432C81BDE8FF874FF416510160002156
:102F30008180C18001810C21418100218181704704
:102F400010B502460020108A20F470600B884C886F
:102F500023438C882343CC8823431843108210BD1D
:102F60000021018041808180C180704721B1828928
:102F700042F40052828104E082894DF6FF731A40C8
:102F800082817047028B02F47F420283028B0A43E4
:102F90000283704721B1828942F40042828103E0BA
:102FA0008289C2F30E028281704721B1828A42F483
:102FB0000062828204E0828A4FF2FF731A408282AA
:102FC0007047C1F308028280704701468888C0F3C9
:102FD00008007047028A4FF6F0731A400282028A94
:102FE0000A430282704721B1828942F00202828143
:102FF00004E082894FF6FD731A408281704782890E
:103000004FF2FF731A40828182890A43828170479E
:10301000028A4FF6DF731A400282028A0A43028252
:10302000704721B1028A42F48042028204E0028A9F
:103030004BF6FF731A4002827047818941F001010B
:103040008181704721B1828A42F00802828204E0C5
:10305000828A4FF6F7731A4082827047028BD2B28F
:103060000283028B42EA01220283704721B1828AE5
:1030700042F02002828204E0828A4FF6DF731A4017
:103080008282704721B1828A42F01002828204E07B
:10309000828A4FF6EF731A4082827047828A4FF617
:1030A000FB731A408282828A0A438282704721B16E
:1030B000828A42F00202828204E0828A4FF6FD7325
:1030C0001A40828270471AB1838A0B43838202E0DE
:1030D000838A8B4383827047F0B503460024002621
:1030E0000025002040F66A17B94200D100BF1846FB
:1030F000C1F3421401F01F06012707FA06F5012C5F
:1031000001D10C3004E0022C01D1103000E0143069
:103110001AB107682F43076002E00768AF430760F2
:10312000F0BD02460020B1F5007F00D100BF13883A
:103130000B400BB1012000E00020704701F4007249
:10314000B2F5007F00D100BFCA430280704770B55E
:103150000246002400230025002040F66A16B142F2
:1031600000D100BFC1F3421501F01F03012606FA8A
:1031700003F3012D02D19689334006E0022D02D1DE
:10318000168A334001E0968A33400C12012606FA73
:1031900004F41688344013B10CB1012000E0002083
:1031A00070BD10B50022002340F66A14A14200D180
:1031B00000BF0A1201249440A3B2DC43048010BD76
:1031C000003801400044004000480040004C0040EE
:1031D0000050004010B5FE49FE4803F0FCF93220D3
:1031E000FD490870302048700846F9490A68C0F85F
:1031F00002208988C1800CF0A9FDF84908600F21E0
:10320000F5480CF05AFDF448F2490A6802608988D2
:1032100081800CF09BFDF24908600F21EE480CF014
:103220004CFDED48EF490A680260496841600CF0C6
:103230008DFDED4908600F21E7480CF03EFDE649A1
:10324000E84882680A608089888008460CF07EFD24
:10325000E6490860E1480068E3490968884201D905
:10326000002010BDDD480068DF490968884201D2AE
:103270000120F6E7DA480068DC490968884201D98C
:103280000020EEE70120ECE74FF4FA700DF00CFCA3
:103290008CE0D74800680EF069FA401C38B9D54870
:1032A000007820F00100401CD249087005E0D148A8
:1032B000007820F00100CF490870CF4800680EF078
:1032C00055FA401C38B9CB48007820F00400001DA6
:1032D000C849087005E0C748007820F00400C549D7
:1032E0000870C64800680EF041FA401C38B9C14861
:1032F000007820F008000830BE49087005E0BD489D
:10330000007820F00800BB4908704FF40051BC4819
:10331000FDF77EFB08B9012000E00020B9490978DB
:1033200081F001010840B3490978B24A1278C2F32A
:1033300080021140AF4A1278C2F3C0021140B14A74
:103340001278C2F3800282F001021140084050B3AB
:10335000A4486B3890F87A0031280AD1FFF73AFF79
:1033600038B10020FEF767FA00214FF48070FEF7B5
:10337000DDF94FF40050FDF781FA4FF48040FEF77D
:1033800020FD4FF48010FDF779FA4FF40050FEF75E
:1033900018FD4FF48050FEF714FD4FF40030FDF798
:1033A0006DFAFDF70EFC32200DF07EFB71E7F2B0F6
:1033B00000200A900B900C900D90069007900890BA
:1033C0000990E8E04FF480618F4800680DF0BAFB87
:1033D0004FF47A700DF068FB8C48007820F04000C4
:1033E00040308A4908700AA906A803F0F4F8874813
:1033F0000078C0F38000C0B94FF0FF318448006806
:103400000EF04CF98349844803F0E5F80AF02CFBF0
:1034100001F09CF901217A48FDF712FB0CF059FAF2
:1034200001F0A0F90BF00DFC05E04FF0FF317848FA
:1034300000680EF033F90AAA78A176480EF0EAFF88
:1034400006AA76A174480EF0E5FF05F074FC6F48FB
:10345000007800F0010038B94FF0FF317048006883
:103460000EF01CF909F027F9674800680DF040FBE1
:1034700000F02000002832D04021634800680DF0A1
:1034800061FB42F21073012280215F4800680DF059
:103490007FFB04AA05A963A005F0B2FC62480CF00A
:1034A00033FC04466148C078DDE90412CDE901210E
:1034B00000905E490B784A795B4908195CA10EF0CF
:1034C000A9FF05F0CDF940214F4800680DF0FEFA44
:1034D0004FF480714C4800680DF034FB23E040212C
:1034E000494800680DF02EFB04AA05A94DA005F07F
:1034F00087FC4D480CF008FC04464C48C078DDE9D8
:103500000412CDE90121009048490B784A794649D7
:10351000081947A10EF07EFF05F0A2F940213A48B4
:1035200000680DF0D3FA40480CF0EEFB851C3E48D5
:103530002B4644A245A100900EA80EF06BFF4FF061
:10354000FF31454800680DF005FC0EA80CF0DCFBCF
:10355000054600232A460EA9184609F076FF3E4884
:1035600000680DF01BFC2E4800680EF0D3F82848C8
:1035700000680EF0CFF82548007820F0400023497D
:1035800008704FF48061204800680DF09FFA3348BE
:1035900000680EF00FF915E70024E6E04FF0FF3168
:1035A0001B4800680EF07AF80DF014FB2C490860F7
:1035B0001648007820F00400001D144908701549D1
:1035C000154803F008F8074B1B3B124A4AE000007D
:1035D0005B6400205164002042640020906200205F
:1035E0009462002034660020886200208C620020F3
:1035F000A062002078620020AC6200209C62002063
:10360000000802401E630020C0620020716200209A
:10361000B862002024640020336400202573000079
:10362000BC62002030000000406F00203D6300209D
:103630002C25642C25642C25642C256C642C256C8D
:10364000640000005075622C0000000025732564A2
:103650002C25732C2A000000CC620020B4620020CC
:1036600080620020FAA1FD480EF0D4FEFC480078EC
:1036700078B1FC49FC4802680A6080888880FB4970
:10368000F948801E82680A60808988800020F44999
:1036900008700AF0E9F901F059F80A2000F075FD08
:1036A0000121F348FDF7CCF90CF013F901F05AF8B9
:1036B0000BF0C7FA05F03FFBEE4800680DF018FA72
:1036C00000F02000D0B14021EA4800680DF03AFA3D
:1036D00042F2107301228021E64800680DF058FA8A
:1036E00004F069FD4021E34800680DF0EFF94FF464
:1036F0008071E04800680DF025FA0BE04021DD48BC
:1037000000680DF01FFA04F056FD4021D94800680A
:103710000DF0DCF9D84800680DF0FCFFD7480078C0
:1037200020F00400D5490870D54800680EF042F832
:10373000D34800680EF03EF8054606E0D048006821
:103740000EF038F80546601CC4B20DB1012000E04F
:1037500000200A2C01DA012100E0002108400028A5
:10376000ECD14FF47A700DF09FF917E700243EE09A
:1037700000250220C349087000241BE04FF0FF31F0
:10378000C14800680DF0E6FA09F099FE0546022DE1
:1037900006D1002400230B22BCA1184609F055FED7
:1037A000B94800680DF0FAFA4EF660200DF07CF989
:1037B000601CC4B2042CE1DBB2480078022812D0AD
:1037C0000821AC4800680DF0BDF94FF40071A9481C
:1037D00000680DF07BF9B04800680DF0EBFFAF48D2
:1037E00000680DF0E7FF05200DF05EF900BFBFE7B0
:1037F00028E0A04800680DF07BF900F4007090B953
:10380000994A3B3A02F10A01A1F11E000AF08CF834
:1038100001219748FDF714F94FF4007195480068AD
:103820000DF090F900BF4FF0FF31974800680DF0A0
:1038300091FA03F0D9FC944800680DF0AFFA142017
:103840000DF032F9D5E700240025A9E04FF0FF3153
:10385000934800680DF022FF0DF0BCF99149086013
:103860008648007820F00100401C84490870002040
:103870008D490871002416E008F01DFF8A48C078C1
:10388000012808D1062409F03CF877495939A1F1FB
:10389000140009F071F88448407900B90624601CCE
:1038A000C4B2601CC4B2052CE6DB01F02DFF7FA082
:1038B0000EF0A0FD20216F4800680DF043F96D481F
:1038C00000680DF015F900F0400018B140F6B8306E
:1038D0000DF0EAF87448C078012832D100240025A0
:1038E00008E0601CC4B2052000F04FFC73A005F096
:1038F0000BF805461E2D01D8012000E00020322CD7
:1039000001DA012100E0002108400028E9D11E2D44
:1039100017D92A46002169A005F02FF800240EE0EF
:103920004FF47A700DF0C0F866A167480CF0D0F93A
:1039300018B101F0F1FF01F0E7FE601CC4B20A2CDF
:10394000EEDB20214B4800680DF0C0F808F0ADFE1A
:103950004A48007820F00100484908700024504887
:1039600000680DF0D7FE594800680DF023FF0646A9
:1039700006E0564800680DF01DFF0646601CC4B204
:103980000EB1012000E000200A2C01DA012100E044
:10399000002108400028ECD14FF4FA700DF084F8B3
:1039A00054E771E14A48007800F00100F0B147485F
:1039B00000680DF0DBFE0446601C20B12F48007843
:1039C00000F0010038B9434A0021AFF285100DF034
:1039D000DFFE3E4908603E48007820F001003C4987
:1039E000087001F038FE064602F083FF3848007880
:1039F000C0F34000C8B1224800680DF0B7FE04468D
:103A0000601C38B9344A0021AFF273400DF0C0FE9B
:103A10001B4908602E48007820F002002C490870ED
:103A200003F0CFF901202D49087029480078C0F330
:103A3000800058B1124800680DF098FE0446601CE2
:103A400028B10E480078C0F3800049E071E048E0FA
:103A500025735F25732E747874000000C4780020ED
:103A60002063002024640020366600203364002098
:103A700000080240C0620020B8620020716200208D
:103A8000AC6200206E620020CC620020486561724A
:103A900074626561742C2A009C620020A46200207C
:103AA000BC6200207C6200203D63002041542B4317
:103AB0004750414444523F0D0A0000004243323512
:103AC000000000007061720083660020A062002088
:103AD0001E630020AC3A0208883A02088462002083
:103AE00038B9C74A0021AFF24F500DF051FEC54919
:103AF0000860C548007820F00400C349087005B983
:103B0000012501F09EFD461E304602F035FE02F012
:103B10001EFEC5EB051100EB8100BC49086008469C
:103B20000068BB49884204D9B8480068401AB749C0
:103B30000860B8480078C82807D1B348007820F05A
:103B40000800B149087001F0DEFCB24800781E2878
:103B500001DB012000E00020AF4909780843F8B1FB
:103B6000AE4800680DF002FE0446601C78B9AC4A0D
:103B70000021AFF283300DF00BFEAA490860AA4A7B
:103B80000021AFF217400DF003FEA44908609E48E3
:103B9000007820F008009C49087000209E490870B9
:103BA00099480078C0F3001080B39748007820F05F
:103BB0001000954908709D4890F87A0031280BD183
:103BC000FFF708FB40B103F0A8F89948007820F00F
:103BD00002009749087019E08A4800680DF0C6FD98
:103BE0000446601C38B9864A0021AFF253600DF0DC
:103BF000CFFD8449086001F024FD461E304602F0E6
:103C0000BBFD01F028FD064602F073FE7E480078F9
:103C1000C0F34010A0B17B4800680DF0A7FD04463A
:103C2000601C38B9764A0021AFF293600DF0B0FD08
:103C3000744908607448007820F0200072490870C8
:103C400071480078C0F38010D8B17A4800680DF050
:103C50008DFD0446601C30B1774800680CF048FFC9
:103C600000F4806038B9754A0021AFF6BD000DF050
:103C70008FFD704908606448007820F04000624978
:103C800008700A200CF010FF8CE610B5012267497D
:103C900056316E2001F00AFA69480DF06DF8694955
:103CA000086069480DF068F86849086068480DF0D8
:103CB00063F868490860684A0021AFF219300DF0D6
:103CC00067FD66490860664A0021AFF643200DF0A3
:103CD0005FFD6449086010BD0024FFF7D6FF4AE08D
:103CE0000CF078FF60490968451A0CF073FF5F49D2
:103CF0000968461A601CC4B20A2C00DB00245C4828
:103D00000078022801D10025002601F09AFC00EB82
:103D10004001C1EBC010574901EBC000A84201D2DD
:103D2000012000E0002052490978022901D0012138
:103D300000E00021084008B100F050F801F08BFCD1
:103D400000EB4001C1EBC0104B4901EBC000B04299
:103D500001D2012000E0002045490978022901D064
:103D6000012100E00021084008B100F037F84FF4CD
:103D70007A700CF099FEB3E740484149086000F0C2
:103D800046F900F03DFB0CF039FF3E480CF0C8FE50
:103D9000294908603C480CF0C3FE3C4908603C4897
:103DA0000CF0BEFE3B4908603B4A012108460DF07D
:103DB0009FFC3A4908603A4A012108460DF098FCF8
:103DC00038490860384A0021AFF2F3000DF0E0FCFA
:103DD000364908600CF028FF00BFFEE7BFF34F8FA5
:103DE0002748001D006800F4E06031490843001DC9
:103DF0002349091D0860BFF34F8F00BFFEE7000095
:103E0000883A0208AC6200201E6300207462002021
:103E1000805101001F6300207A6200209C62002014
:103E2000C8390208A462002080390208C965002050
:103E300071620020B4620020C0620020103A0208C3
:103E4000D03A0208CC620020E03A0208D06200209A
:103E5000F03A0208D4620020643A0208B0620020FE
:103E6000EC39020898620020806200207C62002009
:103E70006E620020400D030000DD6D0000000108AF
:103E800008ED00E0343A0208443A0208C462002017
:103E9000543A0208C8620020003B0208B8620020C1
:103EA000103B0208BC620020A4390208A86200206E
:103EB0000000FA050CB500200190009087480068CA
:103EC00040F480308549086000BF8448006800F4F1
:103ED000003000900198401C0190009818B901989A
:103EE000B0F5A06FF1D17D48006800F4003010B14A
:103EF0000120009001E0002000900098012859D195
:103F00007748006840F0040075490860084600687A
:103F100040F0020008600846006840F001000860B8
:103F20006E482430006840F080506C4924310860AD
:103F3000C8146C49086000BF6A48406800F010006F
:103F40000028F9D1654808300068644908310860E4
:103F5000084600680860084600680860084600686F
:103F600020F47D0008600846006840F49A0008606C
:103F70005A48006840F080705849086000BF5748B0
:103F8000006800F000700028F9D05448083000683C
:103F900020F003005149083108600846006840F0ED
:103FA0000300086000BF4D480830006800F00C00B6
:103FB0000C28F8D10CBD10B54848006840F480705A
:103FC0004649086045480830006847490840434969
:103FD0000831086041480068444908403F4908608A
:103FE0000846006820F4802008603C4808300068DB
:103FF00020F47D003949083108600020091D08605F
:10400000FFF758FF4FF000603949086010BD70B5E8
:1040100000220020002100240023304D08352D68A7
:1040200005F00C0232B1042A10D0082A12D00C2A52
:1040300039D113E0294D2D1D2D68C5F342335D1C88
:104040000126AE40F5032B4E356038E02A4D294E4F
:10405000356034E0294D274E356030E01F4D08357E
:104060002D6805F470101D4D08352D6805F44001CC
:10407000234D05EB90452878012505EB9151174D0F
:1040800008352D6805F4803434B91B4D4543B5FB24
:10409000F1F5184E356005E0184D4543B5FBF1F5D7
:1040A000144E35600BE00D4D2D1D2D68C5F34233C8
:1040B0005D1C0126AE40F5030E4E356000BF00BF0B
:1040C000064D08352D68C5F303150E4E725D094D7A
:1040D0002D68D540074E356070BD000000380240A5
:1040E000003C0240007000400CC0FF88FEFFFEEE66
:1040F00008ED00E0D86200200024F40000127A00ED
:10410000DC620020E5620020704710E000BFBFF3D2
:104110004F8F0B48006800F4E0600A490843001D17
:1041200007490860BFF34F8F00BF00BFFEE7EDE710
:1041300000BFFEE700BFFEE700BFFEE770470000DC
:104140000CED00E00000FA051A48006840F08070AD
:10415000184908600020184948600846006840F087
:1041600001000860704730B5134C63680021134CA0
:104170002468134DB4FBF5F404FB00F202E00E4C8E
:104180006468E11A9142FAD330BD10B504464FF489
:104190007A7104FB01F0FFF7E6FF10BD10B50021B6
:1041A0000246054C636802E0034C6468E11A9142E0
:1041B000FAD310BDFCED00E0001000E0D862002052
:1041C00040420F0070B504460D4629462046FEF7D2
:1041D000F8FE00BF40212046FEF7A3FF0028F9D0DB
:1041E00070BD70B505460C4604E021782846FFF7FF
:1041F000E9FF641C20780028F7D170BD70B5044633
:104200000D4640217748FEF799FFE1B27548FEF769
:10421000D8FE00BF80217348FEF783FF0028F9D045
:10422000204670BD1CB500216F48FEF79FFE6E480A
:10423000FEF7D4FD01210220FCF764FEC0200090AF
:1042400001208DF8040000208DF8060001208DF873
:10425000070000208DF8050069466448FCF776FBEE
:1042600040216248FCF7ECFB80216048FCF7E8FB4A
:104270001CBD10B588B00446FFF7D4FF01205C498F
:10428000087001218003FCF74EFE01210846FCF76F
:1042900039FE5548FEF7A2FD4FF4C060029002209F
:1042A0008DF80C008DF80D0000208DF80E00012017
:1042B0008DF80F0002A94F48FCF748FB4FF48060CF
:1042C000029002A94B48FCF741FB0722092149480B
:1042D000FCF7C5FB07220A214648FCF7C0FB049403
:1042E0000020ADF81400ADF81600ADF81800ADF8D8
:1042F0001C000C20ADF81A0004A93B48FEF7B1FDE4
:10430000012240F225513848FEF7E6FE25208DF8BF
:10431000040003208DF8050000208DF80600012020
:104320008DF8070001A8FBF71EFF01212E48FEF7BC
:104330001DFE40212C48FEF701FF08B010BD1CB542
:1043400000212948FEF712FE2748FEF747FD01210C
:104350000846FCF7D7FD4FF4C060009001208DF8AF
:10436000040000208DF8060001208DF807000020D1
:104370008DF8050069461F48FCF7E8FA4FF4007114
:104380001C48FCF75DFB4FF480611A48FCF758FBB2
:104390001CBD10B51648007818BB40F225511248D4
:1043A000FEF7D5FEE8B11048FEF70FFEC4B204F0E8
:1043B0007F041148008800F4004090B90E4800883E
:1043C000642808DA0C4801880088401C0A4A1080DA
:1043D0000A48445405E00848008840F40040064973
:1043E000088010BD00440040003801400004024035
:1043F0006D6200200000024024630020A3690020B9
:10440000F0B5B1B0012563480068309001264FF443
:104410004070FBF7A3FE62B6FFF796FE01F0FDF9D0
:104420004FF4165003F01EFC02F086FB04460122F6
:1044300030A9BC2000F03AFE9DF8C000312828D1F8
:104440005548007820F0010053490870084600786C
:1044500020F0020008700846007820F0080008707C
:104460000846007820F0200008700846007820F008
:104470001000103008700846007820F00400087022
:10448000002430208DF8C000012230A9BC2000F0AB
:1044900036FE02F0BEF900F0A5F910213F48FCF706
:1044A000CFFA4FF480513D48FCF7CAFA4FF416504A
:1044B00001F034F94FF4165000F02AFD4FF4E130CA
:1044C00002F09EFD00F080F80BF0BEFA0AF06DFCE1
:1044D0000120FCF795FB012231498C2000F0E6FD1C
:1044E00001A800F0A4FEBA2201A92E480BF0CCFBD3
:1044F0002B480078012805D12BA12A48A6300BF0C3
:10450000E7FB98B900F0FFFF01220021B42000F082
:104510005CFE01A800F08BFEBA2201A921480BF035
:10452000B3FB01221E498C2000F0C0FD44BB0120DA
:104530002049487102F0D4F90BF004FB1E48807842
:104540001D4949781C4FCDE900103B787A7A397AB9
:10455000786801F0B4FF022218A1AA2000F0CFFD74
:1045600008F0A3F81649174802F035F840F6B830BD
:10457000FFF70BFE4FF480510848FCF763FA01E0A7
:1045800001F090FF0E490F4802F025F800BF31B04E
:10459000F0BD0000203B02081E6300200000024026
:1045A000F8620020C9650020534D2D313030304D68
:1045B000000000003D630020847F002032300000B6
:1045C0005B6400205164002000B589B00120FCF735
:1045D000A1FB00BF2120FCF74DFB0028FAD00121F0
:1045E0000420FCF78FFC2020079003208DF820008A
:1045F00000208DF8230007A96B48FCF7A7F90121DB
:104600004802FCF790FC00208DF808008DF80900A6
:1046100004900590019001208DF8180001A96348CD
:10462000FBF71AFE0120FBF791FE01215F48FBF723
:1046300053FE5F4800885F49088009B000BD10B58F
:10464000044601215C48FCF7FBF9072301222146BF
:104650005648FBF78AFE5548FBF733FF00BF02219F
:104660005248FCF761F80028F9D05048FBF765FF85
:1046700010BD2DE9F047044601214F48FCF7E0F951
:104680001120FFF7DCFF4D4908802046FFF7D7FFD8
:1046900007464A4800880BF0BFFD80464548008821
:1046A0000BF0BAFD814646490BF0B5FB0646414684
:1046B0000BF0E3FB4349086038460BF0ADFD804644
:1046C00041490BF0DAFB06463E48016830460BF0E4
:1046D000A2FB05462846BDE8F0872DE9F34F83B0DD
:1046E0000C464FF00009CA4611E00398FFF7A7FFF8
:1046F00006460BF091FD054649460BF034FB81461A
:104700000A20FFF742FD0AF1010000F0FF0AA2456E
:10471000EBDB20460BF080FD0146019048460BF094
:10472000ACFB294902900BF0A8FB83460BF0C2FDBD
:1047300007464FF06632254B0BF084FC05460BF024
:10474000CCFD8146484605B0BDE8F08F10B501218B
:104750001948FCF775F910BD10B501211648FCF792
:1047600071F910BD70B50A210F20FFF7B6FF04469E
:104770004FF4FA70FFF709FD0A210F20FFF7ADFF94
:104780000446134920460BF046FB044611480460DA
:1047900020460BF08FFD05462A460B460EA1104819
:1047A0000DF038FE70BD00000008024000240140FA
:1047B000F800F81F1063002000040240126300207C
:1047C000000040401463002000F07F4566660A4008
:1047D000919B974008630020252E33662C00000033
:1047E000527100201CB501210720FCF78BFB41F220
:1047F0002300009001208DF8040000208DF80600B1
:1048000001208DF8070000208DF805006946274833
:10481000FCF79CF841F61010009001208DF8040080
:1048200000208DF8060001208DF8070000208DF88B
:10483000050069461E48FCF789F8012000908DF8B4
:10484000040000208DF8060001208DF807000020EC
:104850008DF8050069461748FCF778F801211348E0
:10486000FCF7F0F84FF480511048FCF7EBF8022108
:104870000E48FCF7E7F84FF480510D48FCF7E2F8DA
:1048800010210B48FCF7DEF801210A48FCF7DAF8A2
:104890004FF400610648FCF7D5F820210348FCF7E7
:1048A000D1F84FF44870FFF770FC1CBD00040240C3
:1048B000000002400008024000B587B00121062038
:1048C000FCF720FB01208DF8180000208DF81A005D
:1048D00001208DF81B0002208DF819004020059062
:1048E00005A94948FCF732F840214748FCF7A8F8E9
:1048F00002208DF8180000208DF81A0002208DF893
:1049000019004FF46040059005A94048FCF71EF8D7
:104910004FF460413D48FCF793F805220D213B48D8
:10492000FCF79DF805220E213848FCF798F805227F
:104930000F213648FCF793F801218803FCF704FBAC
:104940000020ADF800004FF48270ADF802000020A6
:10495000ADF80400ADF80600ADF808004FF40070A3
:10496000ADF80A001020ADF80C000020ADF80E00E4
:104970000720ADF8100069462548FDF75DFA0121D2
:104980002348FDF7F7FA07B000BD00F00700204903
:1049900009884FF6C77211401D4A118011460988D7
:1049A00041EAC00111801146098841F0400111809F
:1049B00070470246002107E0481C81B24FF6FE70A6
:1049C000814201DB0020704711480830008800F068
:1049D00002000028F0D00E480C300280002107E0D1
:1049E000481C81B24FF6FE70814201DB0020EAE7ED
:1049F00007480830008800F001000028F0D0044883
:104A00000C300088C0B2DEE700080240000402401B
:104A10000038004010B504462046FFF7CAFF10BD1D
:104A200010B53820FFF7B1FF10BD10B50020FFF71B
:104A3000ACFF10BD10B5FFF73FFFFFF7F6FF10BD4D
:104A400010B54021FC48FBF7FBFFFF20FFF7E2FF1A
:104A500010BD10B5002400BFFF20FFF7DBFFFF28CB
:104A600001D1002010BD641C6FF07F408442F3D35D
:104A70000120F7E710B54021EF48FBF7E3FFFFF710
:104A8000E8FF08B9002010BDFFF7DAFF0120FAE7C0
:104A900070B505464FF6FF7401E0601E84B2FF203A
:104AA000FFF7B8FFA84201D0002CF6D10CB9FF20C7
:104AB00070BD0020FCE770B504460D46FE20FFF7F0
:104AC000E7FF08B1012070BD04E0FF20FFF771FF90
:104AD0002070641C281EA5F101018DB2F5D1FF20C4
:104AE000FFF798FFFF20FFF795FF0020EBE770B579
:104AF00006460D46FFF7ADFF08B1012070BD284600
:104B0000FFF788FFFD2D19D0002404E0305DFFF78A
:104B100050FF601C84B2B4F5007FF7DBFF20FFF785
:104B200079FFFF20FFF776FFFF20FFF773FF0446B2
:104B300004F01F00052801D00220DFE70020DDE798
:104B40002DE9F04105460C4617464FF00008FFF7E7
:104B500077FFFFF78FFF10B1FF20BDE8F08145F030
:104B60004000FFF757FF200EFFF754FFC4F3074044
:104B7000FFF750FFC4F30720FFF74CFFE0B2FFF749
:104B800049FF3846FFF746FF0C2D02D1FF20FFF703
:104B900041FF4FF01F0800BFFF20FFF73BFF064615
:104BA00006F0800030B1B8F10000A8F1010101F079
:104BB000FF08F1D13046D0E770B50546012200214B
:104BC0000A20FFF7BDFF044624B910212846FFF74D
:104BD00072FF0446FFF734FF0CB1012070BD0020C6
:104BE000FCE770B50546012200210920FFF7A8FF68
:104BF000044624B910212846FFF75DFF0446FFF75D
:104C00001FFF0CB1012070BD0020FCE77FB5684696
:104C1000FFF7E7FF10B1002004B070BD9DF8000061
:104C200000F0C000402809D19DF809009DF8081047
:104C300000EB0120401C84B2A50220E09DF8050095
:104C400000F00F009DF80A1000EBD1109DF809103C
:104C500001F0030100EB4100861C9DF80800801163
:104C60009DF8071000EB81009DF8061001F003018C
:104C700000EB8120441CA6F1090004FA00F5284647
:104C8000CAE7F8B5FFF7D6FEFFF7CAFE002504E035
:104C9000FF20FFF7BFFE681C85B20A2DF8DB142643
:104CA00000BF952200210846FFF74AFF0446012C69
:104CB00004D0301EA6F101018EB2F2D100205F496E
:104CC0000870012C4AD187224FF4D5710820FFF7D4
:104CD00037FF012847D1002506E0FF20FFF79AFEA5
:104CE0000DF80500681C85B2042DF6DB9DF8020066
:104CF000012879D19DF80300AA2875D14FF6FE76D8
:104D000000BF012200213720FFF71AFF012291077F
:104D10002920FFF715FF044624B1301EA6F101013A
:104D20008EB2EED1002E5FD0012200213A20FFF793
:104D300007FF002858D1002506E0FF20FFF76AFE94
:104D40000DF80500681C85B2042DF6DB9DF8000007
:104D500000F0400018B106203849087044E00420F3
:104D60003649087040E0012200213720FFF7E8FEB5
:104D7000012200212920FFF7E3FE0446012C17DC65
:104D800002202E4908704FF6FE7600BF0122002156
:104D90003720FFF7D5FE012200212920FFF7D0FEA2
:104DA0000446BCB1301EA6F101018EB2EED111E075
:104DB0000120224908704FF6FE7600BF0122002133
:104DC0001046FFF7BDFE044624B1301EA6F10101D6
:104DD0008EB2F3D12EB1012251021020FFF7B0FEA6
:104DE00010B1002015490870FFF72AFEFFF71DFEDD
:104DF0001248007808B10020F8BD0CB12046FBE74E
:104E0000AA20F9E72DE9F04106460F4615460B4862
:104E10000078062800D07F02012D11D101223946E9
:104E20001120FFF78DFE044624BB69023046FFF7D0
:104E300042FE04461EE00000000802401863002005
:104E4000012239461220FFF77BFE044600BF4FF4D3
:104E500000713046FFF72FFE044606F50076681E07
:104E6000C0B2051E01D0002CF1D0012200210C207F
:104E7000FFF766FEFFF7E4FD2046BDE8F0812DE96F
:104E8000F04106460F46154620480078062800D017
:104E90007F02012D0CD1012239461820FFF750FE68
:104EA00004466CBBFE213046FFF721FE044627E096
:104EB00016480078012809D0012200213720FFF789
:104EC0003FFE012229461720FFF73AFE012239460C
:104ED0001920FFF735FE044694B900BFFC21304687
:104EE000FFF705FE044606F50076681EC0B2051EF3
:104EF00001D0002CF2D0FD210020FFF7F8FD044680
:104F0000FFF79EFD2046BDE8F081000018630020F9
:104F100010B588B0044601218804FCF715F801217A
:104F20000220FBF7EFFF5B48FDF758FF4FF44060AE
:104F3000029002208DF80C008DF80D0000208DF8F5
:104F40000E0001208DF80F0002A95348FBF7FEFC6C
:104F500007220A215048FBF782FD07220B214E4809
:104F6000FBF77DFD04940020ADF81400ADF81600A9
:104F7000ADF81800ADF81C000C20ADF81A0004A91B
:104F80004448FDF76EFF01214248FDF7EFFF012283
:104F900040F225513F48FEF79FF827208DF8040086
:104FA00002208DF8050000208DF8060001208DF804
:104FB000070001A8FBF7D7F840213648FEF7BEF8F6
:104FC00008B010BD10B540F225513248FEF7BFF8C9
:104FD00000283AD02F48FDF7F8FFC4B2242C02D1A4
:104FE00000202E4908802D490888411C2B4A118039
:104FF0002B490C540846007824281FD10846007914
:105000004D281BD108464079432817D10A2C15D1C9
:10501000502124480AF051FE2048028820492148A6
:105020000AF032FE01201F4981F8A00000201B4930
:1050300008804FF480711A480AF03FFE1748008834
:10504000FF2802DB00201549088010BD0FB438B5D9
:1050500005A800901448009A04990DF0EFF900207B
:10506000009011480AF050FE85B200240DE000BF08
:1050700040210848FEF755F80028F9D00A48015D9C
:105080000448FDF79EFF601C84B2AC42EFDB38BCE5
:105090005DF814FB00480040000402401A63002041
:1050A00065640020767D00206565002030B5FE4CEB
:1050B000031903E013F8014B01F8014B141EA2F190
:1050C0000105AAB2F6D130BD30B5F74C031903E0A3
:1050D0001C8821F8024B0833141EA2F10105AAB264
:1050E000F6D130BD30B5F04C031902E01C6810C198
:1050F0001033141EA2F10105AAB2F7D130BD30B5AC
:10510000E94C0319E94CEA4D2C60EA4C2C6000BFD5
:10511000E74C083C246804F00104002CF8D1E44C6E
:10512000083C246844F48074E14D083D2C600BE099
:1051300011F8014B03F8014B00BFDD4C0C3424681F
:1051400004F00104002CF8D1141EA2F10105AAB24A
:10515000EED1D74C083C246844F00104D44D083DFE
:105160002C6030BD30B5D04C0319D04CD04D2C60E4
:10517000D04C2C6000BFCE4C083C246804F00104E5
:10518000002CF8D1CA4C083C246844F48074C84D03
:10519000083D2C600BE031F8024B1C60083300BF67
:1051A000C34C0C34246804F00104002CF8D1141E04
:1051B000A2F10105AAB2EED1BD4C083C246844F02E
:1051C0000104BB4D083D2C6030BD30B5B64C031911
:1051D000B64CB74D2C60B74C2C6000BFB44C083CAB
:1051E000246804F00104002CF8D1B14C083C246878
:1051F00044F48074AE4D083D2C600AE010C91C6078
:10520000103300BFAA4C0C34246804F00104002CB5
:10521000F8D1141EA2F10105AAB2EFD1A44C083CAA
:10522000246844F00104A24D083D2C6030BD10B547
:10523000B0B00446BC2101A80AF03FFD142201A928
:105240000020FFF733FF0A2206A91420FFF72EFFE4
:105250000A220DF136011E20FFF728FF142210A9A3
:105260003C20FFF723FF14220DF122012820FFF735
:105270001DFF062215A96420FFF718FF05220DF176
:105280005A016E20FFF712FF06220DF15F01782010
:10529000FFF70CFF0A220DF165018220FFF706FFE0
:1052A0000F220DF16F019620FFF700FF02220DF192
:1052B0007E01A620FFF7FAFE012220A9B920FFF700
:1052C000F5FE01220DF18101BA20FFF7EFFE142255
:1052D0000DF18201F020FFF7E9FE14220DF1960195
:1052E0004FF48270FFF7E2FE14220DF1AA014FF491
:1052F0008C70FFF7DBFEBA2201A920460AF0C4FC3D
:1053000030B010BD18B500200090002400BF05E0AB
:10531000A0B201226946FFF7F2FE641CB4F5967F45
:10532000F6DB18BD0FB410B5FFF7ECFF02A80AF0CA
:10533000EBFC84B2224602A90020FFF7E0FE07A89A
:105340000AF0E2FC84B2224607A91420FFF7D7FE38
:105350000DF13A000AF0D8FC84B222460DF13A0170
:105360001E20FFF7CCFE11A80AF0CEFC84B2224624
:1053700011A93C20FFF7C3FE0DF126000AF0C4FC82
:1053800084B222460DF126012820FFF7B8FE16A8A8
:105390000AF0BAFC84B2224616A96420FFF7AFFED9
:1053A0000DF15E000AF0B0FC84B222460DF15E0100
:1053B0006E20FFF7A4FE0DF163000AF0A5FC84B295
:1053C00022460DF163017820FFF799FE0DF1690087
:1053D0000AF09AFC84B222460DF169018220FFF79F
:1053E0008EFE0F220DF173019620FFF788FE012239
:1053F0000DF18201A620FFF782FE012221A9B9202A
:10540000FFF77DFE01220DF18501B920FFF777FE40
:10541000012229498C20FFF772FE0DF186000AF067
:1054200073FC84B222460DF18601F020FFF767FE7F
:105430000DF19A000AF068FC84B222460DF19A013F
:105440004FF48270FFF75BFE0DF1AE000AF05CFCDA
:1054500084B222460DF1AE014FF48C70FFF74FFE7F
:1054600010BC5DF814FB10B5142114480AF025FC9B
:1054700012480021416181618183323001604160C5
:10548000018114210A300AF018FC14210B481E3047
:105490000AF013FC094800210165A0F854105630A9
:1054A00001600171401D0BE000000808EFCDAB89E1
:1054B0000C3C024005040302F8620020C96500208C
:1054C00001608180801D0160416001810F210A30EF
:1054D0000AF0F3FB65480021A0F87A1014217E3011
:1054E0000AF0EBFB1421614892300AF0E6FB14212C
:1054F0005E48A6300AF0E1FB00205C4981F87C00A0
:1055000081F87D0010BD00B5DBB0FFF7ACFF58A2FD
:105510005CA156480CF07EFF5BA25AA153481430A0
:105520000CF078FF5AA257A1504832300CF072FFAD
:1055300059A254A14D483C300CF06CFF59A251A126
:105540004A481E300CF066FF59A24EA14748503021
:105550000CF060FF58A24BA1444856300CF05AFFA3
:1055600056A248A141485B300CF054FF54A245A11B
:105570003E4861300CF04EFF54A242A13B486B30D4
:105580000CF048FF55A23FA138487A300CF042FF9A
:1055900053A23CA135487E300CF03CFF53A239A108
:1055A000324892300CF036FF53A236A12F48A63075
:1055B0000CF030FF00202D4981F87C0081F87D003F
:1055C000AA22103168460AF05FFBBA2227492CA8AC
:1055D0000AF05AFB2CA80FC8FFF7A4FE0120494986
:1055E000087001228C20FFF78AFD5BB000BD2DE919
:1055F000F0410546002628460AF086FB87B2082FB0
:1056000002DD0020BDE8F081002416E0285D30288E
:105610000FDB285D39280CDC002C05DD06EB86004D
:105620004FF6FF7101EA4006285D3038304486B2FB
:1056300001E00020E6E7601C84B2BC42E6DB3046B5
:10564000E0E710B509485030FFF7D1FF0446C4EB3E
:105650000410800010BD10B504485B30FFF7C7FF91
:105660000446C4EB04108000783010BDC9650020EA
:105670002233392E3130352E3233302E3139372224
:1056800000000000257300003138383300000000AE
:10569000383038300000000038383838383838387A
:1056A000000000006C6963617769666900000000B2
:1056B0003030303031000000303000003500000064
:1056C0003132333435363738390000003230323237
:1056D00031313330313134343030000030000000AB
:1056E000226C696368616F2200000000223931304A
:1056F000353137406C632200534D2D313030304D01
:1057000000000000F862002010B50020FE4908806B
:105710004FF4C871FD480AF0D0FA10BD10B588B03A
:10572000044601214804FBF70FFC01210846FBF762
:10573000E9FBF748FDF752FB0C20029002208DF8A0
:105740000C008DF80D0000208DF80E0001208DF862
:105750000F0002A9EF48FBF7F9F807220221ED48F4
:10576000FBF77DF907220321EA48FBF778F9049457
:105770000020ADF81400ADF81600ADF81800ADF833
:105780001C000C20ADF81A0004A9E148FDF769FBE4
:105790000121DF48FDF7EAFB012240F22551DC48F8
:1057A000FDF79AFC26208DF8040003208DF80500F3
:1057B00000208DF8060001208DF8070001A8FAF7F7
:1057C000D2FC4021D248FDF7B9FC08B010BD0FB49F
:1057D00038B5FFF799FF05A80090CF48009A0499C3
:1057E0000CF02CFE00200090CB480AF08DFA85B218
:1057F00000240DE000BF4021C548FDF792FC0028C1
:10580000F9D0C548015DC248FDF7DBFB601C84B2DE
:10581000AC42EFDB38BC5DF814FB1FB50121084634
:10582000FBF792FB40F2E730029040F67F40ADF884
:1058300004000120ADF80C000020ADF8060001A91D
:105840004FF08040FCF732FE012211469007FDF731
:10585000BAF901218807FDF7DEF900214FF08040F9
:10586000FCF79EFE1C208DF8000001208DF8010041
:1058700000208DF8020001208DF803006846FAF739
:1058800072FC01218807FCF78BFE1FBD10B5044692
:105890004CB100214FF08040FCF742FE0121880707
:1058A000FCF77EFE04E000214FF08040FCF778FE1C
:1058B00010BD10B501218807FDF79CF938B1012111
:1058C0008807FDF7A8F901F096FA9449087010BD11
:1058D00010B540F225518E48FDF739FCD8B18C48FF
:1058E000FDF773FBC4B28848008800F4004090B90B
:1058F00085480088B0F5C77F07DC83490888411CCC
:10590000814A118081490C5405E07F48008840F4A9
:1059100000407D49088010BD2DE9F047ADF5287D98
:105920000026B046602190A80AF0C7F97C480068BC
:105930008F9000208C908D9089908A908B902BA8CE
:10594000FFF775FCBC222BA95AA80AF09DF975A196
:105950006E480AF0BDF990B1FFF7D5FD01227449F8
:105960008C20FFF7A3FB7248007820B171A10D20B5
:1059700007F0D0F903E073A10D2007F0CBF975A172
:1059800062480AF0A5F900287ED074495F480AF001
:105990009FF910B14FF0010901E04FF000096F4984
:1059A00011395A480AF094F908B1012000E00020AA
:1059B00009EA000969490A3154480AF089F908B12D
:1059C000012000E0002009EA0009644919314F482C
:1059D0000AF07EF908B1012000E0002009EA000980
:1059E0005E49891F49480AF073F908B1012000E0B7
:1059F000002009EA0009B9F1000F0AD00020574938
:105A0000613981F87C0001220021B920FFF777FB82
:105A100009E001205149613981F87C0001227C3183
:105A2000B920FFF76CFB64218FA80AF046F9002625
:105A3000B2E036B947A135480AF04AF90446A41D38
:105A4000A8E0641C46A120460AF042F9051E49D090
:105A5000012E06D0022E0ED0032E2AD0042E3FD1C6
:105A600033E03E4800210160416001812A1B21464C
:105A70000AF00AF900BF394861380021016580F851
:105A800054102A1B214600E0E2E050300AF0FCF8F6
:105A900032481138FFF7ABFD8046304861380021AD
:105AA000016580F8541042462EA150300CF0B2FC33
:105AB00017E00F2129480A300AF0FFF82A1B214677
:105AC00026480A300AF0E0F80BE02448613800214B
:105AD00080F87A102A1B21467A300AF0D5F800E0C7
:105AE00000BF00BF2C46042E54D1641C1EA12046CA
:105AF0000AF0EEF805461948801F002101608180F8
:105B00002A1B214632E000001C630020836600202F
:105B10000044004000000240136800207962002029
:105B2000243B0208706172772D72737400000000CC
:105B3000F8620020706172772D7273742C4F4B2CB9
:105B40002A000000706172772D7273742C6661698F
:105B50006C2C2A00706172772D3100002A660020BB
:105B60002C000000256400002C2A00000AF08CF8AC
:105B7000FA48FFF73CFD8046B8F1010F01DA4FF01B
:105B80000108F6480021016081804246AFF22C01F5
:105B90000CF040FC701CC6B2052EFFF64AAFEF4871
:105BA0000B38FFF724FD012805DAEDA2EEA1EB4842
:105BB0000B380CF02FFCAA22E8494B3968460AF052
:105BC00063F8BA22E5495B392BA80AF05DF82BA8E7
:105BD0000FC8FFF7A7FBE5A10B2007F09BF8DF49F3
:105BE000891D0DF2C9100AF096F8C8B9DB490B39C6
:105BF0006EA80AF090F898B9D84910310DF2D31078
:105C00000AF089F860B9D5491F310DF5F1700AF035
:105C100082F828B9D1490DF2C3100AF07CF848B1D6
:105C20000120CE495B3981F87C0001227C31B9200A
:105C3000FFF765FAC9485B3890F87A00312805D13A
:105C4000FDF7C8FA10B101F068F801E001F0B9F809
:105C5000C9A1CB480AF03CF810B14FF0010901E0AE
:105C60004FF00009C7A1C6480AF032F808B1012078
:105C700000E0002009EA0009B9F1000F75D0B7492A
:105C80005B39BF480AF024F810B14FF0010901E078
:105C90004FF00009B1494739B9480AF019F808B17D
:105CA000012000E0002009EA0009AC493D39B44870
:105CB0000AF00EF808B1012000E0002009EA00090E
:105CC000A6491F39AE480AF003F808B1012000E0E8
:105CD000002009EA0009A1492939A94809F0F8FF7B
:105CE00008B1012000E0002009EA0009B9F1000F25
:105CF0000AD0002099495B3981F87C0001220021FB
:105D0000B920FFF7FCF909E0012094495B3981F8DB
:105D10007C0001227C31B920FFF7F1F900264FE029
:105D200036B995A1964809F0D3FF0446A41D45E075
:105D3000641CAFF2D411204609F0CAFF051E3CD006
:105D4000012E06D0022E11D0032E1BD0042E32D1EC
:105D500024E0142181485B3809F0AFFF2A1B21465B
:105D60007E485B3809F090FF26E06FE07B485B38A7
:105D700000214161816181832A1B2146143009F091
:105D800083FF19E0142175483D3809F096FF2A1B5E
:105D9000214672483D3809F077FF0DE06F485B38C7
:105DA0000021C1630164A0F844102A1B21463C3045
:105DB00009F06AFF00E000BF00BF2C46701CC6B2AD
:105DC000052EADDB65485B38D4F80110C0F8321001
:105DD000AA2200F11001684609F056FFBA225F4975
:105DE0005B392BA809F050FF2BA80FC8FFF79AFAD0
:105DF00065A10B2006F08EFF58495B395AA809F0BF
:105E00008AFFC8B9554947395FA809F084FF98B996
:105E100052493D390DF5C37009F07DFF60B94F4916
:105E20001F3969A809F077FF30B94C4929390DF5B8
:105E3000CD7009F070FF48B1012048495B3981F805
:105E40007C0001227C31B920FFF759F951A14C485F
:105E500009F03EFF20B351A1494809F039FF041E63
:105E600019D051480078C0F300104F490978C1F3A8
:105E70008001084320B14DA10B2006F04BFF0AE042
:105E80004D48007820F0200020304B49087047A191
:105E90000B2006F03FFF49A1394809F019FF0446DD
:105EA00049A1374809F014FF041E56D064218FA879
:105EB00009F003FFE41D0D2221468FA809F0E4FE3E
:105EC0009DF8410230389DF84012303901EB8101D4
:105ED00000EB41000C2801DD012100E000219DF8CC
:105EE000430230389DF84222303A02EB820200EB46
:105EF00042001F2801DD012000E0002008439DF83A
:105F0000451230399DF84422303A02EB820201EB0F
:105F10004201172901DD012100E0002108439DF81D
:105F2000471230399DF84622303A02EB820201EBEB
:105F300042013B2901DD012100E0002108439DF8D9
:105F4000491230399DF84822303A02EB820201EBC7
:105F500042013B293CDD01213BE003E124660020B6
:105F600030303030310000002573000070617277EE
:105F70002D312C4F4B2C2A00706172772D3200008E
:105F80008366002022000000706172772D322C4F52
:105F90004B2C2A00706172772D330000706172778C
:105FA0002D332C3100000000716200207061727787
:105FB0002D332C4F4B2C2A001E630020706172770A
:105FC0002D332C3000000000706172772D340000FA
:105FD0000021084320B1C3A10D2006F09BFEC1E0C3
:105FE0009DF8490230389DF84812303901EB8101A3
:105FF00000EB41019DF8470230389DF84622303AC7
:1060000002EB820200EB4200CDE900019DF845C29F
:10601000ACF1300C9DF84492A9F1300909EB8909E3
:106020000CEB49039DF843C2ACF1300C9DF8429251
:10603000A9F1300909EB89090CEB49029DF841C22D
:10604000ACF1300C9DF84092A9F1300909EB8909B7
:106050000CEB49019DF83FC2ACF1300C9DF83E922B
:10606000A9F1300909EB89090CEB490000F027FA86
:106070009DF8490230389DF84812303901EB810112
:1060800000EB4100C1B29DF8470230389DF846222E
:10609000303A02EB820200EB4200C0B2CDE90001CF
:1060A0009DF845C2ACF1300C9DF84492A9F130093D
:1060B00009EB89090CEB490C0CF0FF039DF843C276
:1060C000ACF1300C9DF84292A9F1300909EB890935
:1060D0000CEB490C0CF0FF029DF841C2ACF1300C06
:1060E0009DF84092A9F1300909EB89090CEB490CA4
:1060F0000CF0FF019DF83FC2ACF1300C9DF83E92D0
:10610000A9F1300909EB89090CEB490C0CF0FF00EF
:1061100009F0CCFC02228FA9AA20FEF7F0FF7548F7
:10612000006800F4807020B1FFF795FA814600F016
:10613000E0FB7048006800F4007030B1FFF781FAAE
:10614000A0F10109484600F017FB6BA10B2006F0F7
:10615000E1FD01206B4981F87C0001220021B9207A
:10616000FEF7CDFF68A16A4809F0B2FD041E19D000
:10617000AFF21461204609F0ABFD0446641CA51C77
:106180002978207809F08BF8287809F0B6F80746C6
:1061900027B960A10B2006F0BDFD03E060A10D2032
:1061A00006F0B8FD62A15A4809F092FD041E2AD0FB
:1061B00064218FA809F081FD2BA8FFF738F8BA22D7
:1061C0002BA9504809F060FD4E485B30FFF70FFAED
:1061D00081464C485030FFF70AFA824649487A30E7
:1061E000A0F10F015346A0F11902CDE90109009178
:1061F00051A18FA80CF00EF98FA809F085FD8146FA
:106200008FA906F087FD52A1414809F061FD00B356
:1062100064218FA809F051FD89A98CA800F0DBF951
:106220003849323101F10A00A0F11E02A0F1280321
:10623000CDE90032CDE90201143B45A246A18FA869
:106240000CF0E8F88FA809F05FFD81468FA906F0F1
:1062500061FD46A12E4809F03BFDD8B164218FA80D
:1062600009F02BFD89A98CA800F0B5F902228EA9AE
:10627000AA20FEF71BFF8CA889AB8EAA3DA1009037
:106280008FA80CF0C7F88FA809F03EFD81468FA9B2
:1062900006F040FD3CA11E4809F01AFD041E1CD06A
:1062A00064218FA809F009FD2BA8FEF7C0FFBA22D0
:1062B0002BA9144809F0E8FC12486130FFF797F960
:1062C00081464A4632A18FA80CF0A4F88FA809F0A5
:1062D0001BFD81468FA906F01DFD0DF5287DBDE84B
:1062E000F0870000706172772D342C6661696C2C28
:1062F0002A00000008280040706172772D342C4F6E
:106300004B2C2A00C9650020706172772D35000082
:1063100083660020706172772D352C4F4B2C2A003C
:10632000706172772D352C6661696C2C2A00000033
:10633000706172722D310000706172722D312C25E6
:10634000732C25642C25732C25732C25642C2A0092
:10635000706172722D32000025732C25732C257309
:106360002C25732C25732C25732C2A0070617272D6
:106370002D340000706172722D342C25732573202A
:1063800025732C2A00000000706172722D733F008B
:10639000706172722D362C25642C2A0000B585B0F0
:1063A00001210420FAF7AEFD00208DF804008DF8DD
:1063B00006004FF40050009002208DF80700694657
:1063C000FE48FAF7C3FA00220D21FC48FAF747FB12
:1063D0004FF48010FAF752FA4FF480100290012027
:1063E0008DF80E0000208DF80C0008208DF80D00AF
:1063F00002A8FAF7CCF903208DF8100001208DF8DF
:10640000130000208DF811008DF8120004A8F9F790
:10641000AAFE4FF40030FAF731FA4FF40030029040
:1064200000208DF80C0008208DF80D0001208DF85B
:106430000E0002A8FAF7ABF929208DF81000002011
:106440008DF811008DF8120001208DF8130004A8BA
:10645000F9F789FE05B000BD0EB501210807FAF76E
:1064600073FD0120FAF739FB0120FAF756FC00BF53
:106470004920FAF7FFFB0028FAD04FF48030FAF7F2
:1064800019FD0120FAF736FDFAF710FE7F20019082
:1064900000200090FF2002906846FAF7CEFEFFF73A
:1064A0007DFF0EBD10B501210807FAF74DFD012053
:1064B000FAF713FBFAF7FAFDFFF770FF10BD2DE9AD
:1064C000FC4704460D4616461F46DDE90A89F8B228
:1064D0008DF8040008F0FF008DF8050009F0FF00BA
:1064E0008DF8060000208DF8070001A9FAF740FF9B
:1064F000E0B28DF80300E8B28DF80100F0B28DF83B
:10650000020001208DF8000069460020FAF7CEFF56
:1065100043F2F2210020FBF77AFBBDE8FC872DE96E
:10652000FC47A74890F8CA00F0B3A54890F8CC0003
:106530003038A34991F8CB10303901EB810100EBE1
:1065400041049F4890F8CE0030389D4991F8CD1015
:10655000303901EB810100EB4105994890F8D000FA
:106560003038974991F8CF10303901EB810100EBB9
:106570004106934890F8A3003038914991F8A21051
:10658000303901EB810100EB410000F108078C4834
:1065900090F8A50030388A4991F8A410303901EB01
:1065A000810100EB410800E013E0854890F8A70066
:1065B0003038834991F8A610303901EB810100EBA6
:1065C00041093B46324629462046CDE90089FFF77E
:1065D00076FFBDE8FC877CB504460D4601A9002086
:1065E000FAF730FF69460020FAF7C6FF9DF803006E
:1065F0000A2190FBF1F0303028709DF8030090FBE9
:10660000F1F201FB1200303068709DF8010090FB40
:10661000F1F03030A8709DF8010090FBF1F201FB21
:1066200012003030E8709DF8020090FBF1F030303D
:1066300028719DF8020090FBF1F201FB120030304E
:1066400068719DF8040090FBF1F0303020709DF8E7
:10665000040090FBF1F201FB1200303060709DF8F5
:10666000050090FBF1F03030A0709DF8050090FB24
:10667000F1F201FB12003030E0709DF8060090FB53
:10668000F1F0303020719DF8060090FBF1F201FB33
:106690001200303060717CBD70B504460D4609F0C3
:1066A00051FA484840680A21B0FBF1F030302870B8
:1066B00044484068B0FBF1F201FB120030306870D2
:1066C0004048007A90FBF1F03030A8703D48007AE5
:1066D00090FBF1F201FB12003030E8703948407A4B
:1066E00090FBF1F0303028713648407A90FBF1F29F
:1066F00001FB1200303068713248007890FBF1F0F5
:10670000303020702F48007890FBF1F201FB12002E
:10671000303060702B48407890FBF1F03030A07042
:106720002848407890FBF1F201FB12003030E07015
:106730002448807890FBF1F0303020712148807837
:1067400090FBF1F201FB12003030607170BD38B582
:1067500069460020FAF776FE9DF800004FF461616B
:1067600048439DF80110C1EB011100EB81009DF839
:1067700002104418204638BD3EB504464FF4801040
:10678000FAF77CF84FF48010009001208DF8060095
:1067900000208DF8040008208DF805006846F9F700
:1067A000F6FF03208DF8080001208DF80B00002073
:1067B0008DF809008DF80A0002A805E000080240E3
:1067C000767D0020847F0020F9F7CDFC0020FBF7C8
:1067D00032F84FF48060FBF7C4FAB4F5803F06D37B
:1067E0000620FBF703F8A4F57F44FF3C02E00420F9
:1067F000FAF7FCFF2046FBF70EF84FF48040FBF75A
:10680000E0FA01218803FBF765FA0120FBF713F892
:106810003EBD00B585B001210420FAF773FB0020CE
:106820008DF804004FF40050009002208DF807000E
:106830006946F948FAF78AF800220D21F648FAF776
:106840000EF901210846FAF76EFB0D210220FBF735
:106850007CFC4FF40050FAF711F84FF4005002900E
:1068600001208DF80E0000208DF80C0008208DF816
:106870000D0002A8F9F78BFF28208DF810000120E9
:106880008DF8130000208DF811008DF8120004A877
:10689000F9F769FC01210420FAF72EF905B000BDD3
:1068A000014601F5FA6081B2CA1701EB92729210AB
:1068B000A1EB820292B9642091FBF0F200FB12106E
:1068C00050B94FF4C87091FBF0F200FB121008B9F8
:1068D000012070470020FCE70120FAE70020F8E7DC
:1068E00010B5FFF75BFDFFF7B7FD0120FAF788F958
:1068F00010BD30B589B004464FF40030F9F7BEFF43
:106900004FF40030069000208DF81C0008208DF810
:106910001D0001208DF81E0006A8F9F738FF292078
:106920008DF8200000208DF821008DF82200012034
:106930008DF8230008A8F9F716FC4FF48070FBF7D8
:1069400010FA4FF48050FBF73CFA00214FF48070AE
:10695000FAF7ECFE05A90020FAF774FD04A900205F
:10696000FAF70AFE9DF81100401EAC490D5C9DF837
:106970001100022805D19DF81300FFF791FF00B91F
:106980006D1C9DF814004FF4616148439DF815108B
:10699000C1EB011100EB81009DF8161001449DF838
:1069A000120040F2A322504301EBC0100444D00176
:1069B000B4FBF0F0A84207D9D001B4FBF0F0451BBE
:1069C000E8B28DF80C0005E09548B4FBF0F0C0B2D9
:1069D0008DF80C000020029001908DF80300904883
:1069E000B4FBF0F100FB11404FF46161B0FBF1F03A
:1069F000C0B28DF800008A48B4FBF0F100FB1140F2
:106A00004FF46161B0FBF1F201FB12003C21B0FBDD
:106A1000F1F0C0B28DF801008148B4FBF0F100FB49
:106A200011404FF46161B0FBF1F201FB12003C2117
:106A3000B0FBF1F201FB12008DF802006A464FF440
:106A400080710020FAF7BBFD01210803FBF742F932
:106A500001210802FAF76AFE09B030BD2DE9F043C2
:106A600087B08046894614461D46DDE90E674FF41F
:106A70000030F9F703FF4FF40030049000208DF848
:106A8000140008208DF8150001208DF8160004A8C8
:106A9000F9F77DFE29208DF8180000208DF81900E7
:106AA0008DF81A0001208DF81B0006A8F9F75BFB92
:106AB0004FF40070FBF755F94FF40050FBF781F9E4
:106AC00000214FF40070FAF731FEE0B28DF80C00AF
:106AD0000020029001908DF80300E8B28DF80000CC
:106AE000F0B28DF80100F8B28DF802006A464FF45A
:106AF00000710020FAF763FD01214803FBF7EAF873
:106B000001214802FAF712FE07B0BDE8F08310B584
:106B1000002410E04FF400513F48F9F779FF40B1ED
:106B2000601CC4B21E20FDF730FB642C03DB012087
:106B300010BD0020FCE7EDE710B54FF48050FBF7E7
:106B40001FF970B14FF40030F9F798FE4FF4805000
:106B5000FBF737F93348007820F00100401C314939
:106B600008704FF40050FBF70BF970B14FF4003090
:106B7000F9F784FE4FF40050FBF723F92948007819
:106B800020F00200801C274908704FF48040FBF77A
:106B9000F7F870B14FF48010F9F770FE4FF48040B1
:106BA000FBF70FF91F48007820F00400001D1D4975
:106BB00008704FF400511848F9F72AFF88B1FFF721
:106BC000A6FF194908700846007830B115480078CA
:106BD00020F008000830134908704FF40050F9F70E
:106BE0004DFE1048007800F001000E490978C1F30D
:106BF000400108430B490978C1F380010843094962
:106C00000978C1F3C001084328B30648007800F0B2
:106C1000010058B1012010BD00080240283B0208C5
:106C2000805101001E6300207A6200209E48007897
:106C3000C0F3400008B10220EDE79B480078C0F3A4
:106C4000800008B10320E6E797480078C0F3C00051
:106C500050B10420DFE79448007820F01000103095
:106C6000914908700020D6E70020D4E710B54FF412
:106C70008050FBF785F8A0B14FF48050FBF7A1F8E6
:106C80008948007820F00100401C874908700021E5
:106C90004FF48070FAF74AFDFEF7DDFC0446FFF77B
:106CA00028FE4FF40050FBF76BF890B14FF4005002
:106CB000FBF787F800214FF40050FAF737FD7A48C8
:106CC000007820F00200801C774908700120774985
:106CD00008704FF40030F9F7D1FD10BD10B54FF436
:106CE0008040FBF74DF8B8B14FF48040FBF769F8EE
:106CF0000020FAF7A0FD4FF48010F9F7BFFD6A48B5
:106D0000007820F00400001D67490870FEF799FC28
:106D1000441E2046FFF730FD10BD2DE9FE43002143
:106D20004FF48070FAF702FD0020FAF784FD604806
:106D3000D0F86B00029002A809F008F8074600207E
:106D400002905B48B0F86F00ADF8080002A808F0A8
:106D5000FDFF80465648B0F87100ADF8080002A863
:106D600008F0F4FF81465248B0F87300ADF808000F
:106D700002A808F0EBFF06464D48B0F87500ADF8E4
:106D8000080002A808F0E2FF04464948B0F877007E
:106D9000ADF8080002A808F0D9FF054635B93B2533
:106DA00014B93B24761E02E0641E00E06D1E3346DB
:106DB0004A4641463846CDE90045FFF74FFEBDE85B
:106DC000FE8310B53848007820F00100401C364999
:106DD00008700846007820F00400001D08700021AB
:106DE0004FF40070FAF7A2FC10BD10B54FF400503C
:106DF000F9F744FD10BD10B500242E48007820B1ED
:106E0000012818D002284BD133E04FF400512A4812
:106E1000F9F7FEFD18B101202649087002E00020B4
:106E20002449087000202549087008460078244944
:106E30000870002435E04FF400511F48F9F7E8FDD1
:106E400098B11E480078401C1C490870084600781C
:106E50001B49087019480078C82809DBC820174961
:106E6000087002201349087002E0022011490870DE
:106E700017E04FF400511048F9F7CAFD78B9002027
:106E80000C4908700D4800780A2800DD03240B48DF
:106E90000078642800DD042400200849087000E020
:106EA00000BF00BF204610BD1E63002020630020ED
:106EB000C9650020216300200008024022630020F1
:106EC0001F63002010B588B00446002046490870B2
:106ED00001218803FAF727F801210220FAF712F8B6
:106EE0004248FBF77BFFC020029002208DF80C0087
:106EF0008DF80D0000208DF80E0001208DF80F0098
:106F000002A93B48F9F722FD072206213848F9F784
:106F1000A6FD072211463648F9F7A1FD049400208A
:106F2000ADF81400ADF816004FF48060ADF818000D
:106F30000020ADF81C000C20ADF81A0004A92B4865
:106F4000FBF78FFF01212948FCF710F8012240F2DE
:106F500025512648FCF7C0F825208DF804000320B1
:106F60008DF805008DF8060001208DF8070001A8B6
:106F7000F9F7F9F840211D48FCF7E0F808B010BD1A
:106F800010B564211B4808F098FE00201A490880BB
:106F900010BD10B56421194808F08FFE10BD0FB464
:106FA00038B505A800901548009A04990BF046FAE8
:106FB00000200090114808F0A7FE85B200240DE0E3
:106FC00000BF40210948FCF7ACF80028F9D00B4875
:106FD000015D0648FBF7F5FF601C84B2AC42EFDBB5
:106FE00038BC5DF814FB00006D62002000380140E1
:106FF00000040240A369002024630020076A0020E7
:1070000010B588B004460121C804F9F79DFF01219D
:107010000420F9F777FFFD48FBF7E0FE4FF44060EE
:10702000029002208DF80C008DF80D0000208DF8E4
:107030000E0001208DF80F0002A9F548F9F786FC33
:107040004FF40060029002A9F148F9F77FFC082292
:107050000B21EF48F9F703FD08220A21EC48F9F764
:10706000FEFC04940020ADF81400ADF81600ADF855
:107070001800ADF81C000C20ADF81A0004A9E34874
:10708000FBF7EFFE0121E148FBF770FF30208DF8A0
:10709000040005208DF8050000208DF80600012071
:1070A0008DF8070001A8F9F75EF8012240F225519A
:1070B000D648FCF711F84021D448FCF73FF80122EC
:1070C00040F22441D148FCF707F808B010BD10B5D4
:1070D000D048B0F8C80020F40040CE49A1F8C8005C
:1070E0000846B0F8C8006FF30E00A1F8C800C82128
:1070F000C84808F0E2FD10BD10B540F22551C34864
:10710000FCF725F858B3C148FBF75FFFC4B2C1488C
:10711000B0F8C800C0F30E00C7280FDABD49B1F8B7
:10712000C810C1F30E00411CBA4AB2F8C82061F37E
:107130000E02B849A1F8C8200C5410E0B548B0F8C8
:10714000C8006FF30E00B349A1F8C8000846B0F8B4
:10715000C80020F4004000F50040A1F8C800082154
:10716000AA48FBF7F4FF30B1A848FBF72EFF08212F
:10717000A648FBF7E3FF40F22441A448FBF7E7FFF2
:1071800068B1A448B0F8C80020F4004000F5004001
:10719000A049A1F8C8009D48FBF717FFC4B210BD75
:1071A0000FB438B505A800909B48009A04990BF0DD
:1071B00045F900200090984808F0A6FD85B200240B
:1071C0000DE000BF40219148FBF7ABFF0028F9D04C
:1071D0009148015D8D48FBF7F4FE601C84B2AC421F
:1071E000EFDB38BC5DF814FB2DE9F047ADF5287DE9
:1071F0000026B0460020A590A690A290A390A4904F
:107200006422864989A808F03FFD2BA8FEF70FF8F5
:10721000BC222BA95AA808F037FD7E48B0F8C80058
:107220000121B1EBD03F71D17DA17A4808F050FD2A
:10723000B0B1FEF768F901227C498C20FDF736FFDA
:107240007A48007830B100230D2279A1184606F063
:10725000FCF805E000230F2279A1184606F0F5F8A6
:107260007BA16C4808F034FD00287DD064217A4869
:1072700008F023FD002680E036B975A1654808F0C6
:1072800027FD0446A41D76E0641C74A1204608F086
:107290001FFD051E48D0012E06D0022E0ED0032E53
:1072A00028D0042E3ED132E06D48002101604160BB
:1072B00001812A1B214608F0E7FC00BF68486138BD
:1072C0000021016580F854102A1B2146503008F037
:1072D000DBFC63481138FEF78AF980466048613864
:1072E0000021016580F8541042465EA150300BF039
:1072F00091F818E00F215A480A3008F0DEFC2A1BEA
:10730000214657480A3008F0BFFC0CE0FEE3544821
:107310006138002180F87A102A1B21467A3008F063
:10732000B3FC00E000BF00BF2C46042E23D1641C38
:107330004DA1204608F0CCFC05464948801F00219D
:10734000016081802A1B214608F09EFC4448801F72
:10735000FEF74DF98046B8F1010F01DA4FF0010850
:107360003F48801F002100E0ADE00160818042467F
:107370003CA10BF04FF8701CC6B2052EFFF67CAF97
:1073800037481138FEF733F9012805DA37A239A159
:10739000334811380BF03EF8AA223149513968467A
:1073A00008F072FCBA222E4961392BA808F06CFC57
:1073B0002BA80FC8FDF7B6FF00230B222EA11846FD
:1073C00006F043F826490DF2C91008F0A4FCD0B924
:1073D000234911396EA808F09EFCA0B920490A3152
:1073E0000DF2D31008F097FC68B91D4919310DF55D
:1073F000F17008F090FC30B91949891F0DF2C310E3
:1074000008F089FCF0B3012015493CE0004C004035
:1074100000080240AC7C0020CF6A0020343B020808
:10742000706172772D72737400000000F8620020A2
:10743000706172772D7273742C4F4B2C2A000000F0
:10744000706172772D7273742C6661696C2C2A00DE
:10745000706172772D3100006B6A00202C000000F3
:107460002A660020256400002C2A000030303030CD
:107470003100000025730000706172772D312C4FB0
:107480004B2C2A0007E0613981F87C0001227C3115
:10749000B920FDF734FEFE4890F87A00312804D177
:1074A000FBF798FE08B1FFF738FCF9497A310DF582
:1074B000F17008F030FC30B1F54890F87A003028CF
:1074C00001D1FFF77EFCF3A1F44808F001FC10B1F4
:1074D0004FF0010901E04FF00009F1A1EF4808F079
:1074E000F7FB08B1012000E0002009EA0009B9F12A
:1074F000000F76D000267AE036B9E6A1E74808F01A
:10750000E7FB0446A41D70E0641CAFF2B001204606
:1075100008F0DEFB051E67D0092E63D2DFE806F017
:1075200062050F1A26323D4955001421D84808F04B
:10753000C4FB2A1B2146D64808F0A6FB53E0D448DA
:1075400000214161816181832A1B2146143008F0AA
:107550009BFB48E01421CE481E3008F0AEFB2A1BEE
:107560002146CB481E3008F08FFB3CE0C848002184
:10757000C1630164A0F844102A1B21463C3008F086
:1075800083FB30E0C248323000210160416001815C
:107590002A1B214608F078FB25E01421BC487E30E8
:1075A00008F08BFB2A1B2146B9487E3008F06CFBA3
:1075B00019E01421B648923008F07FFB2A1B2146BF
:1075C000B348923008F060FB0DE01421B048A630BB
:1075D00008F073FB2A1B2146AD48A63008F054FB87
:1075E00001E058E000BF00BF2C46701CC6B2092E57
:1075F00082DBAA22A6491031684608F045FBBA2270
:10760000A3492BA808F040FB2BA80FC8FDF78AFE62
:1076100000230B22A3A1184605F017FF9C495AA886
:1076200008F079FB70BB9A4914315FA808F073FB2E
:1076300040BB97491E310DF5C37008F06CFB08BBC9
:1076400093493C3169A808F066FBD8B990493231BA
:107650000DF5CD7008F05FFBA0B98D497E310DF5B9
:10766000F37008F058FB68B9894992310DF5FD7047
:1076700008F051FB30B98649A6310DF20E2008F012
:107680004AFB40B10120824981F87C0001227C3113
:10769000B920FDF734FD86A1804808F019FB50B3EE
:1076A00085A17E4808F014FB041E1FD08548007891
:1076B000C0F3801030B100230B2283A1184605F0DF
:1076C000C4FE0CE08348007820F04000403081493F
:1076D000087000230B227CA1184605F0B6FE7D48F9
:1076E000007820F0400040307A4908707AA16B4859
:1076F00008F0EEFA04467BA1684808F0E9FA041E97
:107700005FD06421794808F0D8FAE41D0D222146A3
:10771000764808F0B9FA75484079303873490979E4
:10772000303901EB810100EB41000C2801DD012122
:1077300000E000216D48C07930386C4A9279303AC7
:1077400002EB820200EB42001F2801DD012000E075
:10775000002008436549497A3039644A127A303A40
:1077600002EB820201EB4201172901DD012100E059
:10777000002108435D49C97A30395C4A927A303A2F
:1077800002EB820201EB42013B2901DD012100E015
:10779000002108435549497B3039544A127B303A1D
:1077A00002EB820201EB42013B2901DD012100E0F5
:1077B0000021084330B100230D224DA1184605F0E9
:1077C00044FE1CE14948407B30384849097B303948
:1077D00001EB810100EB41014448C07A3038434A53
:1077E000927A303A02EB820200EB4200DFF8FCC0F2
:1077F000CDE900019CF809C0ACF1300CDFF8EC9049
:1078000099F80890A9F1300909EB89090CEB4903B3
:10781000DFF8D8C09CF807C0ACF1300CDFF8CC9092
:1078200099F80690A9F1300909EB89090CEB490296
:10783000DFF8B8C09CF805C0ACF1300CDFF8AC90B4
:1078400099F80490A9F1300909EB89090CEB490179
:10785000DFF898C09CF803C0ACF1300CDFF88C90D6
:1078600099F80290A9F1300909EB89090CEB49005C
:10787000FEF725FE1D48407B30381C49097B303916
:1078800001EB810100EB4100C1B21848C07A37E03A
:10789000C9650020706172772D320000AC7C002039
:1078A00022000000706172772D322C4F4B2C2A0081
:1078B000706172772D330000706172772D332C3137
:1078C0000000000071620020706172772D332C4F30
:1078D0004B2C2A001E630020706172772D332C30F0
:1078E00000000000706172772D3400006B6A002088
:1078F000706172772D342C6661696C2C2A0000004F
:107900003038A94A927A303A02EB820200EB420008
:10791000C0B2DFF894C2CDE900019CF809C0ACF117
:10792000300CDFF8849299F80890A9F1300909EB3E
:1079300089090CEB490C0CF0FF03DFF86CC29CF8D2
:1079400007C0ACF1300CDFF8609299F80690A9F10D
:10795000300909EB89090CEB490C0CF0FF02DFF848
:1079600048C29CF805C0ACF1300CDFF83C9299F8A5
:107970000490A9F1300909EB89090CEB490C0CF0D2
:10798000FF01DFF824C29CF803C0ACF1300CDFF833
:10799000189299F80290A9F1300909EB89090CEBCA
:1079A000490C0CF0FF0008F081F802227E49AA2061
:1079B000FDF7A5FB7D48006800F4807020B1FDF75D
:1079C0004AFE8146FEF795FF7848006800F4007093
:1079D00030B1FDF736FEA0F101094846FEF7CCFEB6
:1079E00000230B2272A1184605F02FFD01207349D8
:1079F00081F87C0001220021B920FDF780FB70A1F5
:107A0000714808F065F9041E1DD0AFF2B051204650
:107A100008F05EF90446641CA51C2978207807F05C
:107A20003EFC287807F069FC074637B900230B2293
:107A300066A1184605F009FD05E000230D2266A1A8
:107A4000184605F002FD68A15F4808F041F9041EE0
:107A50002DD06421544808F030F92BA8FDF7E7FB3E
:107A6000BA222BA9554808F00FF954485B30FDF7AE
:107A7000BEFD814651485030FDF7B9FD82464F4862
:107A80007A30A0F10F015346A0F11902CDE90109A6
:107A9000009157A144480AF0BDFC434808F034F96E
:107AA000814600234A464049184605F0CEFC56A1BF
:107AB000454808F00DF918B364213B4808F0FDF87B
:107AC000A2A9A5A8FEF787FD3C48323000F10A01C3
:107AD000A0F11402A0F11E03CDE90032CDE902109D
:107AE000143B49A24AA130480AF094FC2E4808F001
:107AF0000BF9814600234A462B49184605F0A5FCA0
:107B000048A1314808F0E4F810B300E047E06421F0
:107B1000254808F0D2F8A2A9A5A8FEF75CFD02222C
:107B2000A7A9AA20FDF7C2FAA5A8A2A9A7AB3DA2C2
:107B3000CDE900103DA11C480AF06CFC1A4808F081
:107B4000E3F8814600234A461749184605F07DFCB4
:107B50003AA11D4808F0BCF8041E1ED0642112484A
:107B600008F0ABF807F065FB07467F2F0FD03A46C9
:107B700034A10D480AF04EFC0B4808F0C5F88146C8
:107B800000234A460849184605F05FFC05E000233B
:107B90000E2230A1184605F058FCFFF798FA002095
:107BA0000DF5287DBDE8F0876B6A002008280040AD
:107BB000706172772D342C4F4B2C2A00C965002040
:107BC000706172772D350000AC7C00207061727797
:107BD0002D352C4F4B2C2A00706172772D352C6679
:107BE00061696C2C2A000000706172722D310000F6
:107BF000706172722D312C25732C25642C25732C09
:107C000025732C25642C2A00706172722D320000BD
:107C100025732C25732C25732C25732C25732C256B
:107C2000732C2A00706172722D34000025732C258C
:107C30007325732C25732C2A00000000706172726A
:107C40002D733F00416464726573733A25632C2A77
:107C500000000000416464726573732C6661696C96
:107C60002C2A000010B588B0044601210805F9F758
:107C70006BF901210C20F9F745F98748FBF7AEF8BD
:107C80004FF48050029002208DF80C008DF80D000A
:107C900000208DF80E0001208DF80F0002A97F480A
:107CA000F8F754FE0420029002208DF80C008DF8A5
:107CB0000D0000208DF80E0001208DF80F0002A9A4
:107CC0007748F8F743FE08220C217448F8F7C7FEFE
:107CD000082202217248F8F7C2FE04940020ADF891
:107CE0001400ADF81600ADF81800ADF81C000C201B
:107CF000ADF81A0004A96848FBF7B3F801216648FB
:107D0000FBF734F9012240F225516348FBF7E4F90F
:107D100031208DF8040003208DF8050000208DF837
:107D2000060001208DF8070001A8F8F71CFA402191
:107D30005948FBF703FA08B010BD10B55948B0F820
:107D400064006FF30E005749A1F864000846B0F8CC
:107D5000640020F40040A1F864006421514807F059
:107D6000ACFFC821504807F0A8FF10BD10B540F285
:107D700025514948FBF7EBF9C8B14748FBF725F90E
:107D8000C4B24848B0F86400C0F30E0063280EDAAD
:107D90004449B1F86410C1F30E00411C414AB2F8E5
:107DA000642061F30E023F49A1F864200C5440F2B4
:107DB00024413948FBF7CBF901280DD13948B0F8F7
:107DC000640020F4004000F500403649A1F864004A
:107DD0003148FBF7FAF8C4B210BD0FB438B505A8A6
:107DE00000903148009A04990AF028FB0020009086
:107DF0002D4807F089FF85B200240DE000BF402127
:107E00002548FBF78EF90028F9D02748015D224864
:107E1000FBF7D7F8601C84B2AC42EFDB38BC5DF8EE
:107E200014FB10B5044621461B48FBF7CAF800BFF7
:107E300080211948FBF775F90028F9D010BD70B5FD
:107E400005460E46002404E0285DFFF7EAFF601CAB
:107E500084B2B442F8DB70BD70B50446002504E07E
:107E6000605DFFF7DEFF681CC5B2605D0028F7D1DA
:107E700070BD0FB400B59BB01DA8019002A8019A77
:107E80001C990AF0DBFA0020019002A8FFF7E4FF3A
:107E90001BB05DF814FB00000050004000080240D9
:107EA000000C0240D06C0020366D00201CB5012172
:107EB0000220F9F727F801208DF804008DF806005C
:107EC0008DF8070002208DF805004FF440700090F7
:107ED0006946A248F8F73AFD4FF440719F48F8F719
:107EE000AFFD1CBD10B59E48006820F440209C49A1
:107EF00008600846006840F48020086049159748EB
:107F0000F8F79EFD0120FCF72EF94FF4807193489D
:107F1000F8F796FD0620FCF726F94FF400718F481C
:107F2000F8F790FD0620FCF71EF94FF480718B489E
:107F3000F8F788FD0220FCF716F910BD10B5884847
:107F4000006820F44020864908600846006840F434
:107F50008020086089158148F8F774FD4FF400719E
:107F60007E48F8F76FFD0520FCF7FDF84FF48071AF
:107F70007A48F8F765FD0120FCF7F5F84FF4007139
:107F80007648F8F75DFD0520FCF7EDF810BD10B55B
:107F900000247348006820F44020714908604915A6
:107FA0006E48F8F74DFD0120FCF7DDF84FF48071C5
:107FB0006A48F8F745FD0120FCF7D5F809E00120F3
:107FC000FCF7D1F8641CFA2C03D9FFF7B7FF0120A6
:107FD00010BD4FF400716148F8F71AFD0028EED18A
:107FE0004FF480715D48F8F72DFD0020F0E710B5E3
:107FF0004FF480715948F8F725FD5948006820F47E
:108000004020574908600846006840F48020086016
:1080100049155248F8F716FD0220FCF7A4F84FF472
:1080200080714E48F8F70CFD0220FCF79CF84FF4E5
:1080300080714A48F8F706FD10BD10B54FF4807105
:108040004648F8F7FFFC4648006820F440204449C1
:1080500008600846006840F48020086049153F48E1
:10806000F8F7EEFC0220FCF77EF84FF480713B48F5
:10807000F8F7E6FC0220FCF776F84FF480713748F9
:10808000F8F7E0FC10BD70B504463548006820F4F0
:108090004020334908600846006840F480200860AA
:1080A00089152E48F8F7CEFC002523E0E00928B119
:1080B0004FF400712948F8F7C3FC04E04FF4007155
:1080C0002648F8F7BFFC6006040E0220FCF74BF8C8
:1080D0004FF480712148F8F7B3FC0220FCF743F815
:1080E0004FF480711D48F8F7ADFC0220FCF73BF817
:1080F000681CC5B2082DD9DB70BD70B505460024DB
:108100001748006820F440201549086000261BE04D
:108110004FF480711148F8F795FC0220FCF723F822
:108120004FF480710D48F8F78BFC6006040E4FF495
:1081300000710A48F8F76CFC08B1601CC4B2012059
:10814000FCF711F8701CC6B2082EE1DB15B9FFF779
:1081500074FF01E0FFF74BFF204670BD00040240B2
:108160000008024070B586B004460D461646FDA3D1
:108170002246FEA168460AF04DF90122FDA1FE4803
:1081800002F080FD13222146FC4802F0A6FDFB48C8
:10819000C16803F057F905AB32462946F74802F0AB
:1081A000ADFFF64803F0F1F80022F2A1104602F00C
:1081B00069FD06B070BD70B586B000250020049042
:1081C0000590029003900122EAA1EB4802F05AFDCB
:1081D0000222EB49E94802F080FD0446042C04D059
:1081E000E84890F87C0001287ED1E44803F0CDF8FF
:1081F0001322E349E14802F070FDE048C16803F052
:1082000021F9E14B0D22E1A1DC4802F077FFDD48C6
:10821000613007F079FD0646DB4B3246D9496131C2
:10822000D64802F06BFFD84B0222DCA1D34802F003
:1082300065FFD54B0722DAA1D04802F05FFFD14895
:1082400007F062FD0646D04B3246CE49CB4802F0DD
:1082500055FFCD4B0222D1A1C84802F04FFFCA4BB7
:108260000922D1A1C54802F049FFC648143007F0E1
:108270004BFD0646C44B3246C2491431BF4802F09A
:108280003DFFC14B0222C5A1BC4802F037FFBE4BE7
:108290000A22C8A1B94802F031FFBA481E3007F0DF
:1082A00033FD0646B84B3246B6491E31B34802F09C
:1082B00025FFB54B0222B9A1B04802F01FFFB24B17
:1082C0000922BFA1AD4802F019FFAE483C3007F0CB
:1082D0001BFD0646AC4B3246AA493C31A74802F08A
:1082E0000DFFA94B022200E085E0ACA1A34802F0FB
:1082F00005FFA54B0A22B5A1A04802F0FFFEA14848
:10830000323007F001FD06469F4B32469D4932311F
:108310009A4802F0F3FE9C4B0222A0A1974802F07B
:10832000EDFE994B1122ACA1944802F0E7FE95486E
:10833000503007F0E9FC0646934B324691495031E4
:108340008E4802F0DBFE904B022294A18B4802F093
:10835000D5FE8D4B0D22A5A1884802F0CFFE89489D
:108360005B3007F0D1FC0646874B324685495B31CE
:10837000824802F0C3FE844B022288A17F4802F0AB
:10838000BDFE814B11229DA17C4802F0B7FE7D48C5
:108390006B3007F0B9FC06467B4B324679496B31AE
:1083A000764802F0ABFE784B02227CA1734802F0C3
:1083B000A5FE754B0D2296A1704802F09FFE7148F4
:1083C0007A3007F0A1FC06466F4B32466D497A3190
:1083D0006A4802F093FE6C4B022270A1674802F0DB
:1083E0008DFE694B4FF4D0728D49644802F086FED1
:1083F000624802F0CAFF13226149604802F06DFC36
:1084000004463CB3002514E0681CC5B25B4802F08A
:10841000BCFF002257A1104602F034FC012255A1F6
:10842000554802F02FFC13225549544802F055FCE0
:1084300004460CB1012000E00020642D01DA012186
:1084400000E0002108400028DED1622D02DD052079
:1084500006B070BD4948C16802F0F4FF714807F0EA
:1084600053FC0646484B32466E49444802F046FEED
:10847000454B022249A1414802F040FE3F4802F02C
:1084800084FF01223BA13C4802F0FCFB022266A1D2
:108490003A4802F022FC04463A4890F87C00012851
:1084A00001D0042C5CD10020364981F87C000122E7
:1084B0000021B920FCF723FE01220DF10601BA20AC
:1084C000FCF71DFE2D4802F060FF132256A12B4839
:1084D00002F003FC2948C16802F0B4FF2A4B0D22C8
:1084E0002AA1264802F00AFE2648613007F00CFC5B
:1084F0000646254B324623496131204802F0FEFDF5
:10850000214B022225A11D4802F0F8FD1E4B072237
:1085100023A11A4802F0F2FD1A4807F0F5FB0646BF
:10852000194B32461749154802F0E8FD164B022256
:108530001AA1124802F0E2FD134B09221AA10F48BA
:1085400002F0DCFD0F48143007F0DEFB06460E4B50
:1085500032460C491431094802F0D0FD0A4B69E05B
:108560002CE100002E747874000000002573257340
:1085700000000000303A0000407500201073002019
:10858000C4780020C96500202C63002045717569FE
:10859000706D656E745F49443A0000000D0A00007A
:1085A0005443505F49703A005443505F506F7274A7
:1085B0003A000000576966695F535349443A000026
:1085C000576966695F5077643A00000057696669C9
:1085D0005F506F72743A00004D6561737572655F2C
:1085E000496E74657276616C3A0000005075625F86
:1085F000496E74657276616C3A0000004170706F6C
:10860000696E746D656E745F54696D653A00000043
:108610004D6561737572655F4D6F64653A0000006A
:1086200064490208406F0020424332352E7478744A
:10863000000000000222AFF29C01FE4802F05EFD45
:10864000FD4B0A22AFF29401FA4802F057FDFB48B5
:1086500007F05AFB0646F84B3246F849F54802F057
:108660004DFDF54B0222AFF2CC01F24802F046FD7F
:10867000F14B0922AFF2B801EE4802F03FFDEF489E
:108680001E3007F041FB0646EB4B3246EB491E31EC
:10869000E84802F033FDE84B0222AFF20011E54852
:1086A00002F02CFDE44B0A22AFF2E001E14802F0B7
:1086B00025FDE248143007F027FB0646DE4B324624
:1086C000DE491431DB4802F019FDDB4B0222AFF228
:1086D0003411D84802F012FDD74B1122AFF2081125
:1086E000D44802F00BFDD548323007F00DFB0646AA
:1086F000D14B3246D1493231CE4802F0FFFCCE4B4D
:108700000222AFF26811CB4802F0F8FCCA4B0D22EE
:10871000AFF22811C74802F0F1FCC8483D3007F01D
:10872000F3FA0646C44B3246C4493D31C14802F013
:10873000E5FCC14B0222AFF29C11BE4802F0DEFC08
:10874000BD4B1122AFF24C11BA4802F0D7FCBB4826
:108750004D3007F0D9FA0646B74B3246B7494D318E
:10876000B44802F0CBFCB44B0222AFF2D011B148B6
:1087700002F0C4FCB04B0D22AFF26C11AD4802F018
:10878000BDFCAE485C3007F0BFFA0646AA4B324645
:10879000AA495C31A74802F0B1FCA74B0222AFF214
:1087A0000421A44802F0AAFCA34B4FF4D072A449C0
:1087B000A04802F0A3FC9F4802F0E7FD1322AFF2AD
:1087C00098119C4802F089FA04464CB3002517E042
:1087D000681CC5B2974802F0D8FD0022AFF26C21A8
:1087E000104602F04FFA0122AFF27821954802F0CC
:1087F00049FA1322AFF2D0118E4802F06EFA044605
:108800000CB1012000E00020642D01DA012100E01C
:10881000002108400028DBD1622D01DD052017E68C
:108820008448C16802F00EFE874807F06DFA0646DC
:10883000814B324684497F4802F060FC7E4B022225
:10884000AFF2A8217B4802F059FC7A4802F09DFD66
:108850000022AFF2E021104602F014FA0020F7E502
:1088600010B50122AFF2F421764802F00BFA132280
:1088700076A1704802F031FA6E48C16802F0E2FD5C
:108880006D4B4FF4E47274496A4802F037FC6E484D
:1088900007F03AFA0446684B22466B49654802F0F5
:1088A0002DFC654B0222AFF20C31624802F026FC2F
:1088B000604802F06AFD0122AFF24831002002F068
:1088C000E1F910BD3EB504460020009001900290F1
:1088D0005FA32246AFF26C31684609F09BFD01228E
:1088E000AFF27031574802F0CDF9684603F0A1F8B5
:1088F0000546504802F049FD0022AFF2883110468B
:1089000002F0C0F928463EBD70B586B0044650A3BB
:108910002246AFF2A83101A809F07CFD0122AFF296
:10892000AC31484802F0AEF9064601224BA141485D
:1089300002F0D3F9064616B1042006B070BD3D48DA
:10894000C56802F022FD06460022AFF2D83110467B
:1089500002F098F92846F0E70146002000BF0246E1
:10896000431C98B28A5C0A2A06D0421E8A5C0D2AF1
:1089700002D0B0F59D7FF2DD70472DE9F04F87B052
:1089800083460F4614460020069000250590364881
:10899000007910B907B0BDE8F08F40F23B113348C1
:1089A00007F08BF940F23B11314807F086F940F2AD
:1089B0003B11304807F081F9012206A9B420FCF7E9
:1089C00091FB0698A04201D90020069020A35A46A8
:1089D000AFF2684101A809F01DFD0698201A4FF476
:1089E0009671B0FBF1FA0698201AB0FBF1F201FB88
:1089F0001200049040F23B111C4807F05EF91E483B
:108A0000006808F075F800F0400018B140F6B83082
:108A100008F04AF80122AFF2A4410A4802F032F904
:108A20008046012201A9034802F057F9804600263A
:108A300035E00000107300202C630020E765002063
:108A40006449020840750020406F0020746573740B
:108A50002E7478740000000098470208303A2F42C4
:108A60004332352E747874003D630020D87800209E
:108A7000137A00204E7B0020C0620020FE4802F0E6
:108A800084FC80460122AFF21451FC4802F0FAF84F
:108A90008046012201A9F84802F01FF98046B8F18A
:108AA000000F01D0012000E00020642E01DA012136
:108AB00000E0002108400028E0D106983918EE486F
:108AC00002F0C0FC4FF00009D7E0ED48006808F064
:108AD0000FF800F04000002870D04021E8480068FE
:108AE00007F0F4FFE44802F050FC80468021E4489F
:108AF000006808F027F841F2883301221102E048AB
:108B0000006808F045F8DC4802F03FFC8046DDA034
:108B1000FFF7FAFE044605E0DAA0FFF7F5FE04468B
:108B2000701CC6B20A2C01D2012000E00020322EB7
:108B300001DA012100E0002108400028ECD106986C
:108B4000201A4FF49671B0FBF1FACA440698201A25
:108B5000B0FBF1F201FB120004900122AFF2EC51E4
:108B6000C64802F08FF8012201A9C34802F0B5F807
:108B70008046002607E0012201A9BF4802F0ADF8B7
:108B80008046701CC6B2B8F1000F01D0012000E091
:108B90000020642E01DA012100E0002108400028B5
:108BA000E9D1B8F1000F05D0012206A9B420FCF7E5
:108BB0000CFBEFE6B048069902F044FCB34B4FF4CF
:108BC0009672B349AC4802F0C3F98046B048FFF74B
:108BD000C3FE0546681C80B2059040F23B11AD48CB
:108BE00007F06BF840F23B11AB4807F066F86A1CDF
:108BF000A749A94807F048F8A8A1A74807F068F8CE
:108C000018B10220A84908700EE0A34800782F2868
:108C100007DDA14800783A2803DA0320A24908704A
:108C200002E00120A04908709B4B6A1C9FA1994853
:108C300009F0F0FB9748FFF78FFE054600269A489B
:108C40000078012805D09349A81C04F063F800B10E
:108C5000A0E6DDE905010844069006983918864823
:108C600002F0F0FB012206A9B420FCF7AEFA069848
:108C7000201A4FF49671B0FBF1FAD145FFF425AFFD
:108C800040E0824B4FF4967281497B4802F060F9D4
:108C900080467F48FFF760FE0546681C80B205905D
:108CA00040F23B117B4807F008F840F23B117A484C
:108CB00007F003F86A1C7649774806F0E5FF764B23
:108CC0006A1C7AA1734809F0A5FB7248FFF744FEBD
:108CD000054675480078012805D06E49A81C04F0A7
:108CE00019F800B156E6DDE905010844069006983A
:108CF0003918614802F0A6FB012206A9B420FCF74E
:108D000064FA00BF0698A042BBD30020069001225F
:108D100006A9B420FCF759FA574802F036FB804602
:108D20000122AFF2B071554801F0ACFF55A0FFF73A
:108D3000C9FD00BF2EE610B58AB05F4840795E4994
:108D400009795D4AD2785C4B9B78CDE90632CDE952
:108D50000810594841780078584A5278574B1B7888
:108D6000CDE90232CDE904015448407953490979EB
:108D7000CDE900105148C378827851A1584809F0D4
:108D800049FB4FF4FA71574806F097FF5649A1F195
:108D90001E00A0F11E02A0F13C03CDE90532CDE991
:108DA00007015A3896395A3B4D4A2832CDE90123FA
:108DB000CDE90310A2F10A00494B4C4A4CA10090A6
:108DC000484809F027FB474806F09EFF841C2246CE
:108DD0004FA1504809F01EFB42480078302803DBC1
:108DE00040480078392809DD4FF4FA713D4806F013
:108DF00064FF49A24BA13B4809F00CFB0AB010BD2F
:108E00002DE9FC4781460C4615464FF42F700AF0B9
:108E10000BFD01900020009000278046012243A115
:108E2000019801F02FFF064601AA69463FA002F013
:108E300029FD0646B6B90198C069801E0199498985
:108E400000FB01F801984089009900FB01F74FEA07
:108E500058002060780828602068800A2060286810
:108E6000800A2860012231A1002001F00BFF064694
:108E700001980AF0B1FC5BE01073002040750020FF
:108E8000C062002042433235000000002C63002005
:108E9000D8780020137A00204E7B00204368312DC3
:108EA000536F696C545F43003C6300205075622C23
:108EB00025642C25732A00003364002024640020DC
:108EC000256325632F256325632F323025632563B2
:108ED00020256325633A256325633A2563256300CE
:108EE00034710020406F0020017F00202A6600209E
:108EF00025732C25732C2573257325732C25732C32
:108F000025732C25732C25732C25732C25730000B9
:108F100025642C00EC72002054455354544553549E
:108F20000000000025730D0A000000003000000062
:108F30003046BDE8FC8710B5044620460AF074FCB4
:108F400010BD10B5044620460AF046FC10BD0000D6
:108F500010B502460020404B802A01D290B213E0A7
:108F6000B2F5803F10D240F2B514A1420CD10020DE
:108F700001E0441CA0B2802803DA33F81040944288
:108F8000F7D100F18004E0B210BD10B50246002018
:108F9000314B802A01DA104609E040F2B514A142B3
:108FA00005D1FF2A03DCA2F1800433F8140010BDC0
:108FB00070B5B0F5803F4DD281B2B1F5805F01DA76
:108FC000264E00E0264E324600BF32F8023B0BB17F
:108FD000994200DA3CE032F8024B2512E4B21E1945
:108FE0008E4230DD092D2CD2DFE805F005090F1384
:108FF000171B1F232700CE1A32F8161021E0CE1AB5
:1090000006F001068E1BB1B21BE0A1F11006B1B251
:1090100017E0A1F12006B1B213E0A1F13006B1B220
:109020000FE0A1F11A06B1B20BE001F10806B1B2EE
:1090300007E0A1F15006B1B203E0A1F5E356B1B2E9
:1090400000BF00BF04E0002DBFD102EB4402BCE72B
:1090500000BF084670BD0000983B0208983C02081B
:109060008A3E020870B5044600255CB9FBF709FE8C
:10907000054635B1FBF7D4FCFF20FBF7CBFCFBF733
:10908000D4FC00BF00BF0DB1012070BD0020FCE783
:1090900070B50446002514B1012C0DD10BE0FBF78F
:1090A000F0FD054635B1FBF7BBFCFF20FBF7B2FC3A
:1090B000FBF7BBFC02E001E0012500BF00BF0DB1E2
:1090C000012070BD0020FCE72DE9F04105460E4669
:1090D00017461C464FF0000814B90420BDE8F08183
:1090E00015B1012D14D110E0E2B239463046FBF73C
:1090F00089FE8046B8F1000F06D0FBF791FCFF20F7
:10910000FBF788FCFBF791FC05E04FF0000802E05C
:109110004FF0010800BF00BFB8F1000F01D10020DF
:10912000DCE70120DAE72DE9F04105460E46174657
:109130001C464FF0000814B90420BDE8F08115B1B9
:10914000012D08D106E0E2B239463046FBF797FE22
:10915000804603E002E04FF0010800BF00BFB8F115
:10916000000F01D10020E8E70120E6E72DE9F041FA
:1091700006460F4615463EBB37B1012F1CD0022FC5
:1091800011D0032F1DD113E040212D48F7F75AFCD1
:10919000FBF75FFC08B9002400E0012440212848C7
:1091A000F7F74EFC0FE04FF40070288000240AE02F
:1091B00008202880002406E0FBF728FD2860002412
:1091C00001E0042400BF15E0012E12D137B1012FB8
:1091D0000AD0022F04D0032F08D103E0002407E0B7
:1091E000002405E0002403E0002401E0042400BF83
:1091F00000E001242046BDE8F0811CB501A9002053
:10920000F8F720F969460020F8F7B6F99DF8030051
:10921000143040069DF8011040EA41509DF80210BC
:1092200040EA01409DF8041040EAC1209DF8051075
:1092300040EA41109DF8061040EA61001CBD0000A4
:1092400000080240014648780A7842EA0020704748
:109250000146C8788A7842EA00204A7842EA00202B
:109260000A7842EA0020704700F8011B091200F852
:10927000011B704700F8011B090A00F8011B090ACD
:1092800000F8011B090A00F8011B7047014609B1EB
:10929000002070470020FCE7014609B1002070471C
:1092A0000020FCE72DE9F0410646356815F8014B32
:1092B0002046FFF7EBFF60B115F8017B3846FFF75A
:1092C000EBFF18B94FF0FF30BDE8F08107EB042049
:1092D00084B24CB140F2B5112046FFF756FE044669
:1092E00014B94FF0FF30EFE7A04635604046EBE79A
:1092F0002DE9F04107460C46164640F2B5113846B6
:10930000FFF726FE0546FF2D0BDD022E02D20020C0
:10931000BDE8F081281204F8010B04F8015B02207B
:10932000F6E705B10EB90020F2E704F8015B012071
:10933000EEE730B502460B46002400211CE0FA4857
:1093400000EB01100068A8B1F74800EB01100068BD
:109350001568A8420FD1F44800EB011040689568E9
:10936000A84208D1F04800EB011080685569A84276
:1093700001D103E00124491C0229E0D300BF0229E6
:1093800006D11CB9022B01D0122030BD0020FCE711
:1093900033B9E54800EB01108089B0F5807F01D139
:1093A0001020F2E70020F0E7002100E0491C02292C
:1093B00005D2DD4800EB011000680028F6D1022933
:1093C00001D0012070470020FCE710B502460B4693
:1093D000002116E0D44800EB011000681468A04298
:1093E0000ED1D14800EB011040689468A04207D12B
:1093F000CD4800EB011080685469A04200D102E022
:10940000491C0229E6D300BF022922D1002100E035
:10941000491C022905D2C44800EB0110006800284D
:10942000F6D1022901D1002010BDBF4C04EB01147C
:1094300010682060BC4C04EB011490686060BA4C6A
:1094400004EB01145069A0600020B74C04EB011438
:10945000A081012B06DBB44800EB0110808908B124
:109460000020E1E713B14FF4807004E0AE4800EB58
:1094700001108089401CAC4C04EB0114A081481CF5
:10948000D2E710B50246531E1A46022B17D2A64B3E
:1094900003EB02139989B1F5807F00D100210029E7
:1094A00001DD4B1E99B2A04B03EB0213998121B948
:1094B00000239D4C04EB02142360002000E00220F6
:1094C00010BD014600200BE0974A02EB0012126823
:1094D0008A4204D10022944B03EB00131A60401C13
:1094E0000228F1D3704770B504460025E078E8B152
:1094F0006078012304F13801626BFFF714FEA0B914
:109500000020E070A16A606B401A216A88420DD287
:10951000A07802280AD1236A616BCA1860780123F7
:1095200004F13801FFF7FFFD00E00125284670BD7A
:1095300070B504460D460026606BA84210D0204648
:10954000FFF7D1FF06465EB9607801232A4604F191
:109550003801FFF7B9FD10B14FF0FF350126656303
:10956000304670BD70B504462046FFF7BCFF054687
:10957000002D37D1207803282DD1207901282AD138
:10958000410204F1380006F098FB4AF6552104F236
:109590003620FFF769FE654904F13800FFF76AFEDF
:1095A000634904F50770FFF765FE04F5087061690B
:1095B000FFF760FE04F509702169FFF75BFE606A42
:1095C000401C60636078012304F13801626BFFF78F
:1095D000AAFD00202071607800221146FFF7C6FD29
:1095E00000B10125284670BD0246891ED069801E43
:1095F000884201D8002070475389106B03FB01009B
:10960000F9E72DE9F04781460C46D9F80050022CC5
:1096100002D3E869A04202D84FF001085EE04FF0A3
:10962000FF382878012804D002282CD0032851D1F3
:109630003CE0264606EB5606A86A00EB5621284673
:10964000FFF776FF00B148E03046761CC0F3080112
:1096500005F13800475CA86A00EB56212846FFF761
:1096600067FF00B139E0C6F3080105F13800405C3E
:1096700047EA002704F0010008B1380901E0C7F308
:109680000B00804629E0A86A00EB14212846FFF76A
:109690004FFF00B121E040F2FF1101EA440205F161
:1096A00038015018FFF7CEFD804616E0A86A00EB9F
:1096B000D4112846FFF73CFF00B10EE040F2FF1145
:1096C00001EA840205F138015018FFF7C1FD20F0CE
:1096D000704802E04FF0010800BF00BF4046BDE8FF
:1096E000F0872DE9F04704460D4616464FF0020973
:1096F000022D70D3E069A8426DD92078012804D0EA
:10970000022850D003280DD166E02F4607EB5707FB
:10971000A06A00EB57212046FFF70AFF8146B9F106
:10972000000F07D07CE000008C7C00205252614189
:109730007272416138467F1CC0F3080104F13800A1
:1097400001EB000805F0010028B1F1B298F8000023
:1097500061F31F1000E0304688F800000120E0703F
:10976000A06A00EB57212046FFF7E2FE8146B9F1DF
:10977000000F00D054E0C7F3080104F1380001EBFA
:10978000000805F0010010B1C6F3071006E098F8D4
:10979000000000F0F000C6F30321084388F8000041
:1097A0000120E0703CE0A06A00EB15212046FFF7A5
:1097B000BFFE8146B9F1000F00D031E0B1B240F2F6
:1097C000FF1202EA450304F138029818FFF74CFD36
:1097D0000120E07024E024E0A06A00EBD5112046CF
:1097E000FFF7A6FE8146B9F1000F00D018E040F265
:1097F000FF1101EA850204F138015018FFF728FD36
:1098000066F31B00064640F2FF1101EA850204F1EF
:10981000380150183146FFF72DFD0120E07000BFE0
:1098200000BF4846BDE8F0872DE9F04781460E4667
:1098300017464FF00008D9F80040022E02D3E06925
:10984000B04202D80220BDE8F08767B100BF4FF0F8
:10985000FF3239462046FFF744FF8046B8F1000F3B
:1098600001D04046EFE700BF31464846FFF7C9FE4A
:10987000054605B922E0012D01D10220E3E7681C6D
:1098800008B90120DFE7002231462046FFF729FF13
:109890008046B8F1000F01D04046D4E7E069801E51
:1098A0006169814206D26069401C6061207940F0A4
:1098B000010020712E46E069B042D5D800BF0020DB
:1098C000C1E72DE9F04782468846DAF80040B8F152
:1098D000000F06D1276917B1E069B84215D80127F2
:1098E00013E041465046FFF78CFE0546022D02D29A
:1098F0000120BDE8F087681C08B92846F9E7E0694F
:10990000A84201D92846F4E74746606908B9002013
:10991000EFE70026474518D17E1CE069B04200D829
:10992000022631465046FFF76CFE0546012D01D058
:10993000681C08B92846DCE73DB12569022D03D330
:10994000E069A84200D92F460026E6B93E4600BF8E
:10995000761CE069B04204D80226BE4201D900203C
:10996000C7E731465046FFF74CFE054605B909E00A
:10997000012D01D0681C08B92846BAE7BE42E7D1DC
:109980000020B6E700BF4FF0FF3231462046FFF718
:10999000A8FE8146B9F1000F08D1B8F1000F05D03B
:1099A000324641462046FFF79CFE8146B9F1000F42
:1099B0000DD12661E069801E6169814202D860692B
:1099C000401E6061207940F00100207107E0B9F18C
:1099D000010F02D14FF0FF3000E001200646304673
:1099E00087E7F0B503460D461E68D86A021D680A6F
:1099F0007789B0FBF7F400BF02CA09B90020F0BDB7
:109A00008C4200D202E0641A121DF5E700BF106814
:109A10002044F4E72DE9F047044689462046FFF745
:109A200062FD10B10120BDE8F08749462046FFF7EE
:109A3000DBFD074667634FF4007104F1380006F060
:109A40003CF960894FF40041B1EB402F01D8084642
:109A500001E06089400206464FF0000800E0760809
:109A6000B6F5007F05D93046FFF765FAB0F100087A
:109A7000F5D0B6F5007F16D93146404606F01DF9FF
:109A8000760A002500E035446089A84207D97A1992
:109A9000607833464146FFF746FB0028F3D0404646
:109AA000FFF74FFA10E004F138080126002500E026
:109AB00035446089A84207D97A196078334641460F
:109AC000FFF731FB0028F3D06089A84201D00120C4
:109AD000A9E70020A7E72DE9F04104460D462668D6
:109AE000B5F5001F02D205F01F0010B10220BDE83D
:109AF000F0816561A7681FB93078032800DBF76A39
:109B000047B93089B0EB551F01D80220EFE7F06A62
:109B1000E0611CE070894FEA402811E03946204698
:109B2000FFF76FFD0746781C08B90120DFE7022F19
:109B300002D3F069B84201D80220D8E7A5EB0805A6
:109B40004545EBD239463046FFF74EFDE061A7614F
:109B5000E06908B90220CAE7E06900EB5520E0613E
:109B6000C5F3080106F13800084420620020BEE772
:109B70002DE9F041044688462768606900F1200617
:109B8000B6F5001F01D30020E061E06910B90420A0
:109B9000BDE8F081C6F30800002845D1E069401C0B
:109BA000E061A06938B93889B0EB561F3CD8002075
:109BB000E0610420ECE77889401E00EA562098BB5B
:109BC0002046A169FFF71DFD0546012D01D80220A1
:109BD000DEE7681C08B90120DAE7F869A8421DD859
:109BE000B8F1000F03D10020E0610420D0E7204647
:109BF000A169FFF766FE05460DB90720C8E7012DEC
:109C000001D10220C4E7681C08B90120C0E7294639
:109C10003846FFF7FFFE08B10120B9E7A5612946E4
:109C20003846FFF7E1FCE0616661C6F3080107F121
:109C30003800084420620020AAE72DE9F0410446DC
:109C40000E46D4F8008000212046FFF744FF054669
:109C5000EDB9002700BF4046E169FFF769FC054602
:109C600005B113E0206A0078E52802D0206A007868
:109C700020B9781C0746B04201D107E00027012136
:109C80002046FFF775FF0546002DE4D000BF042DE8
:109C900000D107252846BDE8F08170B505460C4681
:109CA00004F11A00FFF7CEFA06462878032805D1FA
:109CB00004F11400FFF7C6FA46EA0046304670BDCC
:109CC00070B506460C461546A9B204F11A00FFF716
:109CD000CBFA3078032804D1290C04F11400FFF7E3
:109CE000C3FA70BD2DE9F04780460C4604F11A0016
:109CF000FFF7A8FA10B10020BDE8F087207800F047
:109D00003F00401E00EB800101EBC0054FF0010950
:109D1000002621E0FA49895D0819FFF793FA074602
:109D2000B9F1000F11D0FF2D0BD83846FFF740F9DD
:109D3000824629466D1C38F81100FFF739F9824533
:109D400001D00020D8E7B94605E04FF6FF70874202
:109D500001D00020D0E7761C0D2EDBD3207800F058
:109D6000400038B1B9F1000F04D038F8150008B13F
:109D70000020C1E70120BFE72DE9F04780460C46EF
:109D800004F11A00FFF75EFA10B10020BDE8F08779
:109D9000207820F04000401E00EB800101EBC00560
:109DA0004FF00109002619E0D549895D0819FFF730
:109DB00049FA0746B9F1000F09D0FF2D01D900205B
:109DC000E4E7B94628466D1C28F8107005E04FF608
:109DD000FF70874201D00020D8E7761C0D2EE3D318
:109DE000207800F0400048B1B9F1000F06D0FF2DF7
:109DF00001D90020CAE7002028F815000120C5E796
:109E00002DE9F04707460C461546984684F80D8024
:109E10000F20E07200202073002104F11A00FFF7E8
:109E200023FA681E00EB800101EBC0090020064602
:109E3000824600BF4FF6FF70864204D0484609F1C3
:109E4000010937F81060AE4911F80A1008193146B7
:109E5000FFF70AFA0EB94FF6FF760AF101008246C3
:109E60000D28E7D34FF6FF70864202D037F819006D
:109E700008B945F040052570BDE8F0872DE9FF4F92
:109E800083B0074691461E460498016839604168D0
:109E9000796001893981807AB872052E19D9B04666
:109EA00012E039F802BB00240CE0584668F35F006A
:109EB00080464FEA6B0B08F4803010B1914888EA75
:109EC0000008641C102CF0D3B9F800000028E8D179
:109ED0004646072400BF06F00F0000F1300A36099D
:109EE000BAF1390F03DD0AF1070000F0FF0A20463E
:109EF000641E01A901F800A00CB1002EEBD17E2058
:109F000001A90855002509E0785DFFF7BFF920B1E8
:109F1000601EA84200D106E06D1C6D1CA54202D255
:109F2000785D2028F0D100BF00BF082C04D2204665
:109F3000641C01A9085C00E0202029466D1C7854AF
:109F4000082DF2D307B0BDE8F08F30B501460020F0
:109F50000B2200BF431003EBC01411F8015B63191F
:109F6000D8B2531E1A1EF5D130BD2DE9F05F04465C
:109F700089460426D4F800A04FF0FF08C34653E0FA
:109F80005046E169FFF7D4FA064606B14FE0206A71
:109F900005780DB904264AE0206AC07A00F03F0730
:109FA000A771E52D0AD02E2D08D027F02000082813
:109FB00001D1012000E00020484502D04FF0FF0809
:109FC0002BE00F2F1DD105F0400038B1206A90F82A
:109FD0000DB005F0BF05A8466069206345450CD16A
:109FE000206A407B584508D1216ADAF80C00FFF757
:109FF000C3FE10B1A8F1010000E0FF2000F0FF084F
:10A000000BE0B8F1000F04D1206AFFF79EFF58451E
:10A0100002D04FF0FF30206309E000212046FFF717
:10A02000A7FD064606B102E0E0690028A8D100BFFE
:10A030000EB10020E0613046BDE8F09F2DE9F04709
:10A040000446D4F800A000212046FFF744FD064650
:10A0500016B13046BDE8F0874FF0FF08C1464FF01B
:10A06000FF30206300BF5046E169FFF761FA064602
:10A0700006B162E0206A05780DB904265DE0206A29
:10A08000C07A00F03F07A771E52D04D007F0080063
:10A0900038B10F2F05D04FF0FF084FF0FF3020638D
:10A0A00044E00F2F22D12F20005D00F0400030BB94
:10A0B00005F0400038B1206A90F80D9005F0BF051A
:10A0C000A8466069206345450CD1206A407B48451D
:10A0D00008D1216ADAF80C00FFF704FE10B1A8F1EC
:10A0E000010000E0FF2000F0FF081FE0B8F1000FC2
:10A0F0000AD1206AFFF729FF484505D11DE015E088
:10A10000483F0208211001002F20005D00F00100EF
:10A1100038B90B2204F12401206A05F00AFE00B9C7
:10A120000BE04FF0FF084FF0FF3020630021204686
:10A13000FFF71EFD0646002E95D000BF304689E78A
:10A140002DE9FE4F044626682F20005D00F0A00098
:10A1500010B10620BDE8FE8F4FF0000901E009F1C3
:10A160000109F06830F819000028F8D1D4E90A1282
:10A17000606A8DE807009DF80B0000F0010028B32D
:10A1800040212F2001554FF001080EE0434669465B
:10A1900004F12400F268FFF771FE2046FFF74EFF3E
:10A1A000054605B104E008F10108B8F1640FEDD3EC
:10A1B00000BFB8F1640F01D10720CBE7042D01D017
:10A1C0002846C7E79DF80B102F2001559DF80B007E
:10A1D00000F0020030B109F10C000D21B0FBF1F0EC
:10A1E000401C00E00120074639462046FFF725FDC8
:10A1F00005464DBB781E071E26D06069A0EB4711AF
:10A200002046FFF768FC0546F5B904F12400FFF786
:10A210009CFE824600BF3046E169FFF789F905469A
:10A2200005B110E0FAB2216A5346F068FFF7E8FD85
:10A230000120F07000212046FFF79AFC054615B971
:10A24000781E071EE7D100BFDDB93046E169FFF790
:10A250006FF90546ADB92021206A05F02EFD206A70
:10A26000616A0160A16A4160A18D018194F82E109C
:10A2700081722F20005D00F01800216A0873012010
:10A28000F070284666E72DE9F041044626686769C4
:10A29000206B401C08B9002003E02046216BFFF72B
:10A2A0001AFC0546E5B900BF3046E169FFF740F901
:10A2B000054605B110E000BFE520216A08700120C5
:10A2C000F0706069B84200D306E000212046FFF735
:10A2D0004FFC0546002DE7D000BF042D00D102251C
:10A2E0002846BDE8F0812DE9F84F07460C4638684E
:10A2F00000900020A075F86908B9BDE8F88F386BA8
:10A30000401C002837D00025A846A94624E0009824
:10A31000C268404608F1010832F81060B9F1000F38
:10A3200007D1B6F5584F04DBB6F5604F01DAB146F8
:10A3300012E0C5F1FF0204F11603591946EA09407B
:10A34000FEF7D6FF8246BAF1000F01D1002509E0E1
:10A3500055444FF0000900BF0098C06830F818005D
:10A360000028D4D100BFB9F1000F00D00025002192
:10A3700004F1160041550020054680461BE040468A
:10A3800008F101083A6A165C202E00D113E0052E70
:10A3900000D1E526B8F1090F07D10C2D05D22E22E8
:10A3A00028466D1C04F109010A5428466D1C04F16D
:10A3B00009010E5400BFB8F10B0FE0D3002104F1E6
:10A3C00009004155A07DB0BB35B93F2228466D1C20
:10A3D00004F116010A5425E00020054680464FF09E
:10A3E000080B19E004F1090010F808602E2E01D1C5
:10A3F0004FF0100B412E09DB5A2E07DC386A007B28
:10A4000000EA0B0010B106F1200086B204F116003C
:10A41000465508F101086D1C04F1090010F8080008
:10A420000028DFD1002104F116004155386A007B75
:10A4300008B900206072386AC07A00F03F002072CC
:10A44000396A01F11C00FEF703FF2060396A01F14F
:10A450001600FEF7F7FEE080396A01F11800FEF7FA
:10A46000F1FEA08000BF48E72DE9F34F83B081469D
:10A47000049800680090D9F80000C768002500BF64
:10A480006846FEF70FFF02900298401C18B906209C
:10A4900005B0BDE8F08F0298B0F5803F05D3029873
:10A4A000020C28466D1C27F81020029884B2202C3C
:10A4B00003DB2F2C01D05C2C00D111E0802C06DABC
:10A4C0002146FEA005F016FC08B10620E0E7FF2DAE
:10A4D00001D30620DCE728466D1C27F81040CFE7A3
:10A4E00000BF202C01DA042611E002E00098401C95
:10A4F0000090009800782F28F8D0009800785C2809
:10A50000F4D0002600980078202800D20426009974
:10A5100004980160012D04D1681E37F810002E2820
:10A520000BD0022D24D1681E37F810002E281FD121
:10A53000A81E37F810002E281AD1002027F8150081
:10A5400080460AE0A84501D22E2100E0202109F131
:10A55000240000F8081008F10108B8F10B0FF1D33E
:10A5600046F0200109F1240000F8081000208FE7D0
:10A5700008E0681E37F81040202C02D02E2C00D0A6
:10A5800002E06D1E002DF4D100BF002027F8150059
:10A590000DB906207CE74FF0000A01E00AF1010A3C
:10A5A00037F81A002028F9D0BAF1000F03D137F894
:10A5B0001A002E2801D146F0030600E06D1E25B1D9
:10A5C000681E37F810002E28F8D120220B2109F13F
:10A5D000240005F06BFB4FF00008C34608200190F3
:10A5E00000BF50460AF1010A37F8104004B968E08C
:10A5F000202C03D02E2C04D1AA4502D046F003060D
:10A60000EFE70198804501D2AA4516D101980B28A1
:10A6100002D146F0030654E0AA4501D046F00306F5
:10A62000AA4500D94DE0AA464FF008080B2001903A
:10A630004FEA8B604FEA106BD3E7802C0EDB46F0BD
:10A64000020640F2B5112046FEF782FC044604F0F3
:10A65000800018B104F07F009B490C5CFF2C10DDDA
:10A660000198401E404504D846F00306DDF80480FA
:10A67000B7E72212404608F1010809F124010A5403
:10A6800018E024B1214691A005F034FB18B15F24F5
:10A6900046F003060EE0412C03DB5A2C01DC4BF0A4
:10A6A000020B612C06DB7A2C04DC4BF0010BA4F1CD
:10A6B000200084B2404608F1010809F124010C543D
:10A6C0008FE700BF99F82400E52802D1052089F81A
:10A6D00024000198082803D14FEA8B604FEA106BE1
:10A6E0000BF00C000C2803D00BF00300032801D161
:10A6F00046F0020606F0020048B90BF0010008B16E
:10A7000046F010060BF0040008B146F008062F20B2
:10A7100000F809600020BBE62DE9F34104462768F4
:10A72000019800782F2807D0019800785C2803D082
:10A7300000BFB869A0600DE002E00198401C0190E4
:10A74000019800782F28F8D0019800785C28F4D080
:10A750000020A06001980078202808D280212F20B6
:10A76000015500212046FFF7B6F9054637E000BF46
:10A7700001A92046FFF778FE054605B12EE02046E8
:10A78000FFF75CFC05462F20065D95B1042D0FD127
:10A7900006F0200040B106F0040000B9E8E780218F
:10A7A0002F200155002503E006F0040000B905251F
:10A7B00014E006F0040000B110E0A07900F01000F1
:10A7C00008B905250AE0A08AC0F3080207F138009D
:10A7D00011183846FFF761FAA060C9E700BF2846A4
:10A7E000BDE8FC8170B504464FF0FF302668314665
:10A7F000324601B970BD00BF12F8013B202B01D3D6
:10A800003A2BF9D13A2B11D101250E78302E08DBE5
:10A810000E78392E05DC8E1C964202D10E78A6F1F8
:10A820003005012D01DA28462260E3E7294E307811
:10A8300000BFDFE72DE9F041044688460020E070C4
:10A84000401E606341462046FEF772FE10B10420B0
:10A85000BDE8F08104F23620FEF7F4FC074694F8D8
:10A860003850EB2D03D0E92D01D0E82D5AD14AF60E
:10A870005520874208D1082217A104F18A0005F06B
:10A8800058FA08B90020E3E704F14300FEF7DAFCC8
:10A8900006464520055D701E3040E8BBB6F5007FDA
:10A8A00040DBB6F5007F3DDCB5B3681E284098BBA1
:10A8B00004F14600FEF7C6FC70B313E02A3A3C3EB2
:10A8C0007C223F7F00000000553F02082B2C3B3DBF
:10A8D0005B5D00003A630020464154333220202063
:10A8E000000000004820005D401E01281AD804F135
:10A8F0004900FEF7A7FC78B104F14B00FEF7A2FC7B
:10A90000802806DA04F15800FEF7A2FCB0F5803F7B
:10A9100008D304F14E0000E004E0FEF793FC08B118
:10A92000002095E74AF65520874201D102208FE7A3
:10A9300003208DE72DE9FF4107460D4600213846EB
:10A94000FFF778FF0646022E06D0032E00D21DB96F
:10A95000304604B0BDE8F08100BF00240AE007F5EE
:10A96000FB7101EB041101F10800FEF771FC4DF8D9
:10A970002400641C042CF2D30DB1681E00E00020FA
:10A98000044600BF5DF8240028B15DF82410384665
:10A99000FFF750FF00E0032006462DB9022E03D337
:10A9A000601C04460428EDD33046D2E72DE9F74F6A
:10A9B00084B00021059801600498FFF713FF03900D
:10A9C0000398002803DA0B2007B0BDE8F08FFE499A
:10A9D000039851F820400CB90C20F5E70598046065
:10A9E000069800F0FE000690207878B16078FEF7B7
:10A9F00039FB074607F0010040B9069820B107F07F
:10AA0000040008B10A20DFE70020DDE70020207005
:10AA1000039860706078FEF73BFB074607F0010083
:10AA200008B10320D0E7069820B107F0040008B170
:10AA30000A20C9E700212046FFF77CFF0546042DC8
:10AA400001D10120C0E7022D01D30D20BCE7D4F8CD
:10AA5000349004F14300FEF7F5FBB0F5007F01D020
:10AA60000D20B1E704F14E00FEF7ECFB064626B9D7
:10AA700004F15C00FEF7ECFB064626624820005D10
:10AA8000A070A078012804D0A078022801D00D2061
:10AA90009AE7A07846434520005D6081608918B13F
:10AAA0006089411E084008B10D208DE704F149007E
:10AAB000FEF7C8FB2081207A00F00F0008B10D20BE
:10AAC00082E704F14B00FEF7BDFB8246BAF1000FAE
:10AAD00004D104F15800FEF7BBFB824604F14600A6
:10AAE000FEF7B0FB8346BBF1000F01D10D206BE7F1
:10AAF0000BEB0600218900EB1110029002988245B1
:10AB000001D20D2060E70298AAEB00006189B0FB3A
:10AB1000F1F8B8F1000F01D10D2055E70025AB4841
:10AB2000804500D803254FF6F570804500D80225F2
:10AB300040F6F570804500D801250DB90D2043E79A
:10AB400008F10200E061C4F8249009EB0B00A06258
:10AB5000029848442063032D13D104F16200FEF7EC
:10AB600071FB08B10D202FE7208908B10D202BE7DC
:10AB700004F16400FEF76CFBE062E0698000019084
:10AB800014E0208908B90D201EE7A06A3044E06275
:10AB9000022D02D1E069400007E0207F00F00100B3
:10ABA000E16901EB410100EB51000190216A01983C
:10ABB00000F2FF10B1EB502F01D20D2004E74FF04F
:10ABC000FF306061206180202071032D2DD104F1C0
:10ABD0006800FEF737FB012827D109F10101204663
:10ABE000FEF7A6FC08BB0020207104F23620FEF719
:10ABF00029FB4AF65521884217D104F13800FEF7A7
:10AC000027FB7349884210D104F50770FEF720FB3B
:10AC10007049884209D104F50870FEF719FB60619C
:10AC200004F50970FEF714FB206125706A4800885E
:10AC3000401C80B268490880E0800020A061204666
:10AC4000FEF73FFC0020BFE670B504460D4609261E
:10AC50008CB1206878B12068007860B1A088216844
:10AC6000C988884207D121684878FEF7FBF900F0CF
:10AC7000010000B900260EB9206800E0002028601D
:10AC8000304670BDF7B582B016460398019001A812
:10AC9000FFF7A8FD0546002D02DA0B2005B0F0BD38
:10ACA000494850F8254024B12046FEF70AFC002010
:10ACB0002070029810B10020029908704249029851
:10ACC00041F825000EB90020E8E7002202A903A8F8
:10ACD000FFF76CFE07463846E0E72DE9F74F90B0E6
:10ACE000044616461CB9092013B0BDE8F08F06F0E3
:10ACF0003F06324602A911A8FFF758FE0546002D6F
:10AD00006CD1029803904FF40070FEF714F983465B
:10AD1000BBF1000F01D11120E6E70298C0F80CB09A
:10AD200003A81199FFF7F8FC05468DB99DF83B0083
:10AD300000F0800008B106250AE026F0010008B105
:10AD4000012000E00020014603A8FEF7F2FA0546C4
:10AD500006F01C00002867D06DB1042D08D1FEF765
:10AD600023FB18B103A8FFF7EBF900E0122005461A
:10AD700046F008060AE09DF8120000F0110008B144
:10AD8000072503E006F0040000B10825002D5CD182
:10AD900006F00800002858D0FEF72FFA00900B9913
:10ADA00001F10E000099FEF765FA0B9901F116000A
:10ADB0000099FEF75FFA0B990298FEF76EFF814645
:10ADC00020200B99C8720AE034630020F5FFFF0FC2
:10ADD000525261417272416138630020B3E0002237
:10ADE0000B990298FEF76CFF0B9901F11C000021F2
:10ADF000FEF740FA01200299C870B9F1000F24D083
:10AE00000298D0F834A00022494603A8FEF70CFDB2
:10AE1000054645B951460298FEF78AFB0546A9F159
:10AE200001000299086110E07DB99DF8120000F060
:10AE3000100008B1042508E006F0020028B19DF8D2
:10AE4000120000F0010000B10725BDB906F00800AE
:10AE500008B146F040060298406B60620B98A06211
:10AE600026F0010008B1012000E00020014603A8FF
:10AE7000FEF7ABFA2061206900B90225002D5FD1F1
:10AE80000B990298FEF709FFA0600B9901F11C00D5
:10AE9000FEF7DEF9E0600020E06202982060029890
:10AEA000C088A0802675002060752062A0614FF4E4
:10AEB000007104F1300004F000FF06F02000E0B360
:10AEC000E068D0B3E068A061029840894002019038
:10AED000A768D4F80C800DE039462046FEF791FBB8
:10AEE0000746012F00D80225781C00B901250198DA
:10AEF000A8EB000815B901988045EDD8E761CDB9F8
:10AF0000C8F30800B0B139460298FEF76DFB8246DF
:10AF1000BAF1000F01D102250CE00AEB58202062A3
:10AF2000226A02994878012304F13001FEF7CCF837
:10AF300000B101250DB1206900E001E0FEF7A1FAA2
:10AF40005846FDF7FEFF0DB1002020602846CBE6F5
:10AF50002DE9FF4F85B0044615469A46DDF818B036
:10AF60000020CAF8000003A92046FFF76DFE0490F8
:10AF7000049810B9607D049018B1049809B0BDE838
:10AF8000F08F207D00F0010008B90720F6E7A169E5
:10AF9000E068401A01900198854200D9019DA8E01F
:10AFA000208BC0F30800002874D103984089401E0C
:10AFB000A16900EA5129B9F1000F1FD1A06910B9A8
:10AFC000A06802900CE0E06A28B12046A169FEF773
:10AFD00008FD029004E02046E169FEF712FB0290B2
:10AFE0000298022802D202206075C7E70298401C2E
:10AFF00010B901206075C1E70298E061E16903982A
:10B00000FEF7F2FA064616B902206075B6E74E441E
:10B010004FEA5528B8F1000F29D009EB0800039931
:10B020004989884203D903984089A0EB090803990C
:10B030004878434632465946FEF746F810B101209B
:10B0400060759BE7207D00F0800068B1206A801B5E
:10B05000404509D2216A891B0BEB41204FF4007255
:10B0600004F1300104F010FE4FEA482737E0206A6F
:10B07000B04220D0207D00F0800080B1226A039988
:10B080004878012304F13001FEF74DF818B1012092
:10B09000607573E710E0207D00F07F002075039954
:10B0A00048780123324604F13001FEF70DF810B163
:10B0B0000120607562E72662208BC0F30800C0F5AE
:10B0C0000077AF4200D92F46208BC0F3080204F16D
:10B0D000300011183A46584604F0D6FD00BFED1B6B
:10B0E000DAF800003844CAF80000BB44A0693844CC
:10B0F000A061002D7FF454AF00203FE72DE9FF4F02
:10B1000083B0044615469B46049800900020CBF877
:10B11000000001A92046FFF797FD0290029810B9A0
:10B12000607D029018B1029807B0BDE8F08F207DD5
:10B1300000F0020008B90720F6E700BFA069284424
:10B14000A169884202D2A069C0F1FF35C3E0208B1B
:10B15000C0F3080000287DD101984089401EA169F4
:10B1600000EA512ABAF1000F26D1A06938B9A768C0
:10B1700097B900212046FEF7A4FB07460CE0E06AE1
:10B1800028B12046A169FEF72CFC074604E02046C2
:10B19000E169FEF796FB074607B99FE0012F02D150
:10B1A00002206075C0E7781C10B901206075BBE70C
:10B1B000E761A06800B9A760207D00F0800078B149
:10B1C000226A01994878012304F13001FDF7ABFFB1
:10B1D00010B101206075A7E7207D00F07F00207589
:10B1E000E1690198FEF700FA064616B9022060757B
:10B1F0009AE756444FEA5529B9F1000F2BD00AEBD4
:10B20000090001994989884203D901984089A0EB36
:10B210000A09019948784B4632460099FDF783FFA9
:10B2200010B1012060757FE7206A801B48450ED26F
:10B23000206A801B009A02EB40214FF4007204F157
:10B24000300004F021FD207D00F07F0020754FEAE2
:10B2500049282BE013E0206AB0420FD0E168A069D2
:10B2600088420BD2019948780123324604F130011B
:10B27000FDF72AFF10B10120607555E72662208B8B
:10B28000C0F30800C0F50078A84500D9A846218B76
:10B29000C1F3080204F1300150184246009904F04D
:10B2A000F3FC207D40F08000207500BFA5EB080571
:10B2B000DBF800004044CBF80000009840440090C8
:10B2C000A0694044A061E168A069884201D9A069F1
:10B2D00000E0E068E060002D7FF439AF00BF207D22
:10B2E00040F04000207500201EE7F8B5044669468E
:10B2F0002046FFF7A9FC0646002E44D1207D00F031
:10B30000400000283FD0207D00F0800070B1226A0C
:10B3100000994878012304F13001FDF704FF08B1DA
:10B320000120F8BD207D00F07F002075FDF765FF4E
:10B330000746616A0098FEF7FBF806461EBBA56A41
:10B34000E87A40F02000E8722946A2682068FEF7FB
:10B35000B7FC05F11C00E168FDF78CFF394605F1EB
:10B360001600FDF787FF002105F11200FDF77CFFB5
:10B3700001200099C8700098FEF7F4F80646207D79
:10B3800000F0BF0020753046CBE738B505462846AB
:10B39000FFF7ABFF044664B969462846FFF754FC43
:10B3A000044634B92869FEF76CF804460CB900204D
:10B3B0002860204638BD31B56846FFF713FA0446C9
:10B3C000002C01DA0B2038BDFD490C700020FAE793
:10B3D00031B58EB0002269460EA8FFF7E7FA0446A1
:10B3E00074BB009801904FF40070FDF7A4FD054672
:10B3F00015B911200FB030BD0098C56001A80E9995
:10B40000FFF78AF90446ACB99DF8330000F08000DC
:10B4100018B10099039888610CE09DF80A0000F0CB
:10B42000100030B109990098FEF737FC0099886147
:10B4300000E005242846FDF784FD042C00D10524F6
:10B440002046D7E72DE9F04F89B004460D4607A9FD
:10B450002046FFF7F9FB0890089808B9607D08902E
:10B46000089818B1089809B0BDE8F08FE06A002884
:10B470007CD0681C002843D1D4F82C9059F8040BD8
:10B48000029002200190A76867B300BF03970020D5
:10B4900004900198801C019000BF05970498401CFF
:10B4A000049039462046FEF7ACF80746012F02D833
:10B4B00002206075D7E7781C10B901206075D2E7CB
:10B4C0000598401C8742E8D0DDE90101884205D893
:10B4D000049849F8040B039849F8040B0798C069CD
:10B4E000B842D3D80198E16A0860DDE901018842D9
:10B4F00003D80020C9F80000FAE011200890F7E016
:10B50000E068A84200D2E568A561002DF4D0691E6C
:10B510002046FEF766FAE061E1690798FEF764F8F5
:10B520008246BAF1000F02D1022060759BE70798AE
:10B530004089401E691E00EA51208244208BC0F3DE
:10B5400008000028D8D0206A5045D5D0207D00F0D2
:10B55000800080B1226A07994878012304F1300104
:10B56000FDF7E1FD18B1012060757CE712E0207D58
:10B5700000F07F002075079948780123524604F1B6
:10B580003001FDF7A1FD10B1012060756BE7C4F833
:10B5900020A0ADE0E068A84204D2207D00F00200C7
:10B5A00000B9E568A06906904FF0000BC4F818B028
:10B5B000002D6AD0079840894FEA4028069890B13C
:10B5C000681EB0FBF8F10698401EB0FBF8F081420F
:10B5D00009D30698401EA8F101018843A061A06923
:10B5E0002D1AE66912E0A6687EB900212046FEF712
:10B5F00068F90646012E02D10220607533E7701CFF
:10B6000010B9012060752EE7A660E661D6B325E08B
:10B61000A5EB0805A0694044A061207D00F0020070
:10B6200040B100BF31462046FEF74BF9064636B919
:10B63000002515E031462046FDF7E3FF0646701C65
:10B6400010B9012060750EE7012E03D90798C06973
:10B65000B04202D80220607505E7E6614545D7D8BB
:10B6600000BFA0692844A061C5F3080050B131466D
:10B670000798FDF7B9FF8346BBF1000F03D1022005
:10B680006075F0E601E00BEB552BE168A06988429C
:10B6900005D9A069E060207D40F040002075208B36
:10B6A000C0F3080020B3206A584521D0207D00F067
:10B6B000800078B1226A07994878012304F13001AB
:10B6C000FDF731FD10B101206075CCE6207D00F062
:10B6D0007F0020750799487801235A4604F130010C
:10B6E000FDF7F2FC10B101206075BCE6C4F820B093
:10B6F0000898B8E673B582B0044614B9092004B0BE
:10B7000070BD002201A903A8FFF750F90546002DDE
:10B710003ED1019820604FF40070FDF70CFC064606
:10B720000EB91120EBE70198C66020460399FEF799
:10B73000F3FF05461DBB2F20005D00F0800050B9CF
:10B74000A07900F0100028B1216A0198FEF7A5FA4F
:10B75000A06000E0052595B90198C088A08000216F
:10B760002046FEF7B8F905464DB9A06840B1002162
:10B770002046FDF72AFE2061206900B9122501E06C
:10B78000002020613046FDF7DCFB042D00D10525AB
:10B790000DB1002020602846B1E738B5044669465F
:10B7A0002046FFF751FA054645B9206918B12069CE
:10B7B000FDF767FE05460DB900202060284638BD1C
:10B7C0003A630020F8B507460E4669463846FFF74B
:10B7D0003BFA044644BB2EB900213846FEF77BF9FC
:10B7E000044621E04FF40070FDF7A5FB05460DB9B6
:10B7F0001120F8BD0098C56000213846FEF7B5FB62
:10B800000446042C00D100245CB931463846FEF7CA
:10B810006AFD00213846FEF7ABF90446042C00D13E
:10B8200000242846FDF78DFB2046E2E773B58EB075
:10B830000E46002201A90EA8FFF7B8F80546FDB98B
:10B840004FF40070FDF777FB044614B9112010B0D7
:10B8500070BD0198C46001A80E99FEF75DFF054612
:10B860005DB99DF8330000F0800008B1062504E0C2
:10B870001EB1314601A8FEF736FD2046FDF761FBFB
:10B880002846E4E72DE9F74F86B089469246002224
:10B8900005A906A8FFF78AF88046B8F1000F6BD11A
:10B8A0000598CAF8000005984169C069801E814268
:10B8B00004D805984069C9F800005DE000250598A6
:10B8C000007801281BD102260598009000BF314660
:10B8D0006846FDF796FE0746781C10B94FF0010840
:10B8E0000CE0012F02D14FF0020807E007B96D1CF0
:10B8F000701C06460599C9698842E8D32FE005986F
:10B90000C6690598D0F828B0002400BF54B959463C
:10B910000BF1010B0598FDF70BFE8046B8F1000F07
:10B9200000D01BE005980078022808D1059938312D
:10B930000819FDF787FC00B96D1CA41C09E00599E6
:10B9400038310819FDF784FC20F0704000B96D1CF7
:10B95000241DC4F30804701E061ED7D100BFB8F121
:10B96000000F09D1C9F80050059845610598007984
:10B9700040F0010005990871404609B0BDE8F08F1C
:10B98000F8B5044669462046FFF75EF9054615B945
:10B99000607D051E01D02846F8BD207D00F0020024
:10B9A00008B90720F8E7E168A06988423FD2A0699A
:10B9B00040B900222046A168FDF736FF0546002069
:10B9C000A06016E02046E169FDF71BFE0646002553
:10B9D000701C00B90125012E00D102254DB9009837
:10B9E000C069B04205D931462046E269FDF71CFF27
:10B9F0000546A069E060207D40F04000207595B9C3
:10BA0000207D00F0800070B1226A009948780123FF
:10BA100004F13001FDF787FB08B1012503E0207D2B
:10BA200000F07F00207515B165752846B4E72846FB
:10BA3000B2E771B59BB00025022269461BA8FEF74C
:10BA4000B5FF0446002C66D100980E904FF40070AC
:10BA5000FDF771FA064616B911201CB070BD0098AA
:10BA6000C6600EA81B99FEF757FE04462CB99DF838
:10BA7000670000F0200000B1062424B902210EA8BE
:10BA8000FDF757FC0446002C42D19DF8670000F0FA
:10BA9000800008B1062405E09DF83E0000F001009A
:10BAA00000B1072414BB16990098FEF7F6F8054676
:10BAB0009DF83E0000F01000C0B100988069A842D7
:10BAC00001D1072412E0009801900395002101A8FC
:10BAD000FEF701F804464CB9002101A8FEF745FA2B
:10BAE000044604B90724042C00D1002484B90EA80C
:10BAF000FEF7C9FB044634B92DB1002229460EA831
:10BB0000FDF792FE04461CB90098FDF72BFD044694
:10BB10003046FDF716FA20469FE72DE9F14193B034
:10BB20000222694613A8FEF741FF0446002C7DD18E
:10BB3000009806904FF40070FDF7FDF906461EB917
:10BB4000112014B0BDE8F0810098C66006A81399D2
:10BB5000FEF7E2FD044604B90824042C05D19DF843
:10BB6000470000F0200000B10624042C6AD10098A0
:10BB70000190002101A8FDF7A4FE0546002405B9A7
:10BB80000724012D00D10224681C00B90124FDF70F
:10BB900034FB8046BCBB29460098FDF73BFF0446BA
:10BBA0008CBB20220B210098383004F07FF82E2027
:10BBB000009981F838001021009880F84310414620
:10BBC00000984E30FDF756FB2A4600993831009810
:10BBD000FEF776F82022009938310098583004F0AA
:10BBE00053F82E21009880F85910089F3A46009982
:10BBF00058310098FEF764F801200099C87006A833
:10BC0000FEF79EFA0446C4B90E9901F116004146AA
:10BC1000FDF730FB2A460E990098FEF751F81020E8
:10BC20000E99C87201200099C87000E00DE01CB99F
:10BC30000098FDF797FC044604E00022294601A87D
:10BC4000FDF7F2FD3046FDF77CF9204679E72DE956
:10BC5000F341A4B025A8FEF7C5FD022209A924A836
:10BC6000FEF7A4FE0446002C70D1099817904FF4FB
:10BC70000070FDF760F907461FB9112026B0BDE836
:10BC8000F0810998C76017A82499FEF745FD04467E
:10BC90002CB99DF88B0000F0A00000B1062424B957
:10BCA000022117A8FDF745FB0446002C6DD1202288
:10BCB00001A81F9903F0E8FF342217A90AA803F08E
:10BCC000E3FF0AA82599FEF727FD04465CB91999F8
:10BCD0000C98884205D11C990F98884201D1042004
:10BCE00000E008200446042C45D10AA8FEF728FAF3
:10BCF0000446002C3FD1129D13220DF1110105F1D4
:10BD00000D0003F0C1FF9DF80F00E872E87A00F023
:10BD1000100018B9E87A40F02000E8720120099973
:10BD2000C870E87A00F0100028B30C99199888427E
:10BD300021D029460998FDF7B0FF80464146099871
:10BD4000FDF752FC064616B9022414E020E0314605
:10BD50000998FDF7EDFB0446099800F1580554B920
:10BD600068782E2807D129460C9A0998FDF7A8FF74
:10BD700001200999C87044B917A8FEF784FA04464F
:10BD80001CB90998FDF7EEFB04463846FDF7D9F8D3
:10BD9000204673E72DE9FF4F85B09A4603AA01219B
:10BDA0000598FDF7E3F918B1012009B0BDE8F08F5F
:10BDB000DDF80C904FF03F08082701E07806070EE9
:10BDC00037B1B9FBF7F0B0FBF8F0B0F5806FF5D8FC
:10BDD00007B9FF274FF40071504603F06EFF0AF5D4
:10BDE000DF764FF0000B444669E0069850F82B5080
:10BDF000642D07D801D1484603E06420B9FBF0F078
:10BE0000684305466019484501D8601901D3A9EB7C
:10BE1000040505B959E0214606F10800FDF72AFAA4
:10BE2000294606F10C00FDF725FA07983071B4FB9E
:10BE3000F8F0B0FBF7F00490B4FBF8F0B0FBF7F1CA
:10BE400007FB1100C0B20290B4FBF8F008FB1040F1
:10BE5000401CC0B2019002987070C021049801EAA1
:10BE6000900001990843B0700498F0706019401E6A
:10BE7000B0FBF8F0B0FBF7F004906019401EB0FB87
:10BE8000F8F0B0FBF7F107FB1100C0B202906019A7
:10BE9000401EB0FBF8F108FB1100401CC0B201903D
:10BEA00002987071C021049801EA9000019908433A
:10BEB000B0710498F07110360BF1010B2C44BBF1FA
:10BEC000040F02D20CB14C458FD300BF4AF6552166
:10BED0000AF5FF70FDF7C8F90123002251460598C5
:10BEE000FDF721F908B101205FE700205DE72DE9AA
:10BEF000FF4F99B00F46154619A8FEF773FC029044
:10BF00000298002803DA0B201DB0BDE8F08FFE492F
:10BF1000029851F8200028B10021FB4A029852F8FB
:10BF2000200001700298C0B216900020159007B949
:10BF3000F64F1698FDF7ACF80190019800F001005B
:10BF400008B10320E0E7019800F0040008B10A20DE
:10BF5000DAE778681390139838B913AA0321169872
:10BF6000FDF704F908B101201390139840B113981C
:10BF7000B0F5004F04D81398401E1399084008B13B
:10BF8000012013904FF40079387800F00F001890DA
:10BF90007878012804DB7878022801DC787800E0E2
:10BFA00001200590B96889B1B968B1F5004F0DD885
:10BFB00048464FEAE97109EBD1614911BA68B2FB11
:10BFC000F1F301FB132109B9B96801E04FF40071E5
:10BFD0000491F868B0F1807F05D8F868411E0840E8
:10BFE00008B9F86800E0002006900698B0FBF9F068
:10BFF00006901C98B0FBF9F01490149808B9112021
:10C0000082E72C462CB9149901FB09F0FCF793FF49
:10C0100004460CB9112077E7002010900F9000BF64
:10C0200010AA01211698FDF7A1F828B115B92046EC
:10C03000FCF787FF012067E7189800F0080040B977
:10C0400010983F2805D93F200F90DDE90F01081A0D
:10C0500010901098802805D215B92046FCF771FF82
:10C060000E2051E700BF00BF0698802801D980202C
:10C070000690189800F0020030B1189800F0010006
:10C0800010B94FF003080CE0189800F0010028B92F
:10C0900015B92046FCF755FF132035E74FF002088D
:10C0A00000BF00BFFDF7A9F810990844119000BF28
:10C0B000069EB8F1030F31D1A6B910984FEA504B44
:10C0C00000200390012603E00398401C03907600B3
:10C0D0008F49039831F8100020B1039831F810000F
:10C0E0005845F1D91098B0FBF6FA082000EB8A0009
:10C0F0004844401EB0FBF9F0089020200990002031
:10C1000007904FF6F570824502D9824882453BD9A7
:10C1100015B92046FCF715FF0E20F5E6A6B91098D4
:10C120004FEA103B00200390012603E00398401CD7
:10C13000039076007849039831F8100020B10398F5
:10C1400031F810005845F1D91098B0FBF6FA40F6D6
:10C15000F570824503D9042000EB4A0B07E04FF04D
:10C1600001080AEB4A00401C032101EB500B0BEBCA
:10C170000900401EB0FBF9F00890012009900498D6
:10C180004001B0FBF9F0079009990F9808440E9010
:10C19000059A08990E9801FB0201079808440D9032
:10C1A00013990D980844401E491E20EA01010D987C
:10C1B000A1EB000BB8F1030F06D109985844099080
:10C1C0000E9858440E9013E00598BBFBF0F100FB6D
:10C1D00011B038B1ABF1010B0998401C09900E98D1
:10C1E000401C0E900598BBFBF0F10898084408909D
:10C1F0000D9800EB06110F98081A1099884205D97E
:10C2000015B92046FCF79DFE0E207DE61099099891
:10C210000A1A0599089800FB11210798081AB0FB23
:10C22000F6FAB8F1030F0FD14FF6F57082450BD82F
:10C23000069818B97008069000B148E015B9204674
:10C24000FCF77FFE0E205FE6B8F1020F31D14FF60A
:10C25000F57082451CD9069830B94020B0EB460FE6
:10C2600002D37000069032E0189800F0020010B17E
:10C270004FF003082BE0069820B970000690802844
:10C2800000D824E015B92046FCF75BFE0E203BE603
:10C2900040F6F57082450CD8069820B970000690DB
:10C2A000802800D813E015B92046FCF74AFE0E207E
:10C2B0002AE6B8F1010F09D140F6F570824505D99B
:10C2C00015B92046FCF73DFE0E201DE600E0EFE626
:10C2D00000BF4946204603F0F0FC10A00168216031
:10C2E0004168616001892181807AA072494604F128
:10C2F0000B00FCF7B9FF6673099881B204F10E00D8
:10C30000FCF7B2FF05980FE034630020F43F020809
:10C31000E43F0208F5FFFF0FD63F0208EBFE904D09
:10C3200053444F53352E30002074B8F1030F01D120
:10C33000002000E0049881B204F11100FCF794FFA2
:10C340001098B0F5803F06D2109881B204F1130026
:10C35000FCF78AFF04E004F120001099FCF78AFF43
:10C36000F82060753F2104F11800FCF77DFFFF21E4
:10C3700004F11A00FCF778FF04F11C000F99FCF798
:10C3800079FFB8F1030F25D104F143001199FCF7AF
:10C3900071FF04F124000899FCF76CFF022104F1FD
:10C3A0002C00FCF767FF012104F13000FCF75CFF73
:10C3B000062104F13200FCF757FF802084F840008A
:10C3C000292084F84200132291A104F1470003F0D0
:10C3D0005BFC16E004F127001199FCF74BFF08986D
:10C3E00081B204F11600FCF73FFF802084F824009E
:10C3F000292084F8260013228AA104F12B0003F0DF
:10C4000043FC4AF6552104F5FF70FCF72DFF01238C
:10C4100021460F9A1698FCF786FE28B115B92046DA
:10C42000FCF78FFD01206FE5B8F1030F32D1012336
:10C430000F9A921D21461698FCF775FE4946204634
:10C4400003F03BFC7C492046FCF714FF7B4904F5D4
:10C45000F270FCF70FFFAAF1010104F5F470FCF78C
:10C4600009FF022104F5F670FCF704FF4AF6552196
:10C4700004F5FF70FCF7F8FE01230F9AD21D214648
:10C480001698FCF750FE01230F9A521C214616986D
:10C49000FCF749FE149800FB09F1204603F00DFC5F
:10C4A0000E980C900020039047E0B8F1030F10D1D4
:10C4B0006FF007012046FCF7DDFE4FF0FF31201D35
:10C4C000FCF7D8FE6FF0704104F10800FCF7D2FED3
:10C4D0000AE0B8F1010F01D1594801E06FF00700FF
:10C4E00001462046FCF7C6FE0898129000BF14993A
:10C4F0001298884201D9149800E0129883465B464E
:10C5000021460C9A1698FCF70EFE28B115B9204664
:10C51000FCF717FD0120F7E44946204603F0CDFB68
:10C520000C9858440C901298A0EB0B0012901298A3
:10C530000028DCD10398401C039005990398884299
:10C54000B3D3B8F1030F01D1304600E00798129041
:10C5500000BF14991298884201D9149800E01298EB
:10C5600083465B4621460C9A1698FCF7DCFD28B101
:10C5700015B92046FCF7E5FC0120C5E40C985844A9
:10C580000C901298A0EB0B00129012980028E0D1AA
:10C5900000BFB8F1030F02D10C2017900DE01098E6
:10C5A000B0F5803F02D30620179006E0B8F1020FE5
:10C5B00001D1042000E00120179000BF189800F07E
:10C5C000080090B910980A9000200B9023460AA901
:10C5D000DDE91602FFF7DEFB0090009828B115B9DF
:10C5E0002046FCF7AEFC00988EE400221146169817
:10C5F000FCF7BCFD28B115B92046FCF7A2FC0120D0
:10C6000082E415B92046FCF79CFC00207CE4000085
:10C610004E4F204E414D452020202046415433327C
:10C62000202020004E4F204E414D45202020204606
:10C6300041542020202020005252614172724161F9
:10C64000F8FFFF001CB501210420F4F75BFC01207A
:10C650008DF8040000208DF8060001208DF80700F9
:10C6600002208DF80500102000906946FE48F4F77E
:10C670006DF91021FC48F4F7E5F91CBD10B5102147
:10C68000F948F4F7DDF9C820F7F77FFD4FF47A7029
:10C69000F7F77BFD1021F448F4F7D4F910BD10B57D
:10C6A0000221F248F4F7CCF910BD10B50221EF4891
:10C6B000F4F7C8F910BD70B500240020EC49C8702B
:10C6C00008704871FFF7BEFFFFF7E9FF4FF47A707B
:10C6D000F7F75BFDFFF7D2FF4FF4FA60F7F755FD70
:10C6E000F9F712F8002513E0F9F70EF8E1A005F0CC
:10C6F00081FE41F28830F7F748FDE1A1E44803F0FC
:10C70000E7FA0546601CC4B2032C01DD012070BDB0
:10C710000A2C01DA012000E000200DB9012100E01F
:10C72000002108400028DFD10120D1494871D9A05B
:10C7300005F060FE4FF47A70F7F727FDD9A005F0F9
:10C7400059FE4FF4FA70F7F720FD41F28830F7F701
:10C750001CFD002518E0F8F7D7FFD6A005F04AFE2B
:10C760004FF4FA70F7F711FDD4A1C94803F0B0FAFD
:10C7700005463DB9FFF793FF4FF4FA70F7F705FD53
:10C78000FFF77CFF601CC4B20DB9012000E000205F
:10C790000A2C01DA012100E0002108400028DAD14A
:10C7A000F8F7B2FFC6A005F025FE4FF49670F7F734
:10C7B000ECFCC9A005F01EFE4FF47A70F7F7E5FC1B
:10C7C000BEA1B34803F084FA0546C5A005F012FEE9
:10C7D0004FF4FA70F7F7D9FCAEA005F00BFE4FF45A
:10C7E0007A70F7F7D2FCB5A1A94803F071FA0546B3
:10C7F000BBA005F0FFFD4FF4FA70F7F7C6FCF8F7A1
:10C8000083FFBBA005F0F6FD4FF4FA70F7F7BDFC0F
:10C81000AAA19F4803F05CFA0546002411E0601CC1
:10C82000C4B2B3A005F0E6FD4FF4FA70F7F7ADFC23
:10C83000B2A1974803F04CFA05460A2C01DD01200D
:10C8400065E70F2C01DA012000E000200DB901217D
:10C8500000E0002108400028E1D10120844948710E
:10C86000F8F752FFA7A005F0C5FD4FF47A70F7F76F
:10C870008CFCA7A1864803F02BFA0546002413E0A0
:10C88000F8F742FF9FA005F0B5FD4FF4FA60F7F707
:10C890007CFC9FA17E4803F01BFA0546601CC4B2D5
:10C8A0000A2C01DD012032E70F2C01DA012000E023
:10C8B00000200DB9012100E0002108400028DFD14F
:10C8C00001206B49C870F8F71FFF94A005F092FD96
:10C8D0004FF49670F7F759FC93A16D4803F0F8F9FF
:10C8E000054655B1287A3038E979303901EB8101B4
:10C8F00000EB41005E49087000BFF8F705FF00201B
:10C9000005E770B50025F8F7FFFE89A005F072FD78
:10C910004FF4FA70F7F739FC89A15D4803F0D8F9B4
:10C9200004460FE0F8F7F0FE81A005F063FD4FF438
:10C93000FA70F7F72AFC82A1554803F0C9F90446BA
:10C94000681CC5B20CB9012000E00020032D01DAFB
:10C95000012100E0002108400028E3D104B170BDAE
:10C9600044B9F8F7D1FE72A005F044FD4FF4FA7017
:10C97000F7F70BFC00BFF2E7F0B585B006460F46AF
:10C9800000241421684603F098F94FF47A70F7F701
:10C99000FCFBF8F7B9FE6E4A6EA1684605F03AFD59
:10C9A0006B4A4D3AA2F114016CA005F023FD4FF43F
:10C9B0007A70F7F7EAFB6FA1354803F089F905466D
:10C9C00019E0FFF79EFF4FF4FA70F7F7DEFBF8F778
:10C9D0009BFE5F4A4D3AA2F1140160A005F00AFDEA
:10C9E0004FF47A70F7F7D1FB62A1294803F070F990
:10C9F0000546601CC4B20DB9012000E00020052CE2
:10CA000001DA012100E0002108400028D9D1F8F71F
:10CA10007BFE4F4B3133A3F114024D4959A005F071
:10CA2000E9FC4FF4FA60F7F7B0FB5DA1184803F09A
:10CA30004FF90546BFE0FFF764FF4FF4FA70F7F7D0
:10CA4000A4FBF8F761FE424B3133A3F114024049D5
:10CA50004CA005F0CFFC4FF47A70F7F796FB50A18D
:10CA60000B4803F035F9A3E000080240000402403F
:10CA70003D63002041542B4350494E3F0D0A0000B6
:10CA80002B4350494E3A2052454144590000000082
:10CA90008366002041542B4350534D533D300D0AC3
:10CAA0000000000041542B5153434C4B3D300D0AC4
:10CAB0000000000041540D0A000000004F4B000030
:10CAC00041542B5153454C465245474953544552C6
:10CAD0003D310D0A00000000415445300D0A0000B0
:10CAE00041542B514C45444D4F44453D310D0A00B6
:10CAF00041542B51434349440D0A00002B514343F9
:10CB00004944000041542B43474154543F0D0A000F
:10CB10002B43474154543A203100000041542B43E9
:10CB20004553510D0A0000002B43455351000000AE
:10CB300041542B514D54434C4F53453D300D0A0049
:10CB40002B514D54434C4F53453A20302C3000006C
:10CB50002A660020222573220000000041542B5138
:10CB60004D544F50454E3D302C25732C25730D0AE6
:10CB7000000000002B514D544F50454E3A20302CB0
:10CB80003000000041542B514D54434F4E4E3D3028
:10CB90002C222573222C25732C25730D0A000000EE
:10CBA0002B514D54434F4E4E3A20302C302C3000F8
:10CBB0000546601CC4B20DB9012000E00020052C20
:10CBC00001DA012100E00021084000287FF433AFA2
:10CBD000F8F79AFDFA49FBA005F00CFC4FF47A70C7
:10CBE000F7F7D3FAAFF22C11FE4803F071F80546BF
:10CBF00017E0FFF786FE4FF4FA70F7F7C6FAF8F77A
:10CC000083FDEF49EFA005F0F5FB4FF47A70F7F7DD
:10CC1000BCFAAFF25811F34803F05AF80546601C0D
:10CC2000C4B20DB9012000E00020052C01DA012179
:10CC300000E0002108400028DBD1F8F765FDE0495D
:10CC4000E9A005F0D7FB4FF47A70F7F79EFAAFF240
:10CC50009411E44803F03CF8054617E0FFF751FE55
:10CC60004FF4FA70F7F791FAF8F74EFDD449DEA0C9
:10CC700005F0C0FB4FF47A70F7F787FAAFF2C411F2
:10CC8000D84803F025F80546601CC4B20DB9012050
:10CC900000E00020052C01DA012100E0002108401D
:10CCA0000028DBD115B10120D649087115B9002043
:10CCB000D449087105B0F0BD2DE9FC4104460D468C
:10CCC0000020009001900026F8F71EFD2246CEA11C
:10CCD000684605F09FFB2A466946CCA005F08AFB12
:10CCE0004FF47A70F7F751FACEA1BE4802F0F0FF88
:10CCF00007460AE04FF47A70F7F747FAC9A1B94836
:10CD000002F0E6FF0746701CC6B20FB90A2EF1DB2F
:10CD1000BDE8FC812DE9F04106460F460025A846F6
:10CD2000F8F7F2FCC1480078012805D13246A44941
:10CD3000BFA005F05FFB0EE0BC480078022805D1DB
:10CD400032469F49C3A005F055FB04E032469C499A
:10CD5000CAA005F04FFB4FF4FA70F7F716FAD0A10E
:10CD6000A04802F0B5FF044640E0681CC5B2AF48D9
:10CD70000078012805D132469149ADA005F03AFB73
:10CD80000EE0AA480078022805D132468C49B1A0AD
:10CD900005F030FB04E032468949B8A005F02AFBD3
:10CDA0004FF4FA70F7F7F1F9BDA18E4802F090FF49
:10CDB0000446002C1AD1F8F7A7FC9C4800780128FB
:10CDC00005D132467E499AA005F014FB0EE0974843
:10CDD0000078022805D1324679499EA005F00AFB69
:10CDE00004E032467649A5A005F004FB0CB9142DE9
:10CDF000BBDB14B90120BDE8F0814FF4FA70F7F7FE
:10CE0000C4F93946A7A005F0F5FA4FF47A70F7F7A0
:10CE1000BCF90025AFF25C31724802F059FF0446BC
:10CE200016E0681CC5B239469EA005F0E3FA4FF43F
:10CE30007A70F7F7AAF9AFF27C316A4802F048FF3E
:10CE400004462CB9F8F760FC394696A005F0D2FAF2
:10CE50000CB9142DE5DB0CB10020CCE70120CAE7AA
:10CE600010B591A15F4802F033FF04460CB1F8F70A
:10CE70004BFC10BD7CB50025FFF7E4FBFFF70FFC72
:10CE80004FF47A70F7F781F9FFF7F8FB4FF4FA7077
:10CE9000F7F77BF9AFF2044005F0ACFA4FF47A7083
:10CEA000F7F773F9AFF2044005F0A4FA4FF4FA5023
:10CEB000F7F76BF9AFF2444005F09CFA4FF4FA70C3
:10CEC000F7F763F97AA005F095FA4FF4FA70F7F7DF
:10CED0005CF97AA005F08EFA4FF4FA70F7F755F97D
:10CEE00079A005F087FA4FF4FA70F7F74EF90024AD
:10CEF00011E0681CC5B2F8F707FCAFF2F83005F096
:10CF000079FA4FF4FA70F7F740F9AFF2FC3135488F
:10CF100002F0DEFE04463C2D01DA012000E0002094
:10CF20000CB9012100E0002108400028E1D104B93A
:10CF30007CBD00240DE0F8F7E7FB66A005F05AFA87
:10CF40004FF4FA70F7F721F965A1264802F0C0FE08
:10CF500004463C2D01DA012000E000200CB901213B
:10CF600000E0002108400028E5D104B9E0E75EA117
:10CF70001C4802F0ADFE0446641C6078303821780D
:10CF8000303901EB810100EB4100584908602079FC
:10CF90003038E178303901EB810100EB4100544930
:10CFA0000860E0793038A179303901EB810100EB7C
:10CFB000410050490860A07A3038617A30399BE0EE
:10CFC0006F66002041542B514D545355423D302C37
:10CFD000312C2225732F636F6E666967222C320D08
:10CFE0000A0000008366002041542B514D545355D4
:10CFF000423D302C312C2225732F64617461222C28
:10D00000320D0A003D6300202564000041542B517D
:10D010004953454E443D302C25732C222573220D57
:10D020000A00000053454E44204F4B003C63002053
:10D0300041542B514D545055423D302C302C302C06
:10D04000302C2225732F636F6E666967222C25644E
:10D050000D0A000041542B514D545055423D302C87
:10D06000302C302C302C2225732F7461626C656853
:10D07000656164222C25640D0A00000041542B5187
:10D080004D545055423D302C302C302C302C222524
:10D09000732F64617461222C25640D0A0000000066
:10D0A0003E000000257300002B51495552430000FB
:10D0B00041542B43455245473F0D0A0041542B43F1
:10D0C00046554E3F0D0A000041542B5142414E44FB
:10D0D0003F0D0A0041542B43434C4B3F0D0A0000C7
:10D0E0002B43434C4B3A00002200000044630020D5
:10D0F000486300204C63002001EB810100EB4100FC
:10D1000015490860607B3038217B303901EB8101A3
:10D1100000EB410011490860207C3038E17B303958
:10D1200001EB810100EB41000D4908600D480068EA
:10D1300014280FDD0846006808490968CDE9001089
:10D1400005480368084802680848016805480068FF
:10D15000F9F7B5F900BFEBE65063002054630020F7
:10D1600058630020446300204C6300204863002083
:10D1700010B504462046F9F743FF10BD2DE9F041F4
:10D1800007460D46144698460026F9F7A0FFFCA175
:10D19000204602F09DFD20B13946FAA0FAF700F8CA
:10D1A00003E03946F8A0F9F7FBFF1DB914B90120D7
:10D1B000BDE8F0814046F6F7E8FF0A20F6F7E5FF04
:10D1C0000020F349B1F8C810C1F30E01F04A5054E1
:10D1D000DDB1D4B12946104602F07AFD08B1012034
:10D1E00000E0002040B92146E94802F071FD08B195
:10D1F000012000E0002008B1012000E000200646E8
:10D200000EB10120D4E70020D2E7D5B12946E0488D
:10D2100002F05EFD08B1012000E0002040B9214687
:10D22000DB4802F055FD08B1012000E0002008B104
:10D23000012000E0002006460EB10120B8E70020E2
:10D24000B6E72946D24802F043FD08B1012000E0CC
:10D25000002040B92146CE4802F03AFD08B1012035
:10D2600000E0002008B1012000E0002006460EB1D9
:10D2700001209DE700209BE710B500240EE040F65A
:10D28000B8330022C3A1C5A0FFF778FF08B100BFE3
:10D2900010BD601C84B26420F6F777FF642CEEDBCF
:10D2A00000BFF5E710B5044624B1012C0AD0022CCA
:10D2B00018D10FE040F6C413BBA2BDA1BDA0FFF77B
:10D2C0005DFF10BD40F6C413B7A2B9A1BCA0FFF723
:10D2D00055FFF6E740F6C413B3A2B5A1BBA0FFF714
:10D2E0004DFFEEE70020ECE730B59FB004460D4659
:10D2F0002B462246B8A101A805F08CF841F28833EC
:10D300000022ABA101A8FFF739FF1FB030BD10B557
:10D3100086B004460CB1012000E000200246B3A113
:10D3200001A805F077F84FF4FA730022A0A101A834
:10D33000FFF724FF06B010BD70B59AB005460E4643
:10D340001446642101A802F0B8FC15B1012D10D1DA
:10D3500007E03346A9A2AAA101A8009405F05AF853
:10D3600008E03346AAA2A6A101A8009405F052F84D
:10D3700000E000BF00BF42F210738BA28CA101A895
:10D38000FFF7FCFE1AB070BDF0B5B5B004460D460F
:10D3900016461F4664211CA802F08FFC642103A8D6
:10D3A00002F08BFC2B4622469AA103A8CDE9006728
:10D3B00005F030F803AB9BA29EA11CA805F02AF84B
:10D3C00041F2883300227AA11CA8FFF7D7FE10B9DA
:10D3D000002035B0F0BD0120FBE730B5B3B0044606
:10D3E0000D4664211AA802F068FC642101A802F02D
:10D3F00064FC23462A4691A101A805F00BF801AB75
:10D4000090A28CA11AA805F005F841F288330022F9
:10D4100067A11AA8FFF7B2FE10B9002033B030BDE3
:10D420000120FBE710B54FF4FA73002260A189A038
:10D43000FFF7A4FE08B9002010BD4FF4FA7389A2CB
:10D440005BA189A0FFF79AFEF6E72DE9F04186B0CF
:10D4500006460F4614461D464FF0000836B13946C1
:10D4600048A0F9F79DFE4FF001081AE0052D06DAF5
:10D4700023462A467FA101A804F0CCFF04E0A21CA9
:10D4800081A101A804F0C6FFC823002282A101A83F
:10D49000FFF774FEC8233AA280A13846FFF76EFE5C
:10D4A0008046404606B0BDE8F08110B54FF47A7072
:10D4B000F6F76BFE4FF4FA70F6F767FE10BD10B585
:10D4C0004FF4FA73002277A17AA0FFF757FE30B12C
:10D4D00074A12F4802F0FCFB08B1022010BD00200F
:10D4E000FCE7F0B503460D461646002729460A2EEE
:10D4F00003D0002008702846F0BD33B9302001F871
:10D50000010B002008702846F6E7002B03DA2D20D7
:10D5100001F8010B5B4242F210720DE093FBF2F452
:10D5200004B937B104F1300001F8010B04FB1233E8
:10D5300001270A2092FBF0F2002AEFDC002008709D
:10D540002846D9E70FB470B586B006460CA80190FE
:10D5500018E10B9800785C280FD10B98401C0B90B9
:10D5600000786E280AD0722809D10D213046F5F7CF
:10D5700028FD0B98401C0B90B0E0B0E0A2E0A9E0C1
:10D58000310000002573000025730D0A0000000023
:10D59000AC7C0020726561647900000041542B521C
:10D5A0004553544F524500004E554C4C000000006E
:10D5B0004F4B000041542B43574D4F44453D3100E4
:10D5C00041542B43574D4F44453D320041542B436A
:10D5D000574D4F44453D330041542B43574A41502A
:10D5E0003D222573222C22257322000041542B4317
:10D5F00049504D55583D25640000000054435000EB
:10D60000222573222C222573222C25730000000072
:10D6100055445000222573222C222573222C256488
:10D620002C25640041542B43575341505F444546D9
:10D630003D000000257325730000000025642C25A3
:10D640007300000041542B434950534552564552F4
:10D650003D00000041542B4349504D4F44453D315E
:10D66000000000003E00000041542B434950534548
:10D670004E44000041542B43495053454E443D25F0
:10D68000642C256C6400000041542B4349505345E1
:10D690004E443D256C6400003E20000053454E443E
:10D6A000204F4B002B4349505354415455533A306B
:10D6B0000000000041542B434950535441545553EA
:10D6C000000000000A213046F5F77BFC0B98401C57
:10D6D0000B9003E00B98401C0B9000BF4BE00B98A5
:10D6E0000078252840D10B98401C0B9000786428C6
:10D6F00018D0732833D1019810C801900BE021781D
:10D700003046F5F75EFC00BF80213046F5F709FD95
:10D710000028F9D0641C20780028F0D10B98401C18
:10D720000B9020E0019820C801900A2202A9284607
:10D73000FFF7D7FE02AC0BE021783046F5F741FC4D
:10D7400000BF80213046F5F7ECFC0028F9D0641CBE
:10D7500020780028F0D10B98401C0B9003E00B9828
:10D76000401C0B9000BF06E00B9810F8011B0B90BB
:10D770003046F5F726FC00BF80213046F5F7D1FC96
:10D780000028F9D00B98007800287FF4E2AE06B0AC
:10D7900070BC5DF814FB70B5A0B004460D4616468B
:10D7A0002B4622463EA102A8009604F033FE4FF419
:10D7B000FA730022AFF2082102A8FFF7DFFC20B0C5
:10D7C00070BD30B59FB004460D462B4622463FA1A2
:10D7D00001A804F01FFE4FF4FA730022AFF23021CB
:10D7E00001A8FFF7CBFC1FB030BD10B59EB00446BA
:10D7F00022463CA1684604F00DFE4FF4FA73002265
:10D80000AFF254216846FFF7B9FC1EB010BD30B529
:10D810009FB004460D462B46224637A101A804F0CE
:10D82000F9FD4FF47A730022AFF27C2101A8FFF7D3
:10D83000A5FC1FB030BD00B59FB036A101A804F013
:10D84000E9FD4FF4FA730022AFF29C2101A8FFF723
:10D8500095FC1FB000BD70B504460D460026294654
:10D860002046FFF7D4FF4FF47A70F6F78EFC0126BE
:10D87000304670BD10B5C8212A4802F01EFA29486A
:10D88000B0F8C80020F400402649A1F8C8000846B6
:10D89000B0F8C8006FF30E00A1F8C80010BD00007A
:10D8A00041542B4D515454555345524346473D30F6
:10D8B0002C312C222573222C222573222C22257315
:10D8C000222C302C302C22220000000041542B4D01
:10D8D000515454434F4E4E3D302C222573222C255B
:10D8E000642C300041542B4D5154545355423D301B
:10D8F0002C222573222C310041542B4D515454506D
:10D9000055423D302C222573222C222573222C31A6
:10D910002C30000041542B4D515454434C45414E42
:10D920003D300000AC7C00202DE9F04106460F465A
:10D93000154600244FF480514648F3F783F84FF41E
:10D940007A70F6F722FC4FF480514248F3F778F8EA
:10D950004FF47A70F6F719FCFFF78EFC00BF01E078
:10D96000601CC4B24FF4FA7300223BA13BA0FFF746
:10D9700005FC80F00100642C01DA012100E00021A7
:10D9800008400028ECD1002401E0601CC4B203234D
:10D99000052239463046FFF7F7FC80F00100642C81
:10D9A00001DA012100E0002108400028EDD1002427
:10D9B00001E0601CC4B20120FFF774FC80F001009C
:10D9C000642C01DA012100E0002108400028F0D198
:10D9D000002401E0601CC4B20120FFF798FC80F035
:10D9E00001000A2C01DA012100E000210840002892
:10D9F000F0D1002401E0601CC4B201212846FFF7E9
:10DA0000ECFC80F00100642C01DA012100E000212F
:10DA100008400028EFD100BFBDE8F08110B5002418
:10DA20004FF4E130FFF7A4FB0E4A02F10A01A1F125
:10DA30001E00FFF779FF0AE0601CC4B24FF47A7051
:10DA400003F032F8FFF73BFD022800D13D243C2CC7
:10DA5000F2DB10BD000002404F4B00004154453046
:10DA600000000000FB65002010B54FF48051FE4817
:10DA7000F2F7E6FF10BD10B54FF48051FA48F2F707
:10DA8000E1FF10BD2DE9F04F91B006460F46144658
:10DA90001D463046394602F0EEFB1090002801DBAF
:10DAA000109901E010994942084602F0BAFB8246FB
:10DAB00005F040FFED4AEE4BCDE90A0102F0C2FA53
:10DAC000EA4AEC4BCDE90E013046394602F0BAFA8B
:10DAD000824622462B4602F0B5FA22462B46CDE975
:10DAE0000A01E248E24902F0ADFA824622462B469C
:10DAF00002F0A8FA22462B46CDE906010020DE49B5
:10DB000002F0A0FA00224FF08043CDE90201304636
:10DB1000394602F097FA82460022D84B02F0EBF920
:10DB2000CDE90001DDE9022302F0E5F9CDE90401C8
:10DB3000DDE9062302F0DFF9CDE90801DDE90A237A
:10DB400002F0D9F9CDE90C01DDE90E2302F0D3F999
:10DB50008046894600224FF080433046394602F025
:10DB600071FAC74AC74BCDE9020102F06BFA82464F
:10DB700005F090FE0022C44BCDE9040102F062FAE8
:10DB80000022C24BCDE908013046394602F05AFA6C
:10DB90008246BB4ABB4B02F055FACDE9020105F0C3
:10DBA00079FE0022B84BCDE9040102F04BFACDE931
:10DBB0000601DDE9082302F09EF900224FF08043C0
:10DBC000CDE90A0102F03EFA0022AB4BCDE90C018F
:10DBD00002F0AAFA42464B46CDE90E0102F08BF95B
:10DBE000804689460022A44B2046294602F09CFA32
:10DBF0008246A34AA34B02F025FACDE9020105F0C3
:10DC000049FE0022A24BCDE9040102F01BFA9C4A16
:10DC10009C4BCDE908012046294602F013FACDE9D4
:10DC2000040105F037FE82460022974B02F00AFA03
:10DC3000CDE90601DDE9082302F05DF900224FF08D
:10DC40008043CDE90A0102F0FDF900228A4BCDE9BB
:10DC50000C0102F069FA42464B46CDE90E0102F092
:10DC60004AF980468946864A864B2046294602F074
:10DC7000E9F982460022874B02F056FACDE902010B
:10DC800005F008FE0022844BCDE9040102F0DAF928
:10DC90000022824BCDE908012046294602F044FAD1
:10DCA000774A784BCDE9020102F0CCF9824605F0C3
:10DCB000F1FD00227A4BCDE9040102F0C3F9CDE970
:10DCC0000601DDE9082302F016F900224FF0804337
:10DCD000CDE90A0102F0B6F90022674BCDE90C014B
:10DCE00002F022FA42464B46CDE90E0102F003F95A
:10DCF000804689464046494611B0BDE8F08F2DE97F
:10DD0000F04F8FB004460D4692469B46204629466A
:10DD100002F0B1FA0E90002801DB0E9901E00E9995
:10DD20004942084602F07DFACDE9080105F002FEFD
:10DD30004E4A504BCDE90A0102F084F94B4A4D4B53
:10DD4000CDE90C012046294602F07CF952465B469B
:10DD5000CDE9060102F076F9444A464BCDE90A01C5
:10DD60002046294602F06EF922462B46CDE90201F3
:10DD700002F068F952465B46CDE9060100204FF0FB
:10DD8000804102F05FF90022464BCDE902012046B6
:10DD9000294602F0B0F8CDE90001DDE9022302F0E6
:10DDA000AAF8CDE90401DDE9062302F0A4F8CDE9E3
:10DDB0000801DDE90A2302F09EF88046DDE90C2324
:10DDC00002F099F806460F4600224FF080432046A5
:10DDD000294602F037F98046294A2A4B02F032F9E7
:10DDE000CDE9000105F056FD0022274BCDE90201E7
:10DDF00002F028F90022254BCDE9060120462946EC
:10DE000002F020F980461E4A1E4B02F01BF9CDE9B4
:10DE1000000105F03FFD00221B4BCDE9020102F09D
:10DE200011F9CDE90401DDE9062302F064F80022CE
:10DE30004FF08043CDE9080102F004F900220E4BB7
:10DE4000CDE90A0102F070F932463B46CDE90C01FA
:10DE500002F051F806460F460022074B204629469D
:10DE600002F062F9064A1FE0000402409A9999996B
:10DE70009999C93F9999B93F00000840000059C0DD
:10DE8000182D4454FB210940000034400000184084
:10DE90000000444000003E40000074400000284064
:10DEA0000000644000C07240FE4BCDE9000102F06A
:10DEB000C9F8804605F0EEFC0022FB4BCDE90201DB
:10DEC00002F0C0F8F94AF74BCDE906012046294691
:10DED00002F0B8F8CDE9020105F0DCFC8046002232
:10DEE000F34B02F0AFF8CDE90401DDE9062302F0BF
:10DEF00002F800224FF08043CDE9080102F0A2F8B9
:10DF00000022EC4BCDE90A0102F00EF932463B4605
:10DF1000CDE90C0101F0EFFF06460F460022E64B6B
:10DF20002046294602F000F98046E04ADD4B02F027
:10DF300089F8CDE9000105F0ADFC0022DF4BCDE909
:10DF4000020102F07FF80022DD4BCDE906012046F8
:10DF5000294602F0E9F8D54AD24BCDE9000102F09A
:10DF600071F8804605F096FC0022D64BCDE90201FF
:10DF700002F068F8CDE90401DDE9062301F0BBFFFA
:10DF800000224FF08043CDE9080102F05BF8002247
:10DF9000C84BCDE90A0102F0C7F832463B46CDE94D
:10DFA0000C0101F0A8FF06460F46304639460FB077
:10DFB000BDE8F08F0FB42DE9F04F8FB0DDE91A45C1
:10DFC000DDE91C67C04AC14B3046394602F03AF8D9
:10DFD000CDE9020105F05EFCBD4ABE4BCDE904016E
:10DFE00002F030F832463B46CDE90801304639466A
:10DFF00002F028F822462B46CDE9020120462946A8
:10E0000002F020F8CDE90001DDE9022301F073FF01
:10E01000CDE9040105F08EFCCDE90601DDE9082318
:10E0200001F069FF80468946A74AA84B2046294649
:10E0300002F008F8CDE9020105F080FBA64AA74BE3
:10E04000CDE9040101F0FEFF22462B46CDE908018F
:10E050003046394605F0B2FACDE90601DDE908237C
:10E0600001F049FF82468B465046594605F066FB53
:10E0700042464B46CDE9060101F0E4FF984A994B30
:10E08000CDE9080101F037FFCDE90A0150465946B4
:10E0900005F000FC42464B46CDE9060101F0D2FFF7
:10E0A000914A924BCDE9080101F025FFCDE90C0121
:10E0B0000AA991E80E101898A0E80E100FB0BDE85C
:10E0C000F00F5DF814FB0FB42DE9F04F91B0DDE9CE
:10E0D0001E010022864BCDE9040101F0ADFFCDE920
:10E0E0000801DDE91C010022824BCDE9040101F0A9
:10E0F000A3FFCDE90601DDE90823FFF7C3FC0646CF
:10E100000F46DDE91E010022794BCDE9040101F043
:10E1100093FFCDE90801DDE91C010022754BCDE933
:10E12000040101F089FFCDE90601DDE90823FFF7CD
:10E13000E6FD80468946DDE91E0100226E4BCDE9F1
:10E14000060101F0F1FF594A564BCDE9080101F0F3
:10E1500079FFCDE90A01DDE90A0105F09BFB0446E0
:10E160000D4622462B466548654901F06BFF224665
:10E170002B46CDE9060101F065FF0022614BCDE998
:10E18000080101F05CFF04460D462046294605F0D3
:10E19000D1FB82468B4652465B462046294601F01B
:10E1A00051FF02460B46CDE902015748574901F09D
:10E1B000BBFF3E4A3B4BCDE9040101F043FF002287
:10E1C0004D4BCDE908013046394601F03BFFCDE922
:10E1D0000601DDE9082301F0A7FF06460F46DDE949
:10E1E0000A0105F0ABFA52465B46CDE902014FF059
:10E1F0008040474901F098FFCDE90001DDE90223A5
:10E2000001F020FF294A274BCDE9040101F01AFF54
:10E210000022394BCDE908014046494601F012FF82
:10E22000CDE90601DDE9082301F07EFF804689463D
:10E23000DDE91E0132463B46CDE9080101F05BFEF7
:10E24000CDE90E01DDE91C0142464B46CDE908014E
:10E2500001F051FECDE90C010CA991E80E101A98BD
:10E26000A0E80E1011B0BDE8F00F5DF814FB2DE929
:10E27000F04F89B08246274903C901F0FCFF83466D
:10E2800001F0CFFFCDE9000122480CC8009801F051
:10E29000D6FE0022204BCDE9020101F0D3FE8046DC
:10E2A00000223BE0FB21094000004440182D44546B
:10E2B000000034400000084000003E4000C07240B2
:10E2C0000000284000C062404E04C777102E4A402C
:10E2D000F168E388B5F8F43E54E41071732AC93E3E
:10E2E00039B4C876BE9F7A3FFA7E6ABC7493783F91
:10E2F0000080414000405A40008066400BEF80AFF4
:10E300008F6A7B3F0000F03FC155E32D102B584131
:10E31000C15458416063002000005940FE4B01F099
:10E3200003FF04460D46FD4903C901F0A4FF8046E2
:10E3300001F077FF064622462B4601F0DCFDCDE9D1
:10E340000601F74903C901F096FF834601F069FF12
:10E35000CDE90001F2480CC8009801F070FE0022DF
:10E36000F04BCDE9020101F06DFE06460022EA4BBA
:10E3700001F0DAFE04460D46E94903C901F07BFFCE
:10E38000064601F04EFF804622462B4601F0B3FDC3
:10E39000CDE9040104A80FC88AE80F0009B0BDE860
:10E3A000F08F2DE9F04F8BB08246DC4903C901F0B4
:10E3B00062FF834601F035FFCDE90201D7480CC862
:10E3C000029801F03CFE0022D64BCDE9040101F099
:10E3D00039FE06460022D04B01F0A6FE04460D464B
:10E3E000CE4903C901F047FF064601F01AFF8046F7
:10E3F00022462B4601F07FFDCDE90801C84903C93B
:10E4000001F039FF834601F00CFFCDE90201C44859
:10E410000CC8029801F013FE0022C24BCDE90401A2
:10E4200001F010FE80460022BB4B01F07DFE044649
:10E430000D46BB4903C901F01EFF804601F0F1FE05
:10E44000064622462B4601F056FDCDE90601DDE9E0
:10E450000801CDE9000102A8DDE90623FFF733FE3C
:10E4600002A80FC806AD0FC506A80FC88AE80F009E
:10E470000BB0BDE8F08F2DE9F04F8BB08246A74975
:10E4800003C901F0F8FE834601F0CBFECDE902019D
:10E49000A2480CC8029801F0D2FD0022A14BCDE9A0
:10E4A000040101F0CFFD064600229B4B01F03CFE2B
:10E4B00004460D46994903C901F0DDFE064601F008
:10E4C000B0FE804622462B4601F015FDCDE908013D
:10E4D000934903C901F0CFFE834601F0A2FECDE9C6
:10E4E00002018F480CC8029801F0A9FD00228D4B53
:10E4F000CDE9040101F0A6FD80460022864B01F023
:10E5000013FE04460D46864903C901F0B4FE804659
:10E5100001F087FE064622462B4601F0ECFCCDE9D1
:10E520000601DDE90801CDE9000102A8DDE90623C5
:10E53000FFF7C9FD02A80FC806AD0FC5DDE9080148
:10E54000CDE9000102A8DDE90623FFF733FD02A8AB
:10E550000FC806AD0FC506A80FC88AE80F000BB09C
:10E56000BDE8F08F704710B54F216F4801F0A5FB53
:10E5700000206D4981F8A00081F8A10001F1A200FE
:10E58000002101604160018181720B3001604160B6
:10E59000018181720B300180817075388167C1679C
:10E5A000C0F8801084300180817000205E4981F8BD
:10E5B000CA0010BD2DE9F04FA1B000265A4890F8CE
:10E5C000A000002874D00020574981F8A00000BFA7
:10E5D000E4E12EB955A1544801F07AFB0446DBE191
:10E5E000641C52A1204601F073FB051E6AD00A2E5E
:10E5F00042D2DFE806F041050C121920272E343AEA
:10E600002A1B21464848A23001F03EFB35E02A1B78
:10E6100021461DA801F038FB2FE02A1B2146424865
:10E62000AD3001F031FB28E02A1B21463E48B830CE
:10E6300001F02AFB21E02A1B21463B48BB3001F0B8
:10E6400023FB1AE02A1B21463748C73001F01CFB88
:10E6500013E02A1B21461AA801F016FB0DE02A1B25
:10E66000214617A801F010FB07E02A1B21462E487F
:10E67000CB3001F009FB00E000BF00BF2C460120B9
:10E68000294981F8A1009DF87400412801D1012099
:10E6900000E00020244991F8CB1009B1012100E0ED
:10E6A0000021084028B101201F4981F8CA0008E074
:10E6B00077E19DF87400562803D100201A4981F8AB
:10E6C000CA0000BF184991F8B510A1F1300001F05F
:10E6D000A8FD07460022164B01F0B4FCCDE91C0151
:10E6E000114991F8B410A1F1300001F09AFD0746EC
:10E6F0000022104B01F0A6FCCDE918010A4991F85F
:10E70000B310A1F1300001F08CFD07460022054B4B
:10E7100001F098FC10E0000000004E406063002013
:10E720006863002000005940767D00202C00000026
:10E730000000F03F00002440CDE91401F84991F8B1
:10E74000B210A1F1300001F06CFD07460022F54B3C
:10E7500001F078FCCDE91001F14991F8B010A1F178
:10E76000300001F05EFD07460022EF4B01F06AFC2D
:10E77000CDE90C01EA4991F8AF10A1F1300001F0A8
:10E7800050FD07460022E94B01F05CFCCDE9080191
:10E79000E34991F8AE10A1F1300001F042FD0746C7
:10E7A0000022E34B01F04EFC82468B46DC4991F897
:10E7B000AD10A1F1300001F034FD07460022DD4B21
:10E7C00001F040FC52465B46CDE9040101F093FBA9
:10E7D000CDE90601DDE9082301F08DFBCDE90A0151
:10E7E000DDE90C2301F087FBCDE90E01DDE9102303
:10E7F00001F081FBCDE91201DDE9142301F07BFB7F
:10E80000CDE91601DDE9182301F075FBCDE91A0108
:10E81000DDE91C2301F06FFBC74A03C2C04991F830
:10E82000C410A1F1300001F0FCFC07460022C34BEC
:10E8300001F008FCCDE91C01B94991F8C310A1F120
:10E84000300001F0EEFC07460022BD4B01F0FAFB60
:10E85000CDE91801B24991F8C210A1F1300001F0E0
:10E86000E0FC07460022B74B01F0ECFBCDE91401B8
:10E87000AB4991F8C110A1F1300001F0D2FC07467C
:10E880000022A84B01F0DEFBCDE91001A44991F86C
:10E89000BF10A1F1300001F0C4FC07460022A24BDA
:10E8A00001F0D0FBCDE90C019D4991F8BE10A1F11A
:10E8B000300001F0B6FC074600229C4B01F0C2FB81
:10E8C000CDE90801964991F8BD10A1F1300001F0A1
:10E8D000A8FC07460022964B01F0B4FBCDE90401E9
:10E8E0008F4991F8BC10A1F1300001F09AFC074665
:10E8F0000022904B01F0A6FB82468B46884991F896
:10E90000BB10A1F1300001F08CFC074600228E4BB9
:10E9100001F098FB52465B46CDE9000101F0EBFAAD
:10E92000CDE90201DDE9042301F0E5FACDE90601B4
:10E93000DDE9082301F0DFFACDE90A01DDE90C2366
:10E9400001F0D9FACDE90E01DDE9102301F0D3FA87
:10E95000CDE91201DDE9142301F0CDFACDE916016C
:10E96000DDE9182301F0C7FACDE91A01DDE91C231E
:10E9700001F0C1FA754A03C200226D4B6E4903C90A
:10E9800001F0D2FB6C4A03C20022694B6F4903C9F4
:10E9900001F0CAFB6D4A03C2701CC6B2092E7FF794
:10E9A00018AE00201E901F9020905D4890F8CF0078
:10E9B0008DF878005A4890F8D0008DF879002D2015
:10E9C0008DF87A00564890F8CD008DF87B005448B9
:10E9D00090F8CE008DF87C002D208DF87D005048F9
:10E9E00090F8CB008DF87E004D4890F8CC008DF863
:10E9F0007F001EA801F088F907463A461EA948483C
:10EA0000CB3001F041F900201E901F902090444827
:10EA100090F8A3003038424991F8A210303901EB48
:10EA2000810100EB4100083000F0FF090A2099FB4A
:10EA3000F0F030303A4981F8A2000A2099FBF0F159
:10EA400000FB11903030C1B2354880F8A31090F827
:10EA5000A2008DF87800324890F8A3008DF8790074
:10EA60003A208DF87A002E4890F8A4008DF87B00AB
:10EA70002B4890F8A5008DF87C003A208DF87D0099
:10EA8000274890F8A6008DF87E00254890F8A7004A
:10EA90008DF87F002248A230002101604160018191
:10EAA00081721EA801F030F907463A461EA91C489B
:10EAB000A23001F0E9F800201E901F90209021B0B4
:10EAC000BDE8F08F10B50024154890F8A10000288B
:10EAD0007ED000BF0020124981F8A1001CA003F0E5
:10EAE00089FC06E00E48A230015D1FA003F082FC05
:10EAF000641C0B48A230005D0028F3D11BA003F07A
:10EB000079FC074890F8CA0000287DD0002004490D
:10EB100081F8CA00002416A003F06CFC3BE0000062
:10EB2000767D002000408F400088C340006AF84096
:10EB300080842E41D0126341606300200000F03FCA
:10EB4000000024400000594084D7974168630020AA
:10EB5000536176655F446174612E55544354696D09
:10EB600065203D2000000000256300000D0A000024
:10EB7000536176655F446174612E6C61746974756C
:10EB80006465203D200000005448015DAFF228007C
:10EB900003F030FC641C5148005D0028F4D1AFF252
:10EBA000340003F027FC00244DA003F023FC4B4865
:10EBB000AD3890F8B810AFF2500003F01BFC474896
:10EBC000AD3890F8B910AFF2600003F013FC00E02C
:10EBD00036E0AFF2680003F00DFC00BF45A003F083
:10EBE00009FC07E03D480E30015DAFF2840003F000
:10EBF00001FC641C39480E30005D0028F2D1AFF2F0
:10EC0000940003F0F7FB00E017E040A003F0F2FBF4
:10EC10003248AD3890F8C710AFF2B40003F0EAFB09
:10EC20002E48AD3890F8C810AFF2C40003F0E2FBF4
:10EC3000AFF2C80003F0DEFB02E039A003F0DAFB1C
:10EC400010BD70B58EB0002400202449AD3981F884
:10EC5000D60035E04FF47A70F5F797FA1F48AD38D3
:10EC600090F8A00008B1FFF7A5FC601CC4B21B48D7
:10EC7000AD3890F8CA00F8B106A8FFF7F8FA06A870
:10EC80000FC80AAD0FC53D242C2114481A30CDE918
:10EC900006100891DDE90A01CDE904012C210F4895
:10ECA0000B30CDE900100291DDE90C532A4623A177
:10ECB000284803F0AFFB03E027A1264803F0AAFB96
:10ECC000322CC7DBFFF74FFC2748F4F787F8012009
:10ECD0000249AD3981F8D6000EB070BD237E002008
:10ECE000536176655F446174612E4E5F53203D2011
:10ECF00000000000536176655F446174612E6C6FA3
:10ED00006E676974756465203D2000005361766507
:10ED10005F446174612E455F57203D200000000074
:10ED20004750532044415441206973206E6F742032
:10ED300075736566756C6C210D0A0000252E3766AB
:10ED4000256325732563252E376625632573256383
:10ED5000000000005C7100204E612C4E612C4E6161
:10ED60002C4E612C00000000003801401CB5FE480C
:10ED7000F4F734F801210220F2F7C4F8C020009023
:10ED800001208DF8040002208DF8050000208DF888
:10ED9000060001208DF807006946F448F1F7D6FD1A
:10EDA0004021F248F1F74EFE1CBD1CB501210420A4
:10EDB000F2F7A8F80E20009001208DF80400022040
:10EDC0008DF8050000208DF8060001208DF8070061
:10EDD0006946E748F1F7BAFD0221E548F1F732FE4E
:10EDE0000421E348F1F72EFE0821E148F1F72AFE5D
:10EDF0001CBD10B50446072C53D2DFE804F05204C2
:10EE0000111E2B3845000821D948F1F71BFE0421BB
:10EE1000D748F1F717FE0221D548F1F713FE4DE070
:10EE20000821D348F1F70EFE0421D148F1F70AFE7C
:10EE30000221CF48F1F704FE40E00821CC48F1F769
:10EE400001FE0421CA48F1F7FBFD0221C848F1F791
:10EE5000F9FD33E00821C648F1F7F4FD0421C44868
:10EE6000F1F7EEFD0221C248F1F7EAFD26E00821A4
:10EE7000BF48F1F7E5FD0421BD48F1F7E3FD0221AC
:10EE8000BB48F1F7DFFD19E00821B948F1F7D8FDDB
:10EE90000421B748F1F7D6FD0221B548F1F7D0FDBE
:10EEA0000CE00821B248F1F7CBFD0421B048F1F79E
:10EEB000C7FD0221AE48F1F7C3FD00BF00BF10BD82
:10EEC00010B54FF49660F7F7FDFF10BD10B5202187
:10EED000A648F1F7B5FD4021A448F1F7B3FD142091
:10EEE000F5F753F94021A148F1F7AAFD10BD70B51F
:10EEF00002460B46FF24FF250BE012F8010B80EAC7
:10EF000005019C4830F8110080EA04059A4830F861
:10EF10001140181EA3F10106B3B2EED145EA042058
:10EF200080B270BD2DE9F04F8FB0044600200490F0
:10EF300082468346039002908146904981F83401CD
:10EF400009218F48FFF7D3FF82460AF0FF008C4962
:10EF5000497A88427DD18A48807AB0EB1A2FF9D15C
:10EF600000200B900C900D90089009900A9005904D
:10EF700006900790824890F80390007900EB0920F2
:10EF80000FFA80F9484601F04CF900227D4BCDE99B
:10EF9000000101F057F8074600227B4B01F0C4F84E
:10EFA000054601F09AF98346584601F083F9054673
:10EFB0002A460B4675A105A803F02CFA704890F874
:10EFC0000590807900EB09200FFA80F9484601F09E
:10EFD00028F900226B4BCDE9000101F033F805461A
:10EFE0000022694B01F0A0F8074601F076F9039082
:10EFF000039801F05FF905462A460B4663A10BA86A
:10F0000003F008FA5E4890F80790007A00EB0920B8
:10F010000FFA80F9484601F0F6F80290029801F0E4
:10F0200049F905462A460B465AA108A803F0F2F909
:10F03000072C41D2DFE804F040040E18222C3600E1
:10F0400008A80BAB05AA55A100904C4803F0E2F9C3
:10F0500033E038E008A80BAB05AA50A10090474860
:10F060001E3003F0D7F928E008A80BAB05AA4BA186
:10F07000009042483C3003F0CDF91EE008A80BABED
:10F0800005AA46A100903D485A3003F0C3F914E0A8
:10F0900008A80BAB05AA41A100903848783003F0CE
:10F0A000B9F90AE008A80BAB05AA3CA100903348C7
:10F0B000963003F0AFF900E000BF00BF01202F49F8
:10F0C00081F834012CE0072C28D2DFE804F0270473
:10F0D000090F151B210034A1284803F09BF91EE0FD
:10F0E00031A126481E3003F095F918E02EA12348DF
:10F0F0003C3003F08FF912E02BA120485A3003F086
:10F1000089F90CE028A11D48783003F083F906E066
:10F1100025A11A48963003F07DF900E000BF00BF3A
:10F120000FB0BDE8F08F1CB50024002000900190C6
:10F13000F7F726FF012479E04FF4FA70F5F725F888
:10F140000020009001901BA300221BA1684603F041
:10F1500061F9FFF70BFEFFF7B9FEFFF7B1FE694655
:10F1600017A0F7F71CFF2DE0003801400004024013
:10F170000008024004400208044202084D7E0020BC
:10F18000D06C00200000F03F00002440252E3166A6
:10F1900000000000252E30660000000025732C259D
:10F1A000732C2573000000004E612C4E612C4E61C3
:10F1B000000000004D2100002564257300000000C0
:10F1C000257300000A20F4F7E0FF2021FE48F1F744
:10F1D00039FC4FF41670F4F7D8FFF7F7D1FE002092
:10F1E00000900190F9A30022AFF23401684603F0C9
:10F1F00011F9F7F7C5FEFFF7B9FDFFF767FEFFF757
:10F200005FFE6946AFF24800F7F7C9FE0A20F4F73F
:10F21000BCFF2021EC48F1F715FC4FF41670F4F711
:10F22000B4FF2046FFF77EFE601CC4B2072C83DBD0
:10F230001CBD10B54FF0FF31E548006801F08AFDB4
:10F240000120FFF7D6FDF5F77AF80020E1490870B4
:10F25000FFF78CFDF7F794FEFFF738FEFFF730FE5F
:10F26000DDA1AFF2A400F7F79AFE0820F4F78DFFB6
:10F270002021D548F1F7E6FB4FF4FA70F4F785FF4B
:10F28000D348006801F08AFDD4A1D54800F020FDE4
:10F29000041E02D0641E207810BD7F20FCE73EB51E
:10F2A00004460D4600200090019002900120FFF7D7
:10F2B000A0FDCCA2AFF2F801684603F0ABF8F5F779
:10F2C0003EF80020C3490870FFF750FDF7F758FEDD
:10F2D000FFF7FCFDFFF7F4FD6946AFF21C10F7F7EE
:10F2E0005EFE0820F4F751FF2021B748F1F7AAFB92
:10F2F0004FF4FA70F4F749FF3EBD7CB50446002098
:10F3000000900190F7F73CFE002000900190AFA321
:10F310002246B6A1684603F07DF8F7F731FEFFF705
:10F3200025FDFFF7D3FDFFF7CBFD6946AFF2701067
:10F33000F7F735FE0820F4F728FF2021A248F1F75F
:10F3400081FB4FF4FA70F4F720FFAAA1A44800F063
:10F35000BFFC0546A8A1A24800F0BAFC06460DB1C4
:10F36000012000E000200EB1012100E0002108434F
:10F3700008B100207CBD0120FCE701460A46106868
:10F38000704710B51E219D4800F097FC1E219B4838
:10F390001E3000F092FC1E2198483C3000F08DFC9D
:10F3A0001E2196485A3000F088FC1E219348783080
:10F3B00000F083FC1E219148963000F07EFC8021F5
:10F3C0008E48B43000F079FC10BDFEB5074600242D
:10F3D000002500200090019002906421884800F0F0
:10F3E0006CFC4FF480718748F1F72CFB0A20F4F78E
:10F3F000CCFEFE222146641C0DF801200622214687
:10F40000641C0DF8012000222146641C0DF8012027
:10F4100030222146641C0DF8012000222146641C84
:10F420000DF8012002222146641C0DF8012006215E
:10F430006846FFF75CFD0646F2B22146641C0DF8F3
:10F440000120320A2046611CCCB20DF8002000BF1A
:10F450000DE000BF40216C48F3F763FE0028F9D0AF
:10F460001DF805106848F3F7ACFD681CC5B2082DFF
:10F47000EFDB0A20F4F789FE4FF480716148F1F761
:10F48000DFFA4FF47A70F4F780FE4FF480715D4834
:10F49000F1F7D8FA0A20F4F778FE002458480278E9
:10F4A0002146641C0DF8012006222146641C0DF83B
:10F4B000012000222146641C0DF801203022214643
:10F4C000641C0DF8012000222146641C0DF8012067
:10F4D0002146641C0DF8017006216846FFF707FD00
:10F4E0000646F2B22146641C0DF80120320A20467D
:10F4F000611CCCB20DF8002000250DE000BF4021BA
:10F500004148F3F70EFE0028F9D01DF805103E48DB
:10F51000F3F757FD681CC5B2082DEFDB0A20F4F79E
:10F5200034FE4FF480713748F1F78AFA4FF47A705D
:10F53000F4F72BFE00BFFEBDFEB5064600240025F5
:10F5400000200090019002902D48B0F864006FF305
:10F550000E002B49A1F864006421294800F0ADFB9E
:10F560004FF480712748F1F76DFA0A20F4F70DFE89
:10F570002146641C0DF8016003222146641C0DF82D
:10F58000012000222146641C0DF801202146641C44
:10F590000DF801202146641C0DF8012003222146AC
:10F5A000641C0DF8012006216846FFF7A0FC074601
:10F5B000FAB22146641C0DF801203A0A2046611C6B
:10F5C000CCB20DF8002021E00004024044302100BC
:10F5D000D06200206D6200203F2100000D0A000073
:10F5E000A36900203341302100000000256325730A
:10F5F000000000002B0000002D0000004D7E0020C8
:10F60000D06C0020000002400050004000BF0DE020
:10F6100000BF4021C348F3F784FD0028F9D01DF84E
:10F620000510C048F3F7CDFC681CC5B2082DEFDB10
:10F630000A20F4F7AAFD4FF48071BB48F1F700FAF5
:10F640004FF47A70F4F7A1FD00BFFEBD30B502465D
:10F650000B464FF6FF70002112E0545C604000241E
:10F660000AE000F0010525B140104AF201056840AA
:10F6700000E04010651CECB2082CF2DB4C1CA1B27F
:10F680009942EADB30BD2DE9FE4380460D46164621
:10F69000002400270020009001900290A348B0F8B9
:10F6A00064006FF30E00A149A1F8640064219F4833
:10F6B00000F003FB4FF480719B48F1F7C3F90A2077
:10F6C000F4F763FD2146641C0DF8018004222146F5
:10F6D000641C0DF801202A0A2146641C0DF8012043
:10F6E000EAB22146641C0DF80120320A2146641C4E
:10F6F0000DF80120F2B22146641C0DF8012006210C
:10F700006846FFF7A3FF814609F0FF022146641C0B
:10F710000DF801204FEA19222046611CCCB20DF8E9
:10F72000002000BF0DE000BF40217E48F3F7F9FC48
:10F730000028F9D01DF807107A48F3F742FC781C2E
:10F74000C7B2082FEFDB00BF40217648F3F7E9FC92
:10F750000028F9D04FF480717348F1F771F900BFB8
:10F76000BDE8FE832DE9F04F85B005460F46914672
:10F770002878012804D06FF0030005B0BDE8F08FB1
:10F78000B81E81B22846FFF761FF8046B81E295C8B
:10F7900008F0FF00814204D1781E285CB0EB182FDE
:10F7A00002D04FF0FF30E8E76878042802D06FF00D
:10F7B0000100E2E7AE78F11706EB91718910A6EB34
:10F7C000810111B16FF00200D7E7002434E0E01CA2
:10F7D000285C0106201D285C41EA0041601D285C70
:10F7E00041EA0020A11D695C08430490DDF810A0E7
:10F7F000504600F027FD8346584600F004FD514670
:10F80000009000F005FB4A49019000F004FB0290D3
:10F8100000F018FD03902046E11704EB9171891068
:10F8200049F831B0E21704EB9272921009EBC20270
:10F8300003995160201DC4B2B442C8DB00209CE78C
:10F840002DE9F043D7B000240E2200210120FFF75C
:10F850001AFF6420F4F799FC3448B0F86400C0F350
:10F860000E042246314917A800F00EFA09AA2146D3
:10F8700017A8FFF777FF054635B12EA1334802F0F0
:10F88000C9FD57B0BDE8F0830A21109890FBF1F64E
:10F8900064210E9890FBF1F70C9890FBF1F80A9810
:10F8A00090FBF1F9119A13991598CDE90562CDE90C
:10F8B00007100D990F98CDE90181CDE903700B98E0
:10F8C00000904B4622A12148099A02F0A3FD00BFF7
:10F8D000D7E710B501244FF4FA70F4F756FCE102B3
:10F8E0001148F1F7ADF84FF47A70F4F74EFCFFF7DA
:10F8F00048FDFFF7A5FF00BF07E02046FFF71CFE0D
:10F900002046FFF70FFB601CC4B2072CF5DB4FF459
:10F9100000610548F1F796F84FF47A70F4F735FC7A
:10F9200010BD00000050004000000240D06C0020DC
:10F9300000007A444E612C4E612C4E612C4E612C9D
:10F940004E612C4E612C4E6100000000017F0020B2
:10F9500025642E253031642C25642E253031642C0D
:10F9600025642E253031642C25642E253032642CFC
:10F9700025642C25642C256400000000014601F05C
:10F980000F00091101F00F0101EB81025100421833
:10F99000D0B2704730B501460A2491FBF4F4E2B2CC
:10F9A0000A2491FBF4F504FB1514E3B203EB0214F3
:10F9B000E0B230BD70B505460C46F8F793FA052065
:10F9C000F4F7D1FBD020F8F75EFBF8F7E0FA05205A
:10F9D000F4F7C9FB2846F8F756FBF8F7D8FA0520E4
:10F9E000F4F7C1FB2046F8F74EFBF8F7D0FA0520F4
:10F9F000F4F7B9FBF8F7A2FA70BD70B5044600251C
:10FA0000F8F770FAD020F8F73EFBF8F7C0FA0520B7
:10FA1000F4F7A9FB2046F8F736FBF8F7B8FA05200B
:10FA2000F4F7A1FBF8F75EFAD120F8F72CFBF8F712
:10FA3000AEFA0520F4F797FB0020F8F75EFB0546C9
:10FA4000F8F77CFA284670BD10B5F8F72FFA402178
:10FA50000E20FFF7AFFF0220F4F797FB00210F20E5
:10FA6000FFF7A8FF0220F4F790FB10BD10B50620A9
:10FA7000FFF7C3FF554948600520FFF7BEFF534914
:10FA800008720420FFF7B9FF504948720220FFF7BF
:10FA9000B4FF4E4908700120FFF7AFFF4B49487093
:10FAA0000020FFF7AAFF4949887010BD2DE9F047F3
:10FAB00007460C4615461E46DDE908894FF0000A48
:10FAC0003846FFF767FF00F0FF0A51460620FFF7B0
:10FAD00071FF4FF0000A2046FFF75CFF00F0FF0ABD
:10FAE00051460520FFF766FF4FF0000A2846FFF752
:10FAF00051FF00F0FF0A51460420FFF75BFF4FF073
:10FB0000000A3046FFF746FF00F0FF0A5146022088
:10FB1000FFF750FF4FF0000A4046FFF73BFF00F0B1
:10FB2000FF0A51460120FFF745FF4FF0000A484603
:10FB3000FFF730FF00F0FF0A51460020FFF73AFFC1
:10FB4000BDE8F08710B50620FFF757FF1F49486052
:10FB50000879FFF713FF1D4948600520FFF74DFFA7
:10FB60001A490872087AFFF709FF18490872042039
:10FB7000FFF743FF15494872487AFFF7FFFE134924
:10FB800048720220FFF739FF1049087008460078D4
:10FB900000F03F0008700878FFF7F0FE0B4908708E
:10FBA0000120FFF72AFF094948704878FFF7E6FE71
:10FBB000064948700020FFF720FF044988708878C4
:10FBC000FFF7DCFE0149887010BD0000847F002033
:10FBD00000BFFEE7062809D2DFE800F008030405AD
:10FBE000060704E003E002E001E000E000BF00BF20
:10FBF00000BFFEE71EF0040F0CBFEFF30880EFF329
:10FC00000980816911F8021CD9B901B590E80F107B
:10FC1000E047BDE800508CE80300194B93E806006C
:10FC2000914208BF704719B12CE9F00FC1F838C0F4
:10FC30001A60906BB0E8F00F80F309886FF0020E45
:10FC40007047104A13689942FAD801B552F821C09A
:10FC50000FC8E047BDE80050CCF800007047000036
:10FC600001B501F03FFABDE80140EFF3098CD4E79C
:10FC700001B501F093FCBDE80140EFF3098CCCE73E
:10FC8000946300206444020840EA01039B0703D008
:10FC900009E008C9121F08C0042AFAD203E011F8CB
:10FCA000013B00F8013B521EF9D27047D2B201E08D
:10FCB00000F8012B491EFBD270470022F6E710B571
:10FCC00013460A4604461946FFF7F0FF204610BDCA
:10FCD00030B505462A460B4612F8010B13F8014BC6
:10FCE00008B1A042F8D01CB1002802D06D1CF1E789
:10FCF000284630BDCAB2401E10F8011F8A4202D009
:10FD00000029F9D100207047421C10F8011B00297E
:10FD1000FBD1801A704710B5002200E0521C835CB2
:10FD20008C5CA34201D1002BF8D1D8B2E1B2401AC9
:10FD300010BD30B504460020034600E05B1C934232
:10FD400003D2E05CCD5C401BF8D030BD70B50646F8
:10FD500002F09AFB046805460A220021304600F0B2
:10FD600050FB2C6070BDF0B480EA0102D40F420059
:10FD7000B2EB410F02D20246084611464A0042D079
:10FD8000C30DDDB2C1F3C752AD1A202D35DAC1F370
:10FD9000160141F4000204B15242C5F1200602FAF4
:10FDA00006F12A411044B3EBD05F23D0C4B1012D3A
:10FDB000A0EBC35009DCF0BC4FF0004202EAC35292
:10FDC000DBB200F5000000F05DBB400000F1807088
:10FDD00000EBC350A0F1807040EAD170490009E007
:10FDE000490841EAC071A0EBC35000F5000040088B
:10FDF00000EBC350F0BC00F03CBB6142012202EBBF
:10FE00004101001BF6E7F0BC704781F00041AAE712
:10FE100080F00040A7E780EA010210B502F000433D
:10FE2000400022D04A001FD0010E01EB1261C0F346
:10FE30005600C2F3560240F4000042F40002A0FB58
:10FE4000022000047F39140400D0401C50EA124004
:10FE500001D44000491EC2B20C0604EBD010401C75
:10FE60004008802A02D003E0002010BD20F00100ED
:10FE7000002900DA0020184310BD30B480EA0102E6
:10FE800002F0004530F0004221F0004013D090B164
:10FE9000C30DD40DC2F31601C0F31600E41A41F4E9
:10FEA000000140F400027D34914201D3641C00E063
:10FEB0004900002C02DA30BC002070474FF40000EB
:10FEC0000023914201D3891A034340084FEA4101BC
:10FED000F7D151B1914202D14FF0004105E002D279
:10FEE0004FF0010101E06FF0010103EBC450284421
:10FEF00030BC00F0BEBA2DE9FE4F804681EA030017
:10FF0000C00F0C46009021F0004123F00045B8EBF3
:10FF10000200A94105D24046214690461C460B46A8
:10FF2000024623F00040104347D0270DC7F30A00D4
:10FF3000C3F30A510290401A019040286BDAC3F3D0
:10FF4000130040F4801B0098924620B10023D2EBAE
:10FF5000030A63EB0B0B01985946C0F1400250466F
:10FF600000F01EFA06460D4650465946019A00F02A
:10FF700036FA10EB08006141002487EA115284EA46
:10FF8000E7731A4340D0009A62B3019A012A4FEAFC
:10FF9000075215DC001B61EB02014FF0004202EA40
:10FFA0000752CDE90042001C41F5801132462B4634
:10FFB00000F0A5FA03B0BDE8F08F40462146F9E70E
:10FFC000001B61EB0201001C41F5801300185B412E
:10FFD0002018A2F5001747EB030140EAD570B619C7
:10FFE0006D4111E06D084FEA360645EAC0754FEAEB
:10FFF0000752001B61EB0201001C41F5801149080A
:020000040802F0
:100000004FEA30000019514132462B4603B0BDE89B
:10001000F04F00F065BA0098012240000023D0EBB9
:10002000020263EBE073009821464FEAE074B8EBFC
:10003000000061EB0401E9E783F000435BE781F036
:10004000004158E72DE9FE4F81EA030404F0004423
:1000500021F0004100944FF0000B23F0004350EAE0
:1000600001045ED052EA03045BD0C3F30A54C1F327
:100070000A552C44A4F2F3340194A0FB0254C1F3BA
:10008000130141F48011C3F3130343F4801301FB04
:10009000024400FB034E840A970A44EA815447EA6B
:1000A0008357A4FB076802958D0A05FB07854FEA75
:1000B000932C04FB0C542705029D4FEA065847EA8F
:1000C0001637B5EB08056EEB070C870E920E47EA64
:1000D000811742EA8312A7FB0201B6EB0B0164EB26
:1000E00000042B0D43EA0C335E1844EB1C50DA4637
:1000F0005146E7FB0201C5F313044FEA0B3343EA11
:1001000014534FEA0432019C43EA0603A4F10C04A1
:100110000294009CCDE900B400F0F1F903B0BDE811
:10012000F08F00200146F9E72DE9F04D81EA030444
:1001300004F0004B21F0004514464FF0000A23F074
:10014000004150EA050220D054EA01021DD0C5F357
:100150000A570246C5F31303C1F31300C1F30A564D
:1001600040F4801543F48013A7EB0608101BD64615
:1001700008F2FD3873EB050002D308F1010801E035
:1001800092185B41B8F1000F03DA00200146BDE888
:10019000F08D00204FF48011064684460EE0171BB8
:1001A00073EB050705D3121B63EB050306434CEA0B
:1001B000010C49084FEA300092185B4150EA0107F0
:1001C000EDD152EA030012D082EA040083EA05016D
:1001D000084305D0101BAB4106D20122002306E0E4
:1001E00000224FF0004302E06FF0010253101AEBBF
:1001F00006004CEB085110EB0A0041EB0B01BDE887
:10020000F04D00F06DB9C10F80EAE0700844CA07F4
:100210009623002100F036B996230022114600F003
:1002200031B90EB5C10F80EAE0700844CA07002159
:1002300040F233438DE80E000A460B4600F05FF9AA
:1002400003B000BD00F0004220F00040C10DC0F33B
:10025000160040F400007F2901DA0020704796293B
:1002600003DCC1F19601C84001E096398840002ABC
:10027000F4D04042704770B5C1F30A5201F0004516
:100280000024C1F3130140F2FF3341F480119A427C
:1002900001DA002070BD40F233439A42A2F23342A9
:1002A00003DC524200F08BF800E090402C43F1D088
:1002B000404270BD00F0004230F000400AD0C10D55
:1002C00001F56071C0F3160042EA0151C20840070F
:1002D0001143704700200146704701F0004330B4DD
:1002E00021F0004150EA010206D00A0DA2F5607229
:1002F000C1F31301002A02DC30BC00207047440F18
:1003000044EAC104C100E01830BC00EBC25000F068
:10031000B0B830B50B46014600202022012409E088
:1003200021FA02F59D4205D303FA02F5491B04FAAE
:1003300002F52844151EA2F10102F1DC30BD2DE9C1
:10034000F05F0546002092469B4688460646814659
:1003500040241BE0284641464746224600F02FF83D
:1003600053465A46C01A914110D3114618462246A8
:1003700000F016F82D1A67EB01084F4622460120BF
:10038000002100F00DF817EB00094E41201EA4F1EA
:100390000104DFDC484631462A464346BDE8F09F6B
:1003A000202A04DB203A00FA02F100207047914035
:1003B000C2F1200320FA03F3194390407047202A2A
:1003C00004DB203A21FA02F00021704721FA02F3FF
:1003D000D040C2F120029140084319467047202ABC
:1003E00006DBCB17203A41FA02F043EAE07306E05D
:1003F00041FA02F3D040C2F120029140084319466D
:1004000070472DE9F04791460F4680460446002686
:1004100014F8015B2DB100F053F90068405DC0078E
:10042000F6D12B2D02D02D2D18D0641E4A46394608
:10043000204600F049F927B13968A14201D1C7F837
:10044000008071054FF002040BD54042002803DD07
:1004500002F01AF80460A007BDE8F08746F4806651
:10046000E4E70028F8DA02F00FF804606FF00040CB
:10047000F2E70029A8BF7047401C490008BF20F0E0
:100480000100704710B4B0FA80FC00FA0CF050EA9A
:10049000010404BF10BC704749B1CCF1200421FA1B
:1004A00004F411FA0CF118BF012121430843A3EB16
:1004B0000C01CB1D4FEA00614FEA102042BF002023
:1004C00010BC704700EBC35010440029A4BF10BCFF
:1004D0007047401C490008BF20F0010010BC704765
:1004E00010B5141E73F1000408DA401C41F100013C
:1004F00092185B411A4301D120F0010010BD2DE993
:10050000F04D92469B4611B1B1FA81F202E0B0FA89
:1005100080F220329046FFF743FF04460F4640EA40
:100520000A0041EA0B0153465A46084313D01146CC
:1005300053EA010019D0C8F140025046FFF73FFFCF
:1005400005460E46504659464246FFF729FF0843E6
:1005500005D0012004E020463946BDE8F08D00209A
:10056000054346EAE0762C4337430A986305E40ADC
:10057000A0EB08000022FD0A44EA47540A3002D5E5
:1005800000200146E9E7010510196941DDE9084548
:1005900000196941BDE8F04DA2E72DE9F04D0023B7
:1005A0001A461B1A8A4103DB00200146BDE8F08D84
:1005B000C1F30A52C1F3130141F480154FF0000B4F
:1005C000D10702D100186D41521E0027044640F2A7
:1005D000FF11384601EB620A3E4680460246002083
:1005E0004FF48011FFF7EBFEC2197141BB1846EBC7
:1005F0000100B4EB030C75EB000C04D3E41A65EBBB
:10060000000517460E46241908F101006D41804689
:100610003428E3DDF91946EB0600091BA84103D293
:100620004FF0FF32134601E0002213461BEB070098
:1006300046EB0A51BDE8F04DFFF752BFC1F30A5235
:10064000C1F3130140F2FF3341F480119A4202DA00
:1006500000200146704740F233439A42A2F23342EF
:1006600002DC5242FFF7ABBEFFF79ABE30B5041E64
:1006700071F1000404DB4FF00044404264EB0101DF
:10068000141E73F1000405DB1C464FF00043524278
:1006900063EB0403994208BF904230BD064C074DFE
:1006A00006E0E06840F0010394E807009847103442
:1006B000AC42F6D3EFF73AFDB44B0208D44B020834
:1006C00000487047AC4602082DE9F05F824600788A
:1006D000002715468B460AF10104B946302801D09F
:1006E0009DB113E014F8010B0127782803D0582896
:1006F00001D045B10AE00DB1102D07D1002710251A
:1007000014F8010B02E0082500E00A250026B04697
:100710000EE005FB080005FB06F1012701EB104682
:100720001FFA80F8B6F5803F00D3B94614F8010BE4
:10073000294600F03CF80028EBDABBF1000F05D0A9
:100740000FB1641E00E05446CBF80040B9F1000F31
:1007500006D001F099FE02210160C81EBDE8F09F9D
:1007600048EA0640FAE770B521F0004303430CD095
:10077000C1F30A550024D5EB040564EB0403D61736
:10078000AD1AB34102DB0020014670BD201841EBD9
:10079000025170BD0EB540F2334102910021CDE906
:1007A00000110A460B46FFF7AAFE03B000BD3A2827
:1007B00000D2303820F02002412A01D3A2F13700C4
:1007C000884201D34FF0FF30704770B58C1810F895
:1007D000015B15F0070301D110F8013B2A1106D186
:1007E00010F8012B03E010F8016B01F8016B5B1EA0
:1007F000F9D12B0705D40023521E0DD401F8013B7B
:10080000FAE710F8013BCB1A921C03E013F8015BE6
:1008100001F8015B521EF9D5A142D8D3002070BD6A
:1008200010B5930712D400F10C03D0071ED153E882
:10083000000F084203D1BFF32F8F002005E020EA0C
:10084000010243E8002404B1F1E710BDC06800EAEA
:1008500001038B42014618BF002112F0010208BFBC
:10086000014653EA020018BF084610BD53E8000FC6
:1008700000EA01028A4203D0BFF32F8F002005E077
:1008800020EA010243E8002404B1EFE710BD10B5EF
:1008900000F1280151E8002F12B9BFF32F8F04E0B7
:1008A000531E41E8003404B1F4E772B12C30012149
:1008B000006850B1821CD2E84F3FC2E8441F04B127
:1008C000F9E71A0602D00830F2E7002010BD70B533
:1008D000024652F8305F4DB1CC7800235DB12E4610
:1008E000ED78A5420DD275683346F7E70023C1E9DC
:1008F0000133C1620DE00024C1E9014300F12C0481
:1009000003E0C1E9016306F108042160002B18BF70
:100910001A1D1160283050E8001F4A1C40E80023CF
:1009200003B1F8E770BDD1E90123002A0EBFC3620D
:1009300093608B68191D002B08BF00F130010A601D
:100940007047000001480068704700BF10E000E0F9
:1009500007480178012905D106494FF080620A60F5
:10096000002101700448016841F0010101607047F5
:10097000907F002004ED00E010E000E04FF0FF3039
:100980007047000040B10B490968B1FBF0F0411E0F
:100990000020B0EB116F02D04FF0FF307047064AD5
:1009A000FF231370054A0623136051600449087041
:1009B00090607047D862002023ED00E010E000E076
:1009C000907F0020B0B500F10C01C289D1E85F3FF3
:1009D0009A4202D8BFF32F8F04E05C1CC1E8554F48
:1009E00005B1F3E7C28999B20020914238BF0120D6
:1009F000B0BD10B5930712D400F12803D0071ED163
:100A000053E8000F084203D1BFF32F8F002005E009
:100A100020EA010243E8002404B1F1E710BD806A36
:100A200000EA01038B42014618BF002112F00102C7
:100A300008BF014653EA020018BF084610BD53E83C
:100A4000000F00EA01028A4203D0BFF32F8F00207B
:100A500005E020EA010243E8002404B1EFE710BDFD
:100A6000B0B5104A0023443215462C683CB12569C4
:100A7000A94209D3491B04F10C052346F5E70024DC
:100A8000C0E90234016106E0C0E902340161A060FE
:100A90002569691A2161002B18BF03F10C0210604F
:100AA000B0BD00BF80630020EFF3058129B9EFF3EB
:100AB000108111B9EFF3118111B16FF0050070478A
:100AC000DFF804C000DF7047D9170208EFF3058292
:100AD0002AB9EFF3108212B9EFF311820AB100F0D4
:100AE00085BEDFF808C000DF704700BFED170208C1
:100AF000EFF3058129B9EFF3108111B9EFF31181FB
:100B000039B120B10178F32904BFC06870470020D3
:100B10007047DFF808C000DF704700BF1B180208ED
:100B2000EFF3058129B9EFF3108111B9EFF31181CA
:100B300009B100207047DFF808C000DF704700BF30
:100B40002D180208B0B5EFF305822AB9EFF3108231
:100B500012B9EFF31182AAB16FF0030480B100293A
:100B60000ED40278F32A0BD100F10C0252E8003FB8
:100B700043EA010442E8004505B1F7E700F0F8FA5E
:100B80002046B0BDDFF804C000DFB0BD99180208F0
:100B900010B5EFF305842CB9EFF3108414B9EFF31B
:100BA00011848CB16FF0030460B100290AD44BB9F1
:100BB0000378F32B06D1FFF733FE0446002808BF65
:100BC0006FF00204204610BDDFF804C000DF10BD46
:100BD00019190208EFF3058028B9EFF3108010B956
:100BE000EFF3118010B10348C0687047DFF808C008
:100BF00000DF7047806300207519020880B500F09F
:100C0000F8F8EFF3058028B9EFF3108010B9EFF38F
:100C1000118010B16FF0050080BDDFF808C000DF63
:100C200080BD00BF81190208EFF3058028B9EFF3FA
:100C3000108010B9EFF3118010B16FF0050070470C
:100C4000DFF804C000DF7047D11A0208F8B5144677
:100C50000E460546EFF3058028B9EFF3108010B972
:100C6000EFF31180F0B16FF003000DB303BBFEB1E1
:100C70002978FA291CD12846FFF709FE78B16A6A5B
:100C8000074600F10C013046FEF7FEFF0CB1F87884
:100C900020703846FD6000F06BFA0020F8BD6FF060
:100CA0000200F8BD2846DFF80CC03146224600DFBE
:100CB000F8BD00BF591B0208EFF305832BB9EFF312
:100CC000108313B9EFF311830BB100207047DFF8E5
:100CD00008C000DF704700BF391C02082DE9F04151
:100CE00090460D460646EFF3058028B9EFF31080D5
:100CF00010B9EFF3118018B36FF00307EEB1E3B949
:100D0000DDB13078FA2818D106F10C0000F0EBF8CC
:100D100088B1726A04460C302946FEF7B5FF0027F9
:100D2000F920C4E9015684F80380A770207020469A
:100D300000F01EFA01E06FF002073846BDE8F081CE
:100D40003046DFF80CC02946424600DFBDE8F0819E
:100D5000691D0208EFF305822AB9EFF3108212B978
:100D6000EFF3118212B16FF005007047DFF804C095
:100D700000DF7047291E0208EFF3058129B9EFF360
:100D8000108111B9EFF3118109B100207047DFF82C
:100D900008C000DF704700BFBD1E0208EFF30581E9
:100DA00029B9EFF3108111B9EFF3118111B16FF08F
:100DB00005007047DFF804C000DF7047251F0208F8
:100DC000F8B5876804469FB13D4695F82320696AC7
:100DD000BF682046FFF724FD0028F4D006462846C9
:100DE00000F02DFB28463146002200F0C5FBEAE763
:100DF000F8BD7047F0B5002390B389B3032A2FD80C
:100E0000034653F8084F0F3121F007012546E61A33
:100E10005C6824F00307F61B8E4205D22C682B4633
:100E2000002CF3D100231BE0D0E900650D444560A0
:100E3000304450F8046CAE4202D2083845605C6819
:100E400054B1186824F00304E05041EA0200E118AC
:100E5000486019600B4602E041EA0200586008331E
:100E60001846F0BDB0B50022E8B1E1B100F10804C8
:100E7000A1F108020023944206D0254624682B469F
:100E8000002CF8D100220EE051F8045C446825F0F3
:100E90000305641B446013B11068186002E0002071
:100EA00041F8040C01221046B0BD08B1420702D03F
:100EB00000221046704700221829FAD311F00703C8
:100EC000F7D110B50A18A2F108038360002342F895
:100ED000083C8268102454600122C0E90014C360F9
:100EE000BDE81040E5E710B5002817D0014600F135
:100EF000140252E8000F10B9BFF32F8F04E003680B
:100F000042E8003404B1F4E740B1043151E8002F65
:100F1000531C41E8003404B1F8E710BD002010BDB7
:100F2000B0B500281ED0C2688A421BD802698A4226
:100F300018D900F1140213680B60BFF35F8F52E8F9
:100F4000003F0C689C42F6D142E8001505B1F2E77B
:100F5000043050E8001F4A1E40E8002303B1F8E7C0
:100F60000020B0BD6FF00300B0BDB0B50446002056
:100F7000ACB1A1B19AB193B10020C4E9001004F161
:100F8000080002FB01352CC0481E636120B199188E
:100F9000196001380B46F9E7002018600120B0BD48
:100FA000F8B50446807868B3E56821462846FFF71F
:100FB000BAFC002005F10C06207030462146FFF7F0
:100FC000AFFFA868E8B13046FFF78DFFC8B104460F
:100FD000284600F015FA002100220646002700F0FE
:100FE000CBFA304600F06CFA81686A6A064604F172
:100FF0000C00FEF749FEF920A7702070F068E07041
:1010000025E0F8BDA568A86808B3407883281ED1FC
:10101000284600F0F5F9002100220646002700F0DE
:10102000ABFA304600F04CFA064680686A6A04F172
:101030000C01FEF729FEF06808B1E1780170277015
:1010400005F10C002146BDE8F840FFF769BF2846CE
:101050002146BDE8F840FFF73ABC2DE9F0410446CF
:1010600000274FF00108D4B12546E87864690007ED
:10107000F9D52F76A8680028F5D0284600F0C0F9E9
:1010800000210022064600F077FAC5E90367F06AFE
:10109000686100B1056185F81880F562E3E7BDE895
:1010A000F081B0B5C278920715D5C068C36A90F8D0
:1010B00021209C688C4208BF8C682CB194F9204098
:1010C00055B2AC42C8BFE2B25B69002BF1D190F8D7
:1010D0002010914200D1B0BD80F82020BDE8B04082
:1010E00000F0BDB970B5214C04F1560504F15A0663
:1010F000B4F85400D5E85F1F11B9BFF32F8F04E097
:101100004A1EC5E8532F03B1F4E7090429D0D6E8F5
:101110005F1F4A1C904200D80022C6E8532F03B13B
:10112000F5E788B2E16D51F82000D0B10178F139CE
:101130000829DDD8DFE801F006050905050C0F05D3
:101140001200D5E7216E8847D2E7616E8847CFE766
:10115000A16E8847CCE7E16E8847C9E7216F8847D1
:10116000C6E70020BDE8704000F0F2B880630020C0
:1011700070B50146194800F15603B0F85420D3E881
:101180005F4FA24202D8BFF32F8F04E0651CC3E873
:10119000565F06B1F3E7A3B2934214D200F15803AD
:1011A000D3E85F4F651CAA4200D80025C3E8565F0C
:1011B00006B1F5E7C36DA2B243F82210417A39B106
:1011C0000121817270BD0220BDE87040FEF702BDB2
:1011D00003484FF08051016070BD00BF8063002064
:1011E00004ED00E010B58168B1B100F10C01D1E867
:1011F0005F2F12B9BFF32F8F04E0531EC1E8543F95
:1012000004B1F4E7110407D000F0FAF8002100223D
:10121000BDE8104000F0B0B910BD000010B50121CC
:1012200041700B4990F920301C310A46896841B160
:1012300091F920409C42F8DCC0E9021290600C3128
:1012400004E00021C0E9021202F10801086010BDAB
:1012500080630020B0B54A1C0DD01A4A00242C32FD
:1012600015462B68DBB1DD69A9421AD3491B03F18E
:1012700010051C46F5E71349002330310C461A4689
:10128000236803F11004002BF9D14FF0FF33C36141
:101290000023C0E904329AB102F1100110E00025E8
:1012A00000E00125002CC0E90434C16118BF04F13D
:1012B000100210602DB1DA69511AD96103F11401DD
:1012C0000860B0BD80630020C2690169531C0AD068
:1012D00021B143694B61CB691A44CA6142693AB989
:1012E0000748C162704709B142694A6142691AB14F
:1012F000002343611161704701480163704700BFDB
:101300008063002070B5114DEC6A1CB1E0690138B2
:10131000E06100D070BD042660781338B6EB301F52
:1013200005D1204600F095F82146FFF7BAFE204689
:1013300000F085F8204600F0B9F8246924B1E0698E
:101340000028E9D000206061EC6270BD806300205D
:10135000B0B5054613484469017A65B1022905D143
:1013600094F9200095F92010814211DC2846BDE84F
:10137000B04000F09BB8022912D1456A85B194F9BA
:10138000200095F9201081420ADD284600F057F828
:101390002046FFF743FF2846BDE8B04000F0C8B83C
:1013A000B0BD00BF8063002010B50446002020803F
:1013B000A07881070DD5C00605D41048216B406F79
:1013C000FFF750FD05E00D48216BD0F88400FFF7D2
:1013D000A7FDA078C00708BF10BD0849D1F8880054
:1013E00020B12146BDE81040FFF79ABDD1F880003A
:1013F0002146BDE81040FFF735BD00BF80630020E7
:101400000146806882688A6002B1D1600021C160B3
:10141000704710B591F920300246806840B190F9CC
:1014200020409C42F8DAC1E9020291600C3004E0ED
:101430000020C1E9020202F10800016010BDC1688C
:1014400031B182688A60826802B1D1600021C160D6
:1014500070470178F12918BF7047C068F9E7B0B547
:101460000446054625B12878F12802D1ED68F9E750
:10147000B0BD2046FFF7E3FF28462146BDE8B04057
:10148000FFF7C7BF10B50446407833280DD194F854
:101490002320616A2046FFF7ACFA30B101462046AE
:1014A0000022BDE8104000F067B810BD01460120E1
:1014B000487002481C30FFF7ACBF00BF80630020BB
:1014C000806B2030704700000748416939B1086BD4
:1014D0008A6B824204D90068044A904200D1704766
:1014E0000120FEF777BB00BF80630020A52E5AE2E3
:1014F00070B50B4C0B48A26D666E002100F034FEF7
:10150000094DA8624EB1E26D0848002100F02CFEA2
:10151000A864002818BF012070BD012070BD00BF65
:10152000084B0208D1FB0108806300200D16020859
:101530000249886102214170FFF7C6BF8063002025
:1015400010B50C4C0246237A0020022B11D1636A9D
:101550007BB160694270FFF77DFE606A81686162FD
:1015600011B104F11C02CA600021C160FFF7E0FF65
:10157000012010BD80630020B0B50446806B154685
:1015800001622046FFF7A0FE20461DB1BDE8B04035
:10159000FFF7DEBEBDE8B040FFF788BFB0B5FFF78C
:1015A000D1F9194DE968286D0131E96000B1804732
:1015B000FFF7A8FE0020FFF7CBFE296C11B3AA6944
:1015C000A86B90421CBFC5E90E21B0BDE96B11B1FB
:1015D0000139E96316D1297A022913D16C6A8CB1D9
:1015E00090F8200094F8201081420BD12046FFF79C
:1015F00026FFA86BFFF75AFF2046FFF799FF286CDC
:10160000C5E90E40B0BD00BF8063002082B00B482A
:101610000821D0E91820FFF74FFB094D09496C4616
:10162000C5E91301214600224FF0FF33FFF70EFBFF
:1016300010B9DDE900108847E86CF3E7084B0208B1
:10164000806300204916020870B5134D6C6C14B30A
:101650002069012601382061ECB12069D8B9E06821
:1016600008B1A16881606864E86C04F11801002287
:101670000023FFF733FB18B103202146FEF7AAFA37
:10168000E078012804D161692046FFF7E9F900E01C
:1016900066706C6CE0E770BD80630020EFF305823C
:1016A0002AB9EFF3108212B9EFF31182CAB16FF0C9
:1016B0000302A0B199B90178F62910D10C30D0E815
:1016C0005F1F11B9BFF32F8F04E04A1EC0E8532FEC
:1016D00003B1F4E70022080408BF6FF002021046CD
:1016E0007047DFF808C000DF704700BFD91F02084D
:1016F000EFF305832BB9EFF3108313B9EFF31183E5
:101700000BB100207047DFF808C000DF704700BF52
:101710003120020810B50446EFF3058028B9EFF335
:10172000108010B9EFF3118090B15CB12078F628E9
:1017300008D12046FFF746F938B12046FFF718FDDB
:10174000002010BD6FF0030010BD6FF0020010BD4F
:101750002046DFF808C000DF10BD00BFB12002083E
:10176000DFF804C000DFFEE7E9200208EFF305819F
:1017700029B9EFF3108111B9EFF3118111B14FF0D5
:10178000FF307047DFF804C000DF704751210208C6
:10179000EFF305832BB9EFF3108313B9EFF3118344
:1017A0000BB100207047DFF808C000DF704700BFB2
:1017B00069210208EFF3058129B9EFF3108111B90E
:1017C000EFF3118111B16FF005007047DFF804C02D
:1017D00000DF70473923020830B180B5014613207D
:1017E000FFF7AEFEBDE880400020704710B588B11D
:1017F00002466FF0030000290BD41378F32B08D1B5
:101800000C3252E8000F20EA010342E8003404B130
:10181000F7E710BD6FF0030010BD20B10178F32988
:1018200004BFC068704700207047000010B550B179
:1018300001460468806870B182070FD1CA68002130
:10184000102A15D221E000241149D1F8900038B1B6
:10185000FFF749FB0AE0C8680028F5D0002114E032
:10186000D1F8800010210122FFF7C4FA58B10121FC
:101870000022C0E90142C2608170F3210170044975
:10188000044A4A6600E000200146084610BD00BF39
:1018900080630020C10D02082DE9F041002831D0FD
:1018A00005466FF00300002934D42A78F32A31D199
:1018B00005F10C0050E8002F42EA010440E8004323
:1018C00003B1F7E7A046AC6804B3264696F8232098
:1018D000716AA4682846FEF7A3FF0028F4D00746E3
:1018E00096F82300800738465CBF706A27EA00003C
:1018F00080463046FFF7A3FD304639460022FFF709
:101900003BFEE1E76FF00300BDE8F0810020FFF748
:101910001FFD4046BDE8F081F8B580B10C46064693
:101920006FF00300002909D43178F32906D130463D
:1019300021461F461546FEF773FF18B1F8BD6FF03C
:101940000300F8BD87B143203946FFF7F9FD40B1E8
:101950000748476930463946FFF75BFD87F8235053
:101960007C626FF00100F8BD6FF00200F8BD00BFAF
:10197000806300200148C068704700BF806300207A
:101980002DE9F8434F4F387A30B1012800F09680A6
:101990004FF0FF30BDE8F88307F108009C21FEF707
:1019A0008CF9DFF82481B8F81000D8E90B41A7F8CA
:1019B0005400D8E90202FA6538642046FFF775FA48
:1019C00008B1C7F88040D8E90541DFF80091D8E9AF
:1019D00007562046C847D7F88010002818BF214670
:1019E000796728463146C847D7F88010002818BFC5
:1019F0002946B967D8E909412046C847D7F8801079
:101A0000002818BF2146D8F83440F9673CB1216856
:101A1000D4E902232046FFF7A8FAC7F88440D8F893
:101A200038403CB12168D4E902232046FFF79DFAF3
:101A3000C7F88840D8F83C403CB12168D4E902237B
:101A40002046FFF792FAC7F88C40D8F840403CB1E6
:101A50002168D4E902232046FFF787FAC7F89040AF
:101A6000D8F844403CB12168D4E902232046FFF76E
:101A70007CFAC7F89440D8F848403CB12168D4E9D2
:101A800002232046FFF771FAC7F89840D8F84C4077
:101A90003CB12168D4E902232046FFF766FAC7F873
:101AA0009C40D8F850403CB12168D4E9022320463C
:101AB000FFF75BFAC7F8A040012038720020BDE8AC
:101AC000F88300BF80630020084B0208AB0E0208B9
:101AD000B0B51D4C207A01281CD1FFF709FDC8B113
:101AE0001A48FF218175817D026881F0FF01B1FAFA
:101AF00081F1C1F12001C2F302228A4228BF511CA8
:101B0000FE2202FA01F1124DC17468681149FEF714
:101B100039FF10B14FF0FF30B0BDFEF72FFF20614D
:101B2000FEF716FF04F11C00FFF76AFCFFF700FD4B
:101B30002878C0070CBF0320022080F314880220FD
:101B400020720020B0BD00BF806300200CED00E0DB
:101B5000084B020871FC01082DE9F84300284CD01D
:101B60000F466FF00305002949D004460078FA2893
:101B700045D1204699469046FEF789FE002841D07F
:101B8000064620463146FEF7CEFE626A06F10C019B
:101B90003846FEF779F8B8F1000F1CBFF07888F8E6
:101BA000000004F10C070025384631463570FFF778
:101BB000B7F9A06818B33846FFF795F90025F0B1DA
:101BC00006462046FFF71CFC002101220746FFF7CE
:101BD000D3FC3846FFF774FC8168626A074606F159
:101BE0000C00FEF751F8F920B5703070F8683146F6
:101BF000F0702046FEF76BFE01E06FF0030528460B
